:020000040800F2
:1000000010310020D9000008313F0008A10100088C
:1000100000000000000000000000000000000000E0
:10002000000000000000000000000000E5000008E3
:1000300000000000000000001F0100087D430008D0
:10004000EB000008EB000008453F0008EB0000084B
:10005000EB000008EB000008EB000008EB000008D4
:10006000EB000008D1220008312300080000000046
:100070009D1300080000000000000000EB000008D5
:10008000EB000008EB000008EB000008EB000008A4
:10009000EB000008EB00000800000000EB00000887
:1000A000EB00000835470008B945000899460008EC
:1000B000253D0008EB000008EB000008EB000008FD
:1000C0000448854600F04CFC00F0B2FA00480047B6
:1000D000911300081031002004488047044800476D
:1000E000FEE7FEE7FEE7FEE7FEE7FEE71144000855
:1000F000C1000008EFF3108072B6704780F31088DB
:1001000070472A4A1368012B03D001231360284A41
:100110001060284A11602848284901607047EFF3B1
:10012000108272B62148016800291DD000210160AB
:100130001F48016800290AD0EFF3098120390068BF
:100140000160F0C144464D4656465F46F0C119492C
:1001500009680968F0C9F0B4F0C9A046A946B246DA
:10016000BB46F0BC81F3098882F31088042040422A
:100170000047104908600E49002008600B49012023
:1001800008600F480F490268114301600A480B4993
:1001900001600D480068006880F3088862B6704707
:1001A000EFF3098000B509F047FB00BD741A002089
:1001B000CC170020D017002004ED00E00000001054
:1001C00020ED00E00000FFFF08ED00E0F0B51FB4F7
:1001D0000646002082B005464024019100901BE0B5
:1001E000019922460F46304600F0A7FA049A059B73
:1001F000801A994110D310461946224600F08DFA14
:10020000361A8F410197224601200021009F00F0FD
:1002100084FA38184D4100902046641E0028DFDC27
:10022000019B00982946324607B0F0BD30B54343E4
:1002300051435C18010C130C0D465D432C1980B220
:1002400092B20546554351430A0C09044D196241C7
:100250005843010C00044019514130BD10B5431AF8
:10026000934209D28318881803E0401E01785B1E70
:100270001970521EF9D210BD03460B439B0703D0E1
:1002800009E008C9121F08C0042AFAD203E00B785B
:100290000370401C491C521EF9D210BDD2B201E0BD
:1002A0000270401C491EFBD270470022F6E710B5D1
:1002B00013460A4604461946FFF7F0FF204610BDD4
:1002C00010B5044605E00B780370401C002B00D0ED
:1002D000491C521EF7D2204610BDCAB2401E4178BA
:1002E000401C8A4202D00029F9D100207047421CEC
:1002F0000178401C0029FBD1801A704730B50446B4
:100300000020034600E05B1C934203D2E05CCD5C1E
:10031000401BF8D030BD30B505460020034600E054
:100320005B1C934205D2EC5CC85C201A01D1002C06
:10033000F6D130BD0FB400B58DB009900B9010A967
:1003400000200091C0430A9000200C9006480690BF
:10035000064807906A4609A80F9900F021FA0DB0E7
:1003600008BC04B018470000C1070008E1070008F6
:10037000FFB50027FF4383B000205C6801909E68B2
:100380001D46A9697F1C049888470090296A884700
:100390000028F6D10098401C0CD003204002844372
:1003A000002E19DD600614D500982B2809D02D28C1
:1003B0000FD103E00020C04307B0F0BD0120800250
:1003C0000443A9697F1C04988847761E0090002E7C
:1003D00002DD0098302803D00598002825D035E0AC
:1003E000012040020443A969761E7F1C04988847B7
:1003F0000090002E03DD782805D0582803D00598FA
:10040000002810D022E00598002801D010281DD126
:10041000012040028443A969761E7F1C0498884706
:100420000090102002E0082000E00A2005900DE076
:10043000012149020C43059A0199761E514308187F
:100440000190A9697F1C049888470090002E05DD63
:100450000599009800F08FF90028E9DAE969049815
:100460008847A00502D40120C043A5E7E00722D1B8
:10047000600611D56005019800D5404229680A1D23
:100480002A600968220501D5087014E0220701D509
:10049000088010E008600EE02868011D29600068EF
:1004A000210502D50199017005E02107019901D5C7
:1004B000018000E0016038467EE7FFB5002083B090
:1004C000009050680190916914460026976804983E
:1004D000884705460C990698084305D009E0A169AC
:1004E000761C049888470546216A284688470028D4
:1004F000F5D1681C03D00198C00704D017E0002094
:10050000C04307B0F0BD2068011D21600068009065
:100510000DE00198C00704D1009805700098401CB8
:100520000090A169761C7F1E049888470546002F1D
:100530001CDD681C1AD0069800280FD0E817C00EE2
:10054000401941118A0006994009511840012A1AA0
:100550000968012090400142DBD107E00C98002897
:10056000D7D1216A284688470028D2D0E16904986B
:1005700088470C98002807D1002E05DD0198C00798
:1005800002D1009800210170A068B84204DD0C98E7
:10059000002804D0002F02D00120C043B1E730462C
:1005A000AFE70000F7B5009C0F4600262578641CD5
:1005B000002D05D000F0D2F80068405DC007F5D1ED
:1005C0002B2D02D02D2D18D0641E39462046029ABC
:1005D00000F018F9002F04D03968A14201D1009928
:1005E00039607105022400290BDA4042002803DD3E
:1005F0000DF058FB0460A007FEBD012080020643F9
:10060000E3E70028F8DA0DF04DFB04600048FEBD7A
:10061000FFFFFF7F70B506460DF044FB04680546FA
:100620000A2200213046FFF7BDFF2C6070BD00009C
:100630007CB507480090074801900546009C04E0FF
:100640002046016808188047241DAC42F8D17CBDC3
:10065000FCFC000800FD000810B5002904DB0C4676
:100660000121C9074042A141002B04DB1C460123A4
:10067000DB075242A341101A8B4101D2012010BD69
:10068000002010BD10B5002904DB0C460121C9076C
:100690004042A141002B04DB1C460123DB075242F0
:1006A000A341101A8B4101D3012010BD002010BDC1
:1006B00010B5002904DB0C460121C9074042A141C5
:1006C000002B04DB1C460123DB075242A341801AA6
:1006D000994101D2012010BD002010BD70B5044623
:1006E000002903D000202022012310E0002801D09F
:1006F0000020C043C046C0460DE02546D5408D428F
:1007000005D30D469540641B1D469540401915467E
:10071000521E002DF1DC214670BD10B5202A04DBED
:100720000146203A9140002010BD914020239C1AA0
:100730000346E3401943904010BD10B5202A04DB66
:100740000846203AD040002110BD0B46D340D0408F
:100750002024A21A91400843194610BD0048704752
:10076000A0DD000810B50446FFF7F8FF0068005D43
:10077000C007C00F10BD3A2800D2303820230246EF
:100780009A43412A01D310463738884201D30020CA
:10079000C0437047026813785118016018467047CB
:1007A00010B5D16004495161044911620021116101
:1007B000114600F0EDF810BD950700086507000828
:1007C0004268002A08D001680B78491C002B03D02E
:1007D000521E06C0184670470121C160881E70472E
:1007E0004268002A0BD0C3680168002B07D18368D8
:1007F0008B4204D0491E521C06C0002070470020C6
:10080000C0437047F7B582B0029C00272078641C73
:1008100015460197302802D0002D15D015E020781C
:100820000127641C782804D0582802D0002D09D054
:100830000BE0002D01D0102D07D1002710252078C6
:10084000641C02E0082500E00A250026009610E05E
:100850000099012769430818020C294680B27143A8
:1008600000908E183804864201D301200190207830
:10087000641C2946FFF77FFF0028E9DA0398002867
:1008800005D0002F01D0641E00E0029C0460019896
:10089000002806D00DF006FA02210160C81E05B03E
:1008A000F0BD009930040843F9E700000FB400B52B
:1008B00089B00A460DA9009100230C99002ACB604B
:1008C000234B0693234B079301D0042300E000231E
:1008D000214A0292214A0892019302466B46002067
:1008E00000F081FA09B008BC04B01847F0B585B033
:1008F00007460020C04301901E46002015460C46C6
:100900000091029104903B466A46314604A8FFF7E5
:10091000CDFF049902466018002D05D0002901D0B2
:10092000034600E023462B6000290ED0002A02DD9A
:100930000099814209D0001B019000943B466A4611
:100940003146029404A8FFF7B1FF05B0F0BD0000E6
:10095000C1070008E1070008FFFFFF7F65070008E7
:100960001CB5094800900948019005460126009CE5
:1009700005E0E36807CC33430C3C98471034AC42A5
:10098000F7D3FFF7A1FB0000DCFC0008FCFC00082B
:10099000F3B58DB000200A9001200B900026084688
:1009A0000C300C4609906269012109989047051E98
:1009B0002ED0252D2DD0216A8847002818D06269B5
:1009C000012109989047216A88470028F7D1411EE4
:1009D00062690998904700E0761CA1690D988847E4
:1009E000216A88470028F7D1E1690D988847DAE73E
:1009F000A1690D9888470746A84201D1761CD2E725
:100A0000E1690D9888477F1C02D10A98002877D0A9
:100A100049E1002762693D463946099890472A28EE
:100A20000CD16269012109989047012506E00A214D
:100A30004F433F18303FEBD410200543626901213A
:100A400009989047014630390A2903D29B498F42C1
:100A5000DEDCECE7E90600D4994F6C280AD04C287C
:100A600010D0682824D06A282ED074280CD07A2878
:100A70000AD00DE062690121099890476C2823D0C3
:100A800004211CE020200543626901210998904758
:100A9000A760656065284FD026DC582839D01ADC5D
:100AA000452849D012DC252834D04128B0D143E074
:100AB0006269012109989047682802D008210D43F6
:100AC000E6E70120C002DEE70220DCE7462833D05B
:100AD00047282CD130E05B2870D061282CD06328C7
:100AE0006CD0642823D161E06F284FD009DC6628E0
:100AF00022D0672820D0692826D06E2817D12EE072
:100B0000CDE070284DD073286FD075284ED078284E
:100B10000DD154E0A1690D9888470546252800D1DC
:100B20006CE7E1690D9888476D1C00D16DE7BAE06C
:100B30000A224CE00A2252E0012023466A46C043C2
:100B40000D9900F050F9A3E0284640210843606069
:100B5000A807234601D5002239E000223FE0E8073C
:100B600000D020E72068011D21600068290501D51B
:100B7000067018E7290701D5068014E7A90703D5F1
:100B8000F117066041600EE706600CE72846402139
:100B900008436060A807234601D5082217E0082211
:100BA0001DE0484928460840606016E0284640217C
:100BB00008436060A8072346BCD5B9E715E028467E
:100BC000402108436060A80707D523461022012072
:100BD000C0430D99C046C0465AE02346102201206A
:100BE000C0430D99FFF7C4FB52E000210C910B4666
:100BF0000091632802D05B2807D043E0E80601D4C7
:100C00000120A060012000903CE062690121099868
:100C100090475E2805D101200C9001466269099831
:100C200090472169002906D10B4601AA8F00491C73
:100C3000D3510829FADB002835D0216900290ED1CB
:100C4000C117C90E09184A11930001AA9A18490937
:100C50004901411A01201368884003431360626907
:100C60000121099890475D28E5D10C98002808D00B
:100C7000002001AB81005A58401CD2435A5008282A
:100C8000F8DB01AB01202246C0430D99FFF715FCAC
:100C900000280ADA401C06D10B98002803D0002057
:100CA000C0430FB0F0BD0A98FBE7E90702D10A99EB
:100CB000491C0A91361800200B9074E6CCCCCC0C61
:100CC000FFFFFF7FF1F7FFFFFFB5087889B01546FA
:100CD000FF2805D0491C2D2804D00022002407E05D
:100CE00000240BE00122F9E70A235C430419491CA4
:100CF0000878FF28F8D1002A00D064420020049030
:100D00002A7801462D2A01D02B2A0FD16D1C2D2ABD
:100D100002D00022049209E00122FBE700260A2209
:100D200033466D1CFFF782FA381871412F78FF2F78
:100D3000F4D10C9AA218069202460A4304D0FF236B
:100D4000069A9133DA4205DA002109980A4606C06C
:100D50000DB0F0BD0024B74AB54D2646079200F00D
:100D60004DFA029006980391002801DA474200E00C
:100D7000074639050020AF4A001C514101910090FF
:100D800012E0F80707D022462B463046079900F0BC
:100D900055F90646079122462B461046194600F0A3
:100DA0004DF904460D467F10002FEAD10698019BAD
:100DB0000028009A0399029806DA00F0A7F9324653
:100DC000079B00F0A3F905E000F038F93246079BD5
:100DD00000F034F9049A002A02D00122D2075140CF
:100DE000099A03C2B4E7FFB591B00020099000252D
:100DF000ED432E209E685C681F460190B9696D1C0A
:100E0000129888470090396A88470028F6D10098E0
:100E1000401C0AD00D20C0018443002E12DD009832
:100E20002B2809D02D280DD103E00020C04315B098
:100E3000F0BD012080020443B9696D1C12988847F7
:100E4000761E009003A9600501D52D2000E02B201F
:100E50006A461073491C0CA80F9102900AE0B96908
:100E60006D1C12988847009001204002044313989B
:100E7000761E0560002E02DD00983028EFD0019923
:100E80000098884245D18020044308E00998401E1C
:100E900009900120400204431399681C0860B96955
:100EA0006D1C761E1298884700903028EED030E0F6
:100EB0000199884205D1200603D480200443761E80
:100EC0001DE000980CF00EFF002825D001214902FA
:100ED0000C43009807AA0F9903323038761E9142CE
:100EE00008D208700F98401C0F90200607D509986B
:100EF000401E03E0200602D40998401C0990A0057A
:100F000002D51399681C0860B9696D1C129888474E
:100F10000090002ECCDC59E0002E57DD00986528AB
:100F200001D0452852D1A00550D5032000028443AA
:100F3000B9696D1C761E129888470090002E0CDD52
:100F40002B2804D02D2808D1FF2001300443B96993
:100F50006D1C12988847761E0090E00501D52D2162
:100F600000E02B21029801700298401C0290019031
:100F700025E00120400204430EA902980131761EAB
:100F800088420ED20098029930380006000E087090
:100F900003D10299019881420AD90298401C02901B
:100FA00006E0E00501D5244801E0234840420990CD
:100FB000B9696D1C12988847009013980560002E3F
:100FC00004DD00980CF08EFE0028D2D1F969129849
:100FD00088470F99FF200870029903AA0870002023
:100FE0000A900B900CA90AA8099BFFF76DFEA005BB
:100FF00002D40120C0431AE72420044209D0E007AC
:1010000013D138680B9A0A99031D3B60006806C02B
:101010000BE00B990A9800F0FFF80146E00704D1B5
:101020003868021D3A60006801602846FFE600004B
:10103000000014400000F03FF1D8FFFFF0B51FB4EE
:1010400088B00B990998002448400999C00F4900BD
:1010500049080991C0070B990090490049080B9174
:1010600009990898A64608431CD00B990A9808438A
:1010700018D0099801244000420D4800410D0998FC
:1010800024050003000B204309900B980003000B7C
:1010900020430B9050181C49401800220190144620
:1010A000104605E0002001460DB0F0BD032801DA2E
:1010B000034600E003239C46C11A0AAE0AE05F0023
:1010C00008ADED5B4F00F75B7D430027AA187C411C
:1010D000491C5B1E6145F2DD410004AB5A522104FC
:1010E000120C0A43240C401C0828DFDB01980290F4
:1010F0000099704601910090059B049A0799069803
:1011000000F0F4F8D0E700000DFCFFFFF0B50C464E
:101110005C4085B0E40FE40703944C0000266408AB
:1011200059009446490802460296224321D062465D
:101130000A431ED06200570D4A000E032303550DCB
:10114000012402462C492405781B1B0B360B401842
:1011500023432643614600901C46501AB44103D3F2
:101160000098401C009002E0921800985B41002813
:1011700003DA0020014605B0F0BD00200121090579
:101180000746864611E064461D46141BB54106D34A
:101190006546521BB341744607430C43A646CD0730
:1011A00040084908284392185B4105460D43EAD19F
:1011B0001046184313D0604619465040714008430A
:1011C00006D06046101AB34106D20122002306E081
:1011D00000220123DB0702E00122D24353100098D2
:1011E00074460105381C6141029C039D0019694148
:1011F00000F06FF8BFE70000FD0300000EB5054AE0
:101200000292002200921346019200F06FF803B0A0
:1012100000BD000033040000CB0FDB07490010B510
:10122000490802460A4307D00A0D07240903E401CE
:10123000090B121B002A01DC002010BDC900440F5D
:101240000C43C100E018D205801800F001F810BD71
:10125000002904DA401C490001D1400840007047D1
:1012600070B40024050C05D11024000402D100291B
:1012700021D01124050E01D100020834050F01D13F
:101280000001241D850F01D18000A41C002801DB72
:101290004000641C002908D020252E1B0D46F54077
:1012A000A14000D001212943084301061B1B000A6D
:1012B000DB1D02D5002070BC7047DB0518188018B4
:1012C0000029F8DA401C4900F5D170BC4008400004
:1012D000704710B5002B08DA0024401C61419218B9
:1012E0005B411A4301D14008400010BDF0B51FB466
:1012F00082B005460C0003D008460CF0BBFC02E0AF
:101300000CF0B8FC20300246009021462846FFF73A
:1013100004FA049B059A04460F46184311430843F8
:1013200014D0184610431BD0009840210A1A1846C2
:101330000599FFF702FA05460E46009A05990498AA
:10134000FFF7EBF9084305D0012004E020463946B9
:1013500007B0F0BD0020C11705430E432C433743AF
:1013600000990E986305401A7905E40A00220C439F
:10137000FD0A0A3002D500200146E9E701051019EF
:1013800069410C9C0D9D00196941FFF7A2FFDFE741
:1013900080B50BF013F9002080BD000080B508F087
:1013A0003DFB0B484168490704D50168490701D551
:1013B000042101604168090607D50168090604D5C2
:1013C00080210160034809F059FB08F041FB80BD12
:1013D0001024014024010020F0B587B0274C20786C
:1013E000002833D1201D2649002207F097FE012056
:1013F000C104820443040504E56623676267A167AC
:10140000C10306918103059143030503C6028702C8
:1014100041020202E26421656765A665E56523660F
:10142000059961660699A1668021069140222023D4
:101430001025082604270221E06221636763A66362
:10144000E563236462640699A164207032200390EE
:10145000142002900B4800900320400201900A4C97
:101460000AA10E4A002520462B460AF081F82046A4
:101470000AF060F9284607B0F0BDC0469000002091
:10148000ADE70008CC0800203C080020616C6172C8
:101490006D5F74687265616400000000A11400084B
:1014A00088B0F04801680901EF4905D4EF48017898
:1014B00001290ED1016B08E0491C02680A43026051
:1014C000EA480178012904D1C16A001D07F06AFFCA
:1014D00002E0E74808F0CEFA7D20C000019000202D
:1014E0000290C643E14D039602E0E14808F0C2FADB
:1014F0002F462C37D0CFAB6BE86B0490286C05904F
:10150000686C0690E96C286D07AA0092214331436C
:10151000039E39431943049A11430143059801433B
:10152000069801432F1D062438462246334607F00D
:1015300019FE0028DCD1E96A079801420FD0072084
:101540000122CC49CCA30CF0CDFA0298687005209A
:1015500001F034FF28780128C7D1296B3AE0296BC4
:1015600001423BD0072006900124C2492246C6A36F
:101570000CF0B8FA6878A8706C70C74E306803F049
:1015800069FF306804F086F8C44E306803F062FFEB
:10159000306804F07FF8C24E3068C249039A04F004
:1015A00027F8306804F028F8BF480AF031F80698A8
:1015B000B0492246BDA30CF095FAC04E3068C04930
:1015C000224604F015F8306804F016F8287801284F
:1015D0008BD1696B384607F0E5FE89E7696B0142FC
:1015E0002DD007200122A349B6A30CF07BFA68781E
:1015F000A87002206870A84C206803F02BFF2068B8
:1016000004F048F8A54C206803F024FF206804F09B
:1016100041F8A34C206804F03DF8206803F036FF41
:10162000A878012800D063E7019809F006FEA34CD2
:10163000206803F00FFF206804F02CF858E7A96B2E
:10164000014244D0072001248A492246A2A30CF07B
:1016500049FA6878A8700320687010270021069165
:10166000384609F0DFF86426304609F0D1FF3846E5
:10167000214609F0D7F8304609F0CAFF112021466B
:1016800009F0D0F8069801F099FE854C206803F027
:10169000E1FE206803F0FEFF804C206803F0DAFED4
:1016A000206803F0F7FF7C4C20688FA1039E324630
:1016B00003F09EFF206803F09FFF804C206879496B
:1016C000324603F095FF206803F096FF10E7E96BC0
:1016D00001422AD00726012430466649224684A3C7
:1016E0000CF000FA6878A87004206870204601F0B9
:1016F00065FE30465F49224682A30CF0F3F91120C3
:10170000002109F08FF830465A49224681A30CF097
:10171000E9F96A4C206803F09DFE206803F0BAFFE7
:101720002878012800D0E0E653E7296C014223D055
:10173000072001224F497C4B0CF0D4F96878A8703F
:1017400005206870544C206803F084FE206803F084
:10175000A1FF534C206803F07DFE206803F09AFF40
:101760004E48006803F092FE022001F027FE534C21
:1017700020686EA1039AA4E7696C01420CD007208F
:1017800001223C496D4B0CF0ADF96878A8706C7083
:10179000032001F013FEBCE7E96C01422DD1296D55
:1017A000014216D00720012232496A4B0CF09AF907
:1017B0006878A8700920687003F040F8287801283C
:1017C00000D092E6A878132815D880002818C16A9E
:1017D00000E7A96C014200D18AE6072401222046D5
:1017E00024495D4B0CF07EF96878A8706C70062077
:1017F00001F0E4FD7CE60021ECE607201D4C01260B
:101800004F4B214632460CF06DF96878A8700820DD
:101810006870042001F0D2FD03204A4B2146324675
:101820000CF060F9484D104E019F029C781E08F0A4
:10183000C7F80094072001220E492B460CF052F9FC
:10184000641CA642F2D1384609F0E2FEBFF34F8F86
:101850003E483F490160BFF34F8F00BF00BF00BF4C
:1018600000BFFAE744100240FFFF00009000002094
:1018700010E70008A8E70008E4B88AE794B5E6A8EE
:10188000A1E5BC8F0A000000E9A284E783ADE6A8C9
:10189000A1E5BC8F0A000000140100201C010020FB
:1018A0001801002099E7000888130000E9A284E7E6
:1018B00083ADE5AE8CE688900A0000002001002090
:1018C00086E70008E6ADA3E5B8B8E6A380E6B58BE9
:1018D000E6A8A1E5BC8F0A00E68AA5E8ADA6E6A8C1
:1018E000A1E5BC8F0A0000003230302C32303000CD
:1018F000E68AA5E8ADA6E681A2E5A48DE6A8A1E565
:10190000BC8F0A00E585B3E997ADE9A38EE69CBAE2
:101910000A000000E585B3E997ADE89C82E9B8A329
:10192000E599A80A000000006AE70008323030306C
:10193000302C3230303030300000000056E70008E4
:1019400078E70008B9E70008A1E700080CED00E01F
:101950000400FA0531E700083FE7000806200549C2
:10196000012205A30CF0BEF804F024FD142009F0B8
:101970004FFEF9E732ED0008627574746F6E5F73A5
:1019800063616E5F7468726561640D0A0000000037
:10199000F0B583B0024E3068002809D502E0C04699
:1019A0001420024030460C38FE490160FE490160B7
:1019B0007B2500950720FD490124FD4B22460CF0B4
:1019C00091F8FEF797FBFB4F3860022029460AF09A
:1019D00067FE05463868FEF791FBE107306808436B
:1019E0003060002D00D0D0E102913068002805D58C
:1019F00030460C38EB490160EB4901607C250095CD
:101A00000720EA490122EA4B0CF06CF8FEF772FB62
:101A1000E84F3860022029460AF042FE0546386841
:101A2000FEF76CFB3068029908433060002D00D04F
:101A3000ABE13068002805D530460C38D949016043
:101A4000D94901607D2500950720D8490122D84B4E
:101A50000CF048F8FEF74EFBD64F386002202946BE
:101A60000AF01EFE05463868FEF748FB306802990A
:101A700008433060002D00D087E13068002805D58C
:101A800030460C38C7490160C74901607825009588
:101A90000720C6490122C64B0CF024F8FEF72AFBAA
:101AA000C44F3860022029460AF0FAFD054638681E
:101AB000FEF724FB3068029908433060002D00D007
:101AC00063E13068002805D530460C38B54901601F
:101AD000B5490160792500950720B4490122B44B2E
:101AE0000CF000F8FEF706FBB24F386002202946E2
:101AF0000AF0D6FD05463868FEF700FB306802990B
:101B000008433060002D00D03FE13068002805D543
:101B100030460C38A3490160A34901607A2500953D
:101B20000720A2490122A24B0BF0DCFFFEF7E2FAEC
:101B3000A04F3860022029460AF0B2FD05463868F9
:101B4000FEF7DCFA3068029908433060002D00D0BF
:101B50001BE13068002805D530460C3891490160FA
:101B60009149016076250095072090490122904B0C
:101B70000BF0B8FFFEF7BEFA8E4F38600220294600
:101B80000AF08EFD05463868FEF7B8FA306802990B
:101B900008433060002D00D0F7E03068002805D5FC
:101BA00030460C387F4901607F49016077250095F8
:101BB00007207E4901227E4B0BF094FFFEF79AFA34
:101BC0007C4F3860022029460AF06AFD05463868D5
:101BD000FEF794FA3068029908433060002D00D077
:101BE000D3E03068002805D530460C386D490160D7
:101BF0006D4901607425009507206C4901226C4BEA
:101C00000BF070FFFEF776FA6A4F38600220294623
:101C10000AF046FD05463868FEF770FA306802990A
:101C200008433060002D00D0AFE03068002805D5B3
:101C300030460C385B4901605B49016075250095B1
:101C400007205A4901225A4B0BF04CFFFEF752FA7B
:101C5000584F3860022029460AF022FD05463868B0
:101C6000FEF74CFA3068029908433060002D00D02E
:101C70008BE03068002805D530460C3849490160B2
:101C80004949016072250095072048490122484BC7
:101C90000BF028FFFEF72EFA464F38600220294647
:101CA0000AF0FEFC05463868FEF728FA306802990B
:101CB00008433060002D68D13068002805D53046D3
:101CC0000C383849016038490160732500950720B8
:101CD00036490122364B0BF005FFFEF70BFA354F64
:101CE0003860022029460AF0DBFC05463868FEF71A
:101CF00005FA3068029908433060002D45D13068FC
:101D0000002805D530460C38264901602649016077
:101D100070250095072025490122254B0BF0E2FE96
:101D2000FEF7E8F9234F3860022029460AF0B8FC94
:101D300005463868FEF7E2F93068029908433060DA
:101D4000002D22D13068002805D530460C381549C1
:101D50000160154901607125009507201349012292
:101D6000134B0BF0BFFEFEF7C5F9124F386002208F
:101D700029460AF095FC05463868FEF7BFF9306839
:101D8000029908433060002D08D0032007490AA3B8
:101D900022460BF0A7FE204603B0F0BD00242046EB
:101DA00003B0F0BD851A7AE591836E7CB0EB000834
:101DB000F7EA000844170020466C6173685F4572BB
:101DC000617365506167655F5265636F726473200C
:101DD0006661696C65640D0A00000000F0B5FFB033
:101DE00082B0334E3068334CA04249D001A8143041
:101DF0007B218900FEF759FA322005900A200490D1
:101E00002D4803902D4802900194FFF7C1FD2C4905
:101E10000868002805D508460C382A4901602A4977
:101E200001607F250095072028490124284B224680
:101E30000BF058FEFEF75EF9264F38600220294667
:101E40000AF02EFC05463868FEF758F9E0071C4AF0
:101E5000116801431160002D05D003201B490122A8
:101E60001D4B0BF03FFE0025802701A84159A81902
:101E700001F00AFA002808D17F1E2D1D002FF4D191
:101E8000002420467FB002B0F0BD03250F4E134B57
:101E90002846314622460BF025FE11A3284631463E
:101EA00022460BF01FFE20467FB002B0F0BDC046B8
:101EB00000FE0008A5A4A3A21A6210141062100A62
:101EC00014200240851A7AE591836E7CB0EB0008FD
:101ED000F7EA00084417002068E900088EEB0008C4
:101EE000466C6173685F57726974655F436F6E66B5
:101EF0006967496E666F206661696C656400000001
:101F000070B584B0154800210A4608F05BFD1449FD
:101F10000860002805D103201249012212A30BF00A
:101F2000E1FD052003900A2002901548009001244D
:101F3000A0020190134E14A1164A002530462B46EC
:101F400009F016FB304609F0F5FB0620054912A3FF
:101F500022460BF0C7FD284604B070BD4EE80008CD
:101F60001012002058E8000868725F72785F73658D
:101F70006D20637265617465206661696C656400DB
:101F8000A41200201412002068725F7468726561E8
:101F9000640000006D3B00084253505F48525F49A7
:101FA0006E69740070B513200F4D002421462A4637
:101FB000234603F0BDF80D4E3060142021462A461A
:101FC000234603F0B5F87060152021462A462346C3
:101FD00003F0AEF8B060122001212A46234603F038
:101FE000A7F8F060204670BD3DED00081401002008
:101FF000F0B583B00125A902484802460C3A13689F
:102000000B43136000BF00BF00BF290713680B43D9
:10201000136000BF00BF00BF2902414A13680B4391
:102020001360026802231343036002681023134302
:1020300008229343036002682A4302600268520741
:1020400008D40268520705D40268520702D4026815
:102050005207F3D5032200921202036893430B4305
:102060000360E90302680A4302602E4ECA27F76044
:102070005324F4600720400531688143680508183F
:102080003060E804316801433160274809F0C0FA44
:102090006803316801433160280431460C390A680D
:1020A000024208D00A68024205D00A68024202D001
:1020B00009680142F1D11D4830611D4802681D497F
:1020C0000A4002601C4A04231360F760F460341F66
:1020D00025681D4325600024F46005680D400560F7
:1020E0001360F4601548019001A80AF08FFD0028E4
:1020F00000D0FEE702A805218170009941701421EB
:1021000001700AF0F1FD002800D0FEE70C49C81C60
:1021100000F034F8002003B0F0BDC046401002408B
:102120000070004018280040B80B0000EB81000050
:1021300000E400E0FFFF00FF00E100E005082324C9
:102140000C01002010B582B01C466B46D8709A7006
:1021500059700698187018460AF058FD002800D0EB
:10216000FEE70599049A01A88170427004700AF094
:10217000BBFD002800D0FEE702B010BDF0B582B074
:1021800000910190284D2B686A68284C07200106B1
:102190002E686D68B3420ED116462640D002084024
:1021A00030430C46E902214F3D40214029438842FB
:1021B00021461E4C29D01C4D2B686A6828686D6822
:1021C00083420ED116462640D002084030430C46CA
:1021D000E902164F3D402140294388422146134CD5
:1021E00013D0114D2B686A6828686D6883421AD134
:1021F00016462640D002084030432C4027460C4665
:10220000E9022140394388420DD100998B70180AA8
:102210004870180C087001998A70300A4870100CC8
:10222000087002B0F0BDFEE700280040FF1FFFFF6E
:1022300010B584B01A48016801220A43026001689F
:10224000890708D40168890705D40168890702D481
:1022500001688907F3D513481349016005244460D8
:1022600012490160062012490122124B0BF03AFC80
:1022700003941E200290E00101900F4800900F4847
:102280000FA1124A002309F073F9002802D00020A0
:1022900004B010BD094809F04DFA002004B010BD8B
:1022A000441002400030004055550000CCCC0000E6
:1022B000C0ED0008C8ED0008902A0020002A002088
:1022C0007764675F746872656164000039DC0008D8
:1022D00010B507F0A3FB244C606840070BD5201F06
:1022E0000068400707D520680421014321601F488A
:1022F000006908F0C3FB606880070BD5201F0068E9
:10230000800707D520680221014321601748006932
:1023100008F0B4FB6068000707D5201F00680007BD
:1023200003D5206808210143216007F091FB10BD0F
:1023300010B507F073FB0C488169890711D5011F9F
:10234000096889060DD5016820220A430260074CFE
:10235000616920464C3005F08BFE0020606102F080
:102360000FFB07F075FB10BD040002407002002057
:10237000F0B58BB0471E062F35D814460D46F9B27E
:102380000AAE30462A4600F029FE7178B3783278DA
:10239000160909960396009701951D06AD0E08953E
:1023A00006951B0259181F270F4004970F26164049
:1023B000002802D1FD20C000361802968805C50EFF
:1023C000059507200949012209A30BF08BFB08980A
:1023D00060712571E7700998A0706670300A2070EE
:1023E00000200BB0F0BD01200BB0F0BDB0EB000839
:1023F00028256429466C6173685F4765745265637C
:102400006F72645B25645D3A253034642D2530326B
:10241000642D253032642C253032643A2530326404
:102420000000000070B50446012045028F4980225B
:1024300008463C3803685B1C00D111E10846383877
:1024400003685B1C00D10BE10846343803685B1C51
:1024500000D105E10846303803685B1C00D1FFE07D
:1024600008462C3803685B1C00D1F9E00846283880
:1024700003685B1C00D1F3E00846243803685B1C4A
:1024800000D1EDE00846203803685B1C00D1E7E08E
:1024900008461C3803685B1C00D1E1E00846183888
:1024A00003685B1C00D1DBE00846143803685B1C42
:1024B00000D1D5E00846103803685B1C00D1CFE09E
:1024C00008460C3803685B1C00D1C9E00846083890
:1024D00003685B1C00D1C3E0081F03685B1C00D1CC
:1024E000BEE00868401C00D1B9E0103A4031002A33
:1024F0009ED15F49802208463C3803685B1C00D1AE
:10250000AEE00846383803685B1C00D1A8E00846F6
:10251000343803685B1C00D1A2E0084630380368F9
:102520005B1C00D19CE008462C3803685B1C00D182
:1025300096E00846283803685B1C00D190E0084606
:10254000243803685B1C00D18AE008462038036801
:102550005B1C00D184E008461C3803685B1C7FD0FC
:102560000846183803685B1C7AD00846143803689C
:102570005B1C75D00846103803685B1C70D0084699
:102580000C3803685B1C6BD00846083803685B1C7A
:1025900066D0081F03685B1C62D00868401C5ED0D0
:1025A000103A4031002AA6D13248802102463C3AF6
:1025B00012680026521C65D00246383A1268521C36
:1025C00060D00246343A1268521C5BD00246303A60
:1025D0001268521C56D002462C3A1268521C51D036
:1025E0000246283A1268521C4CD00246243A12681D
:1025F000521C47D00246203A1268521C42D0024672
:102600001C3A1268521C3DD00246183A1268521CFD
:1026100038D00246143A1268521C33D00246103A9F
:102620001268521C2ED002460C3A1268521C29D055
:102630000246083A1268521C24D0021F1268521C2B
:1026400020D00268521C1DD0103940300029ADD175
:10265000032009490122094B0BF044FA12E0084615
:102660004159491C0CD000260CE0C0463CF600083D
:102670003CF800083CFA0008B0EB00087BE90008D1
:1026800040198608F0B22080EF49802208463C3885
:1026900003685B1C00D111E10846383803685B1CF5
:1026A00000D10BE10846343803685B1C00D105E11A
:1026B0000846303803685B1C00D1FFE008462C3820
:1026C00003685B1C00D1F9E00846283803685B1CEE
:1026D00000D1F3E00846243803685B1C00D1EDE02C
:1026E0000846203803685B1C00D1E7E008461C3828
:1026F00003685B1C00D1E1E00846183803685B1CE6
:1027000000D1DBE00846143803685B1C00D1D5E03B
:102710000846103803685B1C00D1CFE008460C382F
:1027200003685B1C00D1C9E00846083803685B1CDD
:1027300000D1C3E0081F03685B1C00D1BEE008683D
:10274000401C00D1B9E0103A4031002A9ED1BF4967
:10275000802208463C3803685B1C00D1AEE0084686
:10276000383803685B1C00D1A8E008463438036899
:102770005B1C00D1A2E00846303803685B1C00D126
:102780009CE008462C3803685B1C00D196E00846A4
:10279000283803685B1C00D190E0084624380368A1
:1027A0005B1C00D18AE00846203803685B1C00D11E
:1027B00084E008461C3803685B1C7FD00846183844
:1027C00003685B1C7AD00846143803685B1C75D01C
:1027D0000846103803685B1C70D008460C38036844
:1027E0005B1C6BD00846083803685B1C66D0081F6A
:1027F00003685B1C62D00868401C5ED0103A403110
:10280000002AA6D19248802102463C3A126800264E
:10281000521C59D00246383A1268521C54D0024613
:10282000343A1268521C4FD00246303A1268521C99
:102830004AD002462C3A1268521C45D00246283A29
:102840001268521C40D00246243A1268521C3BD0F7
:102850000246203A1268521C36D002461C3A1268D0
:10286000521C31D00246183A1268521C2CD0024633
:10287000143A1268521C27D00246103A1268521CB1
:1028800022D002460C3A1268521C1DD00246083A69
:102890001268521C18D0021F1268521C14D0026811
:1028A000521C11D0103940300029ADD103206949A4
:1028B0000122694B0BF016F906E008464159491C04
:1028C00001D0002600E08608F0B2608063498022D3
:1028D00008463C3803685B1C00D1B0E00846383835
:1028E00003685B1C00D1AAE00846343803685B1C0F
:1028F00000D1A4E00846303803685B1C00D19EE09C
:1029000008462C3803685B1C00D198E0084628383C
:1029100003685B1C00D192E00846243803685B1C06
:1029200000D18CE00846203803685B1C00D186E0AB
:1029300008461C3803685B1C00D180E00846183844
:1029400003685B1C7BD00846143803685B1C76D098
:102950000846103803685B1C71D008460C380368C1
:102960005B1C6CD00846083803685B1C67D0081FE6
:1029700003685B1C63D00868401C5FD0103A40318C
:10298000002AA5D13649802002460B463C3B1B68F5
:102990005B1C68D00B46383B1B685B1C63D00B4646
:1029A000343B1B685B1C5ED00B46303B1B685B1CDA
:1029B00059D00B462C3B1B685B1C54D00B46283B64
:1029C0001B685B1C4FD00B46243B1B685B1C4AD02A
:1029D0000B46203B1B685B1C45D00B461C3B1B6811
:1029E0005B1C40D00B46183B1B685B1C3BD00B4666
:1029F000143B1B685B1C36D00B46103B1B685B1CF2
:102A000031D00B460C3B1B685B1C2CD00B46083BA3
:102A10001B685B1C27D00B1F1B685B1C23D00B683B
:102A20005B1C20D0103A4031002AAED10320094966
:102A30000122094B0BF056F8002014E008464159DA
:102A4000491C0FD080200EE03CF000083CF200084A
:102A50003CF40008B0EB00087BE900083CEC0008FF
:102A60003CEE000880082071BE49802208463C38B0
:102A700003685B1C00D1B0E00846383803685B1C73
:102A800000D1AAE00846343803685B1C00D1A4E0FA
:102A90000846303803685B1C00D19EE008462C389D
:102AA00003685B1C00D198E00846283803685B1C6B
:102AB00000D192E00846243803685B1C00D18CE00A
:102AC0000846203803685B1C00D186E008461C38A5
:102AD00003685B1C00D180E00846183803685B1C63
:102AE0007BD00846143803685B1C76D00846103843
:102AF00003685B1C71D008460C3803685B1C6CD003
:102B00000846083803685B1C67D0081F03685B1C15
:102B100063D00868401C5FD0103A4031002AA5D12C
:102B20009149802002460B463C3B1B685B1C5AD0F7
:102B30000B46383B1B685B1C55D00B46343B1B686F
:102B40005B1C50D00B46303B1B685B1C4BD00B46CC
:102B50002C3B1B685B1C46D00B46283B1B685B1C50
:102B600041D00B46243B1B685B1C3CD00B46203BF2
:102B70001B685B1C37D00B461C3B1B685B1C32D0B0
:102B80000B46183B1B685B1C2DD00B46143B1B6887
:102B90005B1C28D00B46103B1B685B1C23D00B46EC
:102BA0000C3B1B685B1C1ED00B46083B1B685B1C68
:102BB00019D00B1F1B685B1C15D00B685B1C12D057
:102BC000103A4031002AAED10320FD490122FD4BCD
:102BD0000AF088FF002006E008464159491C01D050
:102BE000802000E080086071F749802208463C3868
:102BF00003685B1C00D1B0E00846383803685B1CF2
:102C000000D1AAE00846343803685B1C00D1A4E078
:102C10000846303803685B1C00D19EE008462C381B
:102C200003685B1C00D198E00846283803685B1CE9
:102C300000D192E00846243803685B1C00D18CE088
:102C40000846203803685B1C00D186E008461C3823
:102C500003685B1C00D180E00846183803685B1CE1
:102C60007BD00846143803685B1C76D008461038C1
:102C700003685B1C71D008460C3803685B1C6CD081
:102C80000846083803685B1C67D0081F03685B1C94
:102C900063D00868401C5FD0103A4031002AA5D1AB
:102CA000CA49802002460B463C3B1B685B1C5ED039
:102CB0000B46383B1B685B1C59D00B46343B1B68EA
:102CC0005B1C54D00B46303B1B685B1C4FD00B4643
:102CD0002C3B1B685B1C4AD00B46283B1B685B1CCB
:102CE00045D00B46243B1B685B1C40D00B46203B69
:102CF0001B685B1C3BD00B461C3B1B685B1C36D027
:102D00000B46183B1B685B1C31D00B46143B1B6801
:102D10005B1C2CD00B46103B1B685B1C27D00B4662
:102D20000C3B1B685B1C22D00B46083B1B685B1CE2
:102D30001DD00B1F1B685B1C19D00B685B1C16D0C9
:102D4000103A4031002AAED103209D4901229D4B0B
:102D50000AF0C8FE00200AE008464159491C05D087
:102D6000802004E03CE800083CEA00088008A071EC
:102D70009749802208463C3803685B1C00D1B0E0CC
:102D80000846383803685B1C00D1AAE0084634388E
:102D900003685B1C00D1A4E00846303803685B1C64
:102DA00000D19EE008462C3803685B1C00D198E0F7
:102DB0000846283803685B1C00D192E00846243896
:102DC00003685B1C00D18CE00846203803685B1C5C
:102DD00000D186E008461C3803685B1C00D180E007
:102DE0000846183803685B1C7BD008461438036813
:102DF0005B1C76D00846103803685B1C71D008460F
:102E00000C3803685B1C6CD00846083803685B1CF0
:102E100067D0081F03685B1C63D00868401C5FD044
:102E2000103A4031002AA5D16A49802002460B465B
:102E30003C3B1B685B1C5AD00B46383B1B685B1C39
:102E400055D00B46343B1B685B1C50D00B46303BC7
:102E50001B685B1C4BD00B462C3B1B685B1C46D095
:102E60000B46283B1B685B1C41D00B46243B1B6870
:102E70005B1C3CD00B46203B1B685B1C37D00B46D1
:102E80001C3B1B685B1C32D00B46183B1B685B1C51
:102E90002DD00B46143B1B685B1C28D00B46103B07
:102EA0001B685B1C23D00B460C3B1B685B1C1ED0B5
:102EB0000B46083B1B685B1C19D00B1F1B685B1C77
:102EC00015D00B685B1C12D0103A4031002AAED1ED
:102ED0000320CA490122CA4B0AF004FE002006E082
:102EE00008464159491C01D0802000E08008E0716B
:102EF000394801463C3180220B463C3B1B685B1C39
:102F000055D00B46383B1B685B1C50D00B46343BFE
:102F10001B685B1C4BD00B46303B1B685B1C46D0D0
:102F20000B462C3B1B685B1C41D00B46283B1B68A7
:102F30005B1C3CD00B46243B1B685B1C37D00B460C
:102F4000203B1B685B1C32D00B461C3B1B685B1C88
:102F50002DD00B46183B1B685B1C28D00B46143B3E
:102F60001B685B1C23D00B46103B1B685B1C1ED0F0
:102F70000B460C3B1B685B1C19D00B46083B1B68BF
:102F80005B1C14D00B1F1B685B1C10D00B685B1CF8
:102F90000DD0103A4031002AAED10320E74901227A
:102FA000974B0AF09FFD00202072002070BD002189
:102FB000C9430068401A411E88412072002070BD3C
:102FC000B0EB00087BE900083CE400083CE60008A0
:102FD0003CE000083CE2000800FC0008F0B58FB0BF
:102FE0000B920A908248405C0D900C9188008149B8
:102FF0000E5873420124804A0E942006C00B3546B9
:103000003618801880081F461146B458641C17D023
:10301000401C1B1F121DF8D10E9C641CE0B20D9ABF
:1030200090422E460A463B46E6D9032073490122C8
:10303000734B0AF057FD00200E9005460C9C24E0CF
:103040000E99C9B20D9A91420C9C0CD24902C91A30
:103050000A460968491C2E4616D060006949085A7C
:103060000B9B154612E06000664A105A01292E4655
:1030700008D13168491C00D100200B9B01210E9121
:10308000354603E05D4200E035460B9B61005D4A3A
:10309000515A5A1E8A4209D280B298420DD20093E8
:1030A0000190032055490126764B94E0009301914D
:1030B00003205249012654A38DE008909800B542A0
:1030C000099502D18019001F19E029180D9A33467D
:1030D0005602F218041F914209D90095072047496A
:1030E00001225DA30AF0FEFCA01B401907E0009539
:1030F00007204249012251A30AF0F4FC60190D9007
:1031000001680F0A1F2038400F230B400A06120FD8
:103110000792D21814188A03D20EA4180D02AE0E0C
:10312000A4190D0EAC4238D10A9C2170E570090C2F
:10313000A1706770FD21C90059180C9B00930B9B6F
:10314000019302910799039104A945C107252B4FCB
:1031500001264A4B2846394632460AF0C3FCE0783D
:10316000A178227863780E9CE4B20394089C0294C0
:103170000D9C0194099C00941B029A1809040006F6
:103180004018801804903E4B2846394632460AF0D3
:10319000A9FC002630460FB0F0BD0E98C0B2099AC7
:1031A00000920D9A01920E94089C0294039004914F
:1031B0000327124901262F4B384632460AF092FC6B
:1031C00000940C9801900E98029003950D9804902D
:1031D000294B3846094932460AF084FC00200A99F6
:1031E000C87088704870087030460FB0F0BDC04697
:1031F0008ADF000898DF000800FEFFFFB0EB000840
:103200007BE900087CDF0008696E646578206E75D4
:103210006D2028256429203E206872207265636F26
:103220007264206D6178206E756D202564202626DD
:1032300020696E646578203E20300000726561640C
:10324000203A68725F73746172745F616464723192
:10325000203D20252378000072656164203A687261
:103260005F73746172745F6164647232203D202503
:103270002378000095E90008C4E800082BEB00085B
:103280006DE8000804EB0008F0B585B0044680073F
:103290000AD0009403202949012629A332460AF0C6
:1032A00021FC304605B0F0BD0D462C4F381F1C21C7
:1032B00001603868002805D538460C382849016077
:1032C00028490160386800260028EAD40496FCF7F3
:1032D00011FF254908602046294609F05DFA064697
:1032E00021480068FCF70AFF002E10D020680094E7
:1032F00001900720114901261CA332460AF0F2FB77
:10330000F007396801433960304605B0F0BD012649
:10331000F0073968014339602068A84206D10220CD
:1033200008F076F9049E304605B0F0BD0094019592
:1033300002900720014912A3B0E7C046B0EB000895
:103340006164647220252358206973206E6F742095
:10335000616C69676E65640D0A000000142002400C
:10336000851A7AE591836E7C44170020616464724B
:10337000203D202523582C2072656164202564009F
:10338000466C6173685F577269746520446174614B
:10339000204D69736D617463682061742061646499
:1033A00072202523582C206578706563746564202D
:1033B000256420676F74202564000000F0B595B087
:1033C000062818D1B4490A68511C14D0149201255A
:1033D000002406260096019402950320AF49B0A36D
:1033E0002A460AF07FFB14A831462246FFF7F6FD75
:1033F000284615B0F0BDB849095C109111908000C5
:10340000B649085842420124B54B0E901394210648
:10341000C90B4518C918890814461E46AF597F1CA8
:1034200015D0491C241F361DF8D1139C641CE1B231
:10343000109881420E98E9D9032098490122A94B9E
:103440000AF050FB002113910D91129127E0139A7D
:10345000D2B25302C518AD1910988242119809D200
:103460001B1B1A68521C129517D041009E4A515AD4
:103470000D9314E041009C4B595A012A0AD10E9831
:103480000068401C00D10021012013900E980D907F
:10349000129004E01295604200E00E980D9014AA7C
:1034A00000200790D07013469048057804462E09F6
:1034B0000A277E43AD1908350F20054002460F90BC
:1034C000667834097C43A419240164191C7009939B
:1034D000874C25782E0905407E4370191F2528400A
:1034E0000C904601647820091440784300193F226B
:1034F00002400B9290028219160A9E707B488478D3
:1035000020090F9B1C40784304192C401019099D79
:103510006870149AAE7068701046184013061B0F3E
:103520001818D304DB0EC0189303DB0EC018120268
:10353000920E80180A90E870149F1398C2B289B254
:103540000D980090129E01960891139202A886C0D1
:103550000720099051490125664B2A460AF0C2FA14
:103560003806000F0F9A3A40FD21C9005118119AF0
:1035700000920191029003940C9804900B9805908E
:103580000A9806905C4B099844492A460AF0AAFA20
:10359000129630463946FFF777FE002819D00324EB
:1035A0003E4E56A3204631462A460AF09BFA0D9815
:1035B0000090129801900898029013980390049735
:1035C000534B204631462A460AF08CFA284615B05D
:1035D000F0BD119F139D68020E990818001F1299E3
:1035E000814249D1009106202C490124494B2246B1
:1035F0000AF078FA4848C65D1098854211D27619CB
:1036000046490868002805D508460C384449016039
:10361000444901600096072020490125424B2A4673
:103620000FE03E490868002805D508460C383C499B
:1036300001603C4901600096072018493A4B254635
:1036400022460AF04FFAFCF755FD384F3860022049
:10365000314609F025F804463868FCF74FFDE807C5
:103660002E4A116801431160002C119F04D000966E
:1036700006200A492E4BA6E778001B4A105A089AE2
:10368000824200D2521C14A83946FFF7A7FC079DBE
:10369000284615B0F0BDC04600FC0008B0EB00089D
:1036A000466C6173685F57726974655F2825642989
:1036B0005265636F726428256429206E756D203E03
:1036C0003D207265636F72646564204D6178206E81
:1036D000756D2825642900008ADF000898DF00083E
:1036E00000FEFFFF7BE900087CDF00080F010020DF
:1036F0000C010020EAE900083FEA000868725F77E1
:10370000726974655F646174615F6572726F720083
:10371000F0E9000880EA000891DF00081420024068
:10372000851A7AE591836E7CF7EA00084417002039
:10373000E9EA0008F0B585B006202349012523A356
:103740002A460AF0CFF9264E00241C223046214694
:1037500006F070FB0D200527394607F029F82148AF
:1037600021497160B060B476E12030831F487061F8
:10377000F07EFE210140F176304602F0E5FD0A20A0
:1037800003900297680201901948009019481AA105
:103790001C4A234607F0ECFE002809D003200A4902
:1037A00019A32A460AF09EF92C46204605B0F0BD22
:1037B0000720054901221DA30AF094F90D4807F0DE
:1037C000B9FF204605B0F0BD32ED00086275747493
:1037D0006F6E5F74687265616420737461727400E7
:1037E000E429002019570008395800084B009600BA
:1037F0005C0F0020CC0E0020627574746F6E5F3019
:10380000000000005D190008627574746F6E5F74CB
:1038100068726561642063726561746520666169C0
:103820006C65642E2E2E0D0A000000006275747403
:103830006F6E2074687265616420696E69742073AC
:103840007563636573730000F0B5DDB004460CA8C2
:103850004021FCF72AFD657827780024082D09957A
:1038600016D8C0467D442D796D00AF440414313A1A
:10387000434C55667E00072694490122BA4B3046D8
:103880000AF030F90CA8FEF7CDFD00200A90CDE03B
:1038900026460A97CAE0009707208C490A97012715
:1038A000B04B3A460AF01EF90CAE38460A9F39462C
:1038B0003246FEF75DFD002807D03078002804D19D
:1038C0000CA80021072206F0B5FA002F32D1A6E09D
:1038D000009707207D490122A14B0AF003F902203D
:1038E00022E000970720794901229C4B0AF0FAF860
:1038F000032019E0009707207449012292A30AF0DF
:10390000F1F8042010E0009707207049012288A3F5
:103910000AF0E8F8052007E0009707206B4901222C
:103920007EA30AF0DFF806200CAA3946FEF720FD38
:10393000002F74D007260A9778E00097072663497E
:103940000A9701276EA330463A460AF0CBF80CAA34
:1039500030463946FEF70CFD002867D00A9800284B
:1039600056D00CA8002107265DE00A971CAF002066
:10397000B87038800BAEB070308030463946FEF7F4
:10398000FDFB71780F220B0911400A2043435B189D
:1039900008930CA98B70B3781D0913404543EB18AD
:1039A0000793CB703B781D0913404543EB180693F2
:1039B0000B717B781D0913404543EB184B71BD78A3
:1039C0002F09154047437D198D71367832403609ED
:1039D0004643B018C2B2303848707D20000110183C
:1039E000020A0A70E9B2DAB2069BDBB2079DEDB2B9
:1039F000089EF6B2009001960295039304920591F9
:103A000006203249012232A30AF06CF807260DE0A5
:103A10000CA84078002802D00CA8077035E70CA845
:103A2000002107260A91324606F004FAB01D1CADAB
:103A300028706F1C012002023846214606F0FAF970
:103A40002E710998E8700A98A870AA206870681DFD
:103A50000CA9324606F084F92A78901E26D0032459
:103A600001462140D21E032A02D20022144610E051
:103A70000346A343002214461CADAD186E783419DA
:103A8000AE783419EE7834192D792C19121D934221
:103A9000F2D100290AD0BB5C1C19012906D0D21929
:103AA00053781C19022901D091780C191CA94A1CC1
:103AB000145408788018401E552202700978384640
:103AC00000F0ECF900205DB0F0BDC04658E80008F9
:103AD0006B47657443757272656E7454696D653AAF
:103AE00020253034642D253032642D253032642079
:103AF00020253032643A253032643A253032640071
:103B00006B53656E736F724661696C757265526551
:103B1000636F726428256429000000006B506F7782
:103B200065724F6E5265636F7264282564290000C8
:103B30006B506F7765724661696C7572655265632B
:103B40006F726428256429006B4661756C7452633A
:103B5000795265636F7264282564290029E800089A
:103B60003AE8000818E800085FE800088CB0002573
:103B70000B950A9509950895079506950595049561
:103B80004B2080010121890200F01AF9524E534F57
:103B900001950CE00320012239465B4B09F0A2FF9E
:103BA0000027019D4C4E384605F09CFC4B4F306879
:103BB000E94306F0B3FF07260125304639462A4679
:103BC000474B09F08FFF474F384604F0C7F9C4B29E
:103BD00000943046404E41492A4643A309F082FFF3
:103BE00004AD38463D4F2946224604F0FDF9102128
:103BF00041A02A46019D234609F0C4FC062CD6D3D9
:103C000023462E4604AC02930CE0344F029B039DE6
:103C100004A808184078D1B2884231D0641C761CC0
:103C20009E42B7D004A8805DAA28F7D1F01C04AA50
:103C3000155C4119881880785528EFD103202B4650
:103C4000034003952F1D8743002220460578AA18BC
:103C50004578AA188578AA18C578AA183F1F001DAC
:103C6000002FF3D1002BD0D00578AA18012BCCD08F
:103C70004578AA18022B194FC8D080788218C5E75A
:103C8000E81C05F057FF002820D0074604A830188C
:103C9000417839708078BD707870002D06D004A806
:103CA0003018011DF81C2A4606F05AF80720012298
:103CB0000A49164B09F016FFBB78FA1C102114A014
:103CC00009F060FC3846FFF7BFFD6AE703200122D8
:103CD0000249134B62E7C0461012002058E8000862
:103CE0004EE80008880300206275665F6C656E20F0
:103CF0003D2025640A0000006C7075617274315FAC
:103D000072785F7262000000E9E70008FFE70008D0
:103D1000486F73744672616D6544617461000000A0
:103D2000D8E7000870B582B005F078FE01A8002140
:103D30000170664E306880060AD5F069800607D5A6
:103D4000706A01A9087071482830012204F0BCF99A
:103D50003068000611D5F06900060ED56B4C3C3476
:103D6000204604F0FBF8002821D001AD01222046B6
:103D7000294604F039F92878B0623068400607D542
:103D8000F069400604D540203062316881433160DB
:103D90003068C00707D0F069000704D540203062C2
:103DA000706A01A9087005F053FE02B070BD30685A
:103DB00080218843306030684006E1D4E8E7C0469F
:103DC00070B588B00E460546284C20462830284954
:103DD0002831102204F0F9F83C342649802220468C
:103DE00004F0F3F81B200324214606F0E1FC1A201E
:103DF000214606F0DDFC00200790A1021E4A9368D0
:103E00008B430124E10259189160210513680B438B
:103E1000136000BF00BF00BF069603950190059098
:103E2000200304900C200290144D01A9284608F0AC
:103E300075FD002800D0FEE71148016840220A43C2
:103E4000BF218A43026020070E49086028682021AC
:103E50000143296028682043286006200A490BA3F3
:103E6000224609F03FFE08B070BDC0466003002046
:103E700070020020481700203410024000800040EB
:103E80001CE400E000E100E074F900084C505541EA
:103E90005254315F496E69740000000070B50C46E1
:103EA00005461A4E3C36304604F043F8A04201D293
:103EB000002070BD30462946224604F005F903492A
:103EC0000A68802313430B6070BDC0460080004029
:103ED000B0B582B00D48283004F040F804460C4DCF
:103EE00000280ED0E868A0420BD1009407200949B1
:103EF000012209A309F0F6FD0C48006806F0BEFD9A
:103F000001E0002C00D0EC6002B0B0BD60030020E6
:103F10007002002074F900086C7075617274315F72
:103F200072785F72623A202564000000101200204F
:103F30000120000202490A6802430A607047C04635
:103F40001810024080B505F069FD174801463C395C
:103F50000A68920404D50268920701D502228260A1
:103F6000124A1368DB0704D09368DB0701D00123F2
:103F700013610968C90404D50168C90701D001218A
:103F80008160014640390968490709D5016849033C
:103F900006D50121890481600549C81CFEF7EEF8A9
:103FA00005F056FD80BDC046542800402CB00040AE
:103FB0000C01002080B50B4A1178012908D1132883
:103FC0000AD880001018C16A101D05F0EBF980BDF9
:103FD000054805F04FFD80BD0021101D05F0E2F9F8
:103FE00080BDC0469000002010E70008B0B584B046
:103FF0000E480FA100242246234606F015FD052099
:1040000003901D2002900120800201900C48009036
:104010000C4D0DA10F4A2846234607F0A9FA044685
:10402000284607F087FB204604B0B0BD8001002081
:1040300073656E736F725F72785F73656D000000F9
:104040000C1B00207C1A002073656E736F725F7208
:104050007800000075400008B0B507240025204610
:10406000294606F0A5FB0121204606F0DBFB284689
:10407000B0BD0000C0B00620AF490122AFA305903B
:10408000169209F02FFD4B20C0010025294600F0B3
:10409000ABFA2AA806465436074650370146403147
:1040A0000B91014630310246203210300A9019A897
:1040B000001F139015950D960C970991089204E036
:1040C00001240520FFF776FF159417950026F1438C
:1040D000A04806F023FD299619A84021FCF7E5F831
:1040E0009D4F384603F03AFF85B2222D03D838465B
:1040F00003F014FFC6E0044619A938462A4603F027
:1041000073FF03200440281B001F374619A98A5D4E
:104110007A4089194B7853408A785A40CF78574073
:10412000361DB042F2D1002C10D019A8805D474056
:10413000012C0BD019A8801940787840022C01D1AD
:10414000074603E019A989198F7847407A4E1398DA
:10415000401929AA8149FCF7EDF82998B84242D1C3
:1041600035462AAC58212046FCF79FF8089E009659
:10417000099F01970B9802900C9803900D9804905A
:1041800019A87A4922460A9C2346FCF7D3F8072847
:1041900041D12AA809F0ADFD05460791204609F056
:1041A000A8FD06901891304609F0A3FD14901291D5
:1041B000384609F09EFD119010910B9809F099FD79
:1041C0000F900E91002710260C9839463246FCF7C6
:1041D000E9F904460D983946069F3246564EFCF7DB
:1041E000E1F9079B2AE003250124284631462246AF
:1041F0005B4B09F077FC19A8009006203146224657
:10420000584B09F06FFC29980097019028463146D9
:104210002246554B34E0032001222E462946544BBA
:1042200009F060FC00252B462F4618951495129531
:10423000119510950F950E952C4628465121454A0B
:104240005054502014540F9890640E98D064956286
:10425000D362176318985063149890631298D063D0
:104260001198106410985064104628300021418540
:104270008185C18519A80090062001223146394B5D
:1042800009F030FC3348866AC46A0025304621466E
:104290002A46384BFCF70CFA0746401E8741304649
:1042A000214618952A46344BFCF7ECF90028169D58
:1042B00000D13D4630462146189A2E4BFCF7CCF9EA
:1042C000002800D13D46012D179D04D1002D02D1BB
:1042D000012503201CE030462146189F3A46264B14
:1042E000FCF7D0F9694269410028169800D10846C8
:1042F0001490304621463A461F4BFCF7C3F900287C
:104300003B4600D105461498002803D104201D46E1
:10431000FFF750FE50200F4B185C002804D0159872
:10432000002800D0D1E6CBE600241598002815948B
:10433000059800D0C6E6C8E6B7ED000853656E7371
:104340006F725F5468726561645F456E7472790D57
:104350000A00000080010020D002002092ED000839
:1043600067ED00088BF0000846ED000897ED0008A7
:1043700075ED0008000004400000E03F80B505F046
:104380004DFB07F007FB05F063FB80BDB0B51D4D8D
:104390002C1F20688006400F411E032921D81A488F
:1043A0007944097949008F44220116192968C907FF
:1043B00000D11E4829680906C90E00D120214843B2
:1043C00029684905490F00D10821FCF787F92968B8
:1043D0004903890F0AE07D20000208E00120C003A4
:1043E00005E00C3D2868C004810F1048C8402168D2
:1043F00089091C220A4005498958FCF76FF90A49C6
:104400000860B0BD0C10024000127A005CDF0008AA
:104410000348044901600448044901607047C046EC
:1044200008ED00E0000000080C0000200024F4006B
:10443000BFF34F8F044805490160BFF34F8F00BFA2
:1044400000BF00BF00BFFAE70CED00E00400FA0572
:10445000B0B582B00C460021019103280DD16068EF
:10446000FCF7D8F80546A068FCF7D4F80246E9B294
:1044700001A8FEF7B3FD02B0B0BD0320034901223D
:1044800003A309F02FFB02B0B0BDC046B0EB00089B
:10449000544553545F466C6173685F526561645F55
:1044A0005265636F72642020202020202D2D7573AB
:1044B00065205F636D645F205B7265636F72642863
:1044C000307E36295D205B6E756D5D00F0B583B082
:1044D000032820D10C464868FCF79CF80546A068E4
:1044E000FCF798F8012814DB0446EDB20027264EAD
:1044F0007F1C00950197062001220B491BA309F0A0
:10450000F1FA2846FEF75AFF304607F081F8BC4220
:10451000EED103B0F0BD03200349012203A309F04B
:10452000E1FA03B0F0BDC046B0EB00085445535467
:104530005F466C6173685F57726974655F5265634B
:104540006F72642020202020202D2D757365205F40
:10455000636D645F205B7265636F726428307E36C2
:10456000295D205B6E756D5D00000000466C617317
:10457000685F57726974655F282564295265636FA7
:1045800072643A256400000060EA000070B50C46D1
:104590000546A94E4C36304603F0CBFCA04201D272
:1045A000002070BD30462946224603F08DFD0446AA
:1045B00000F0E6F9204670BD80B582B005F02EFA15
:1045C0002E48016889060AD5C169890607D5406A5F
:1045D00001A9087098486030012203F075FD05F0CC
:1045E00037FA02B080BDC046F0B587B00F46064628
:1045F0001F4860301F49802203F0E7FC1720032585
:10460000294606F0D5F8012460041B490A680243D4
:104610000A6000BF00BF00BF00200690059704900D
:1046200003900296042100910190144E6946304691
:1046300008F0CAFB002800D0FEE730682043306055
:10464000FF2000040E490A688243A805101808607C
:10465000A0060C4908603068202101433160062023
:1046600009490AA3224609F03DFA07B0F0BDC04649
:10467000700200201C28002034100240004400403A
:1046800018E400E000E100E074F9000855415254DC
:104690003220496E69740000B0B582B001A80021D3
:1046A000017005F0BBF9224D286880060AD5E8693B
:1046B000800607D5686A01A908705E481430012297
:1046C00003F002FD286800060FD5E86900060CD546
:1046D000584803F043FC002821D0564801AC012281
:1046E000214603F081FC2078A8622868400607D59F
:1046F000E869400604D54020286229688143296082
:104700002868C00707D0E869000704D54020286260
:10471000686A01A9087005F09BF902B0B0BD28686D
:1047200080218843286028684006E1D4E8E7C04635
:104730000048004010B505F071F909480168C90644
:104740000BD5C169C90608D510210162E94C206961
:1047500006F094F9206806F091F905F079F910BD9A
:104760000038014007201449012214A309F0BAF9C6
:10477000E04F05E0AA1A3846383003F0A5FC7D6208
:10478000144E38690021C94306F0C8F93468802006
:10479000051B7A6A9542F4D00F4989189542E9D8E9
:1047A000821A3E463836304603F08EFC802CE6D026
:1047B000304609492A46E0E774F9000855617274E9
:1047C000315F52785F5468726561645F456E7472E0
:1047D000790000000C000240BC070020B0B5C54DB8
:1047E0002846603003F0BAFB0446002806D068680B
:1047F000A04203D1034806F041F901E0002C00D0AB
:104800006C60B0BD8001002070B50A4D28461430A0
:1048100003F0A4FB0446B74E002807D0B068A042BE
:1048200004D15035284606F029F901E0002C00D0CB
:10483000B46070BD6003002070020020F0B581B04C
:104840003B4E306800F006FE306800F023FF394F21
:10485000386800F0FFFD386800F01CFF364C206817
:1048600000F0F8FD206800F015FF3068334D062495
:104870002946224600F0BCFE306800F0BDFE7D20D7
:104880008600304606F0C4FE38682946224600F00D
:10489000AFFE386800F0B0FE304606F0B9FE264E96
:1048A0003068294622462546009400F0A1FE306873
:1048B00000F0A2FE224806F0ABFE224C20682249FE
:1048C000032200F095FE206800F096FE1F4806F0D7
:1048D0009FFE1F4901261FA32846324609F002F910
:1048E000102500272846394605F09CFF6424204601
:1048F00006F08EFE2846314605F094FF204606F06D
:1049000087FE1AA300981249324609F0EBF81124E9
:104910002046314605F086FF0C4806F079FE204619
:10492000394605F07FFF142006F072FE01B0F0BD9D
:1049300014010020180100201C01002090E700084D
:10494000881300002001002086E70008B80B000053
:10495000A8E70008E887AAE6A380E794B5E7A38163
:10496000E99880E58AA8E4BD9C0A0000E887AAE6E9
:10497000A380E9A38EE69CBAE58AA8E4BD9C0A0060
:10498000F0B587B004F0C0FBD84E7069002803D0A2
:1049900004F08EFD07B0F0BD34464C34204603F0E1
:1049A000FEFA70610028F3D0194D28680127B8433A
:1049B000286018490868802202929043086028689D
:1049C0000221019188432860284618380168202276
:1049D0000A430260204603F0D5FA716906910D4C36
:1049E0002146203105910490039703A807F044FE67
:1049F00028680199084328602868384328602146C0
:104A00002068029A1043206004F052FD07B0F0BD08
:104A10001C00024008380140B0B584B031A000212C
:104A20000A4605F0CFFF334C2061002805D107204E
:104A30003149012231A309F055F838A000210A4676
:104A400005F0C0FF2060002805D107202A49012277
:104A500036A309F047F8022500953DA04049002201
:104A60000A2307F06DF8A061002801D007F022F9B1
:104A700000953CA03F4900220A2307F061F8E0615D
:104A8000002801D007F016F900953BA03D4900220F
:104A90000A2307F055F82062002801D007F00AF930
:104AA00005200390142002903748009001208002D6
:104AB000019036483649374A002306F059FD002850
:104AC00002D0002004B0B0BD304806F033FE0090A4
:104AD000062009490122304B09F004F8002004B0F7
:104AE000B0BDC04675617274315F72785F73656D79
:104AF000000000007002002074F900086372656114
:104B000074652075617274315F72785F73656D20B2
:104B1000637265617465206661696C0075617274A9
:104B2000315F72785F6F6B5F73656D006372656193
:104B300074652075617274315F72785F6F6B5F733B
:104B4000656D20637265617465206661696C000043
:104B500075617274325F72785F74696D6500000010
:104B6000DD47000875617274335F72785F74696D38
:104B700065000000094800086C70315F72785F744E
:104B8000696D6500D13E00081C2000208C1F0020AC
:104B900064F90008654700083CF90008F0B591B0D9
:104BA00004910590514E304638305149802203928D
:104BB00003F00BFA4C360124A20202924D49304612
:104BC00003F003FA4C4908682043086000BF00BFA7
:104BD00000BF06270C9700250A95E00210900F955C
:104BE000102000900E900D950B950AAE304607F000
:104BF00025FD0C970A9410950F950E9520200D9089
:104C00000B95304607F01AFD3C4E306802210143F7
:104C1000316030680421014331603068082101436C
:104C20003160374A106837490840A10301914018A4
:104C300010606002344B1860FF200004116881434B
:104C4000A0050818106002981860039809902F4872
:104C500008902F4824300790069506A807F00CFD11
:104C60003068204330607069A04370610B200326D8
:104C7000314605F09DFD0C2738463146019E05F072
:104C800097FD1D4988683043886000BF00BF00BFA2
:104C9000109504980F900E950D9505980C900A9715
:104CA0000B951B4D0AA9284608F08EF8002800D065
:104CB000FEE7A86840210143A960286820432860D6
:104CC0000F4908690F4A10403043086160060E49D9
:104CD0000860286800990843286006200D490EA343
:104CE000224608F0FFFE11B0F0BDC0467002002061
:104CF0000C1F00201C24002030100240080002403D
:104D000008E400E0FF00FFFF00E100E0BC07002036
:104D10000038014074F9000855534152543120497C
:104D20006E697400B0B5EFF31080EFF3108172B6C6
:104D300001214906154A116080F310883F48046834
:104D400013492046FBF7CAFC124D68607D20C10064
:104D50002046FBF7C3FC2860EFF31084EFF31080CC
:104D600072B601F02FFC0C4DE961A86101F02AFC3C
:104D7000E969A969401A286084F3108800206862F4
:104D80002862A860286100F009F8B0BD04ED00E0D9
:104D900040420F0004000020300300207047000054
:104DA000002807D0C1B2002906D001200F4A515C6B
:104DB0004018704700207047FF210A02024005D0CA
:104DC000110A0920094A515C401870470904014042
:104DD00005D0090C1120054A515C40187047010E9E
:104DE0001920024A515C40187047C046A4DD0008F3
:104DF00070B582B00124204601F022FC0625094E40
:104E000009A328463146224608F06CFE0B4800688C
:104E100000900BA328463146224608F063FE00208E
:104E200002B070BD7DF900085F706572665F636FE8
:104E3000756E7465725F696E697400000C00002005
:104E4000706572665F636F756E74657220696E69F6
:104E5000742C2053797374656D436F7265436C6F66
:104E6000636B3A256400000070B5154604460028BF
:104E70000AD00026002D0FD02A792968A06C03687B
:104E800020469847304670BD044805A1372203F0FC
:104E900017FF0026002DEFD1F04370BD4EFA000839
:104EA0005F70696E5F636F6E74726F6C00000000FC
:104EB00080B586B000200590049003900290019088
:104EC0000B069B0F09D1C9B20C2048433B490B5834
:104ED0005B1C01D0081800E00020062A1BD8C04641
:104EE0007A44127952009744030716090D101200F4
:104EF00000210391012106E0002109E00121039135
:104F0000022100E00321029103E0012100E00221DF
:104F1000039181680191406801A907F0AFFC06B0D8
:104F200080BDC0463F220A400C20504323490A5806
:104F3000521C01D0081800E000204168806809690F
:104F40000140091A484248417047C04670B51E46A4
:104F500014460546002804D1084809A1162203F08A
:104F6000AFFE0020002C08D0082E06D12168A86CC6
:104F70008268284690472071082070BD4EFA0008CC
:104F80005F70696E5F72656164000000002A01D085
:104F9000182000E028203F2211400C224A430749F4
:104FA0008B585B1C04D089184A6889681150704777
:104FB00000214A68896811507047C04610E4000813
:104FC00070B51E4615460446002804D1084809A1BC
:104FD000262203F075FE0020002D08D0082E06D1F1
:104FE0002A792968A06C436820469847082070BD3C
:104FF0004EFA00085F70696E5F7772697465000031
:10500000F0B583B00446089D064628362EC61C30EF
:10501000E0612062232118462A4604F00BFF234654
:1050200028330FCBD218121F144B04F095FC60628A
:1050300025463C350A9E099F202F04D310A019A1B4
:10504000A72203F03DFE6F70AF70E6642665002076
:105050002064A063E86428652870009001902046D1
:105060005430144A2146234606F0DCFD12480168FC
:10507000002901D02046884703B0F0BD2DB40008B8
:105080007072696F72697479203C2052545F544881
:10509000524541445F5052494F524954595F4D4126
:1050A000580000005F72745F7468726561645F69C4
:1050B0006E69740079B800086818002000F004FADE
:1050C000052006F0A5FAF9E7B0B584B0114C2078B8
:1050D000002807D1204608300F49002204F01EFFA7
:1050E00001202070052003901C2002900B480090A6
:1050F0000320000201900A4C0AA10C4A0025204618
:105100002B4606F035FA204606F014FB284604B07C
:10511000B0BDC046E402002046FA0008BC040020EE
:105120002C04002061676C6564000000BD5000081D
:10513000F0B583B007466D48007800281FD01546AB
:105140000E4602932C2004F0F5FC00281DD00446E6
:10515000384600270190211DC1C127616761278062
:10516000002D16D02046294600F0C2F8002810D0A5
:10517000204604F0B7F93C46204603B0F0BD0320BA
:10518000264901220E4B08F0ADFC0024204603B056
:10519000F0BD0298A061E06106F0F8FB0021094A29
:1051A00020626262A162019D284605F001FB714206
:1051B0007141284605F036FB204603B0F0BDC046DD
:1051C00082F90008C951000810B582B004460028D1
:1051D00004D1074807A17A2203F072FD60680090AD
:1051E00007200E4901220EA308F07CFC02B010BD7E
:1051F000ACEB00086167696C655F6C65645F646552
:105200006661756C745F636F6D70656C6574655F06
:1052100063616C6C6261636B00000000CCF9000894
:105220006C65642070696E3A256420636F6D7065EB
:105230006C657465642E0000F0B583B00192029134
:105240000446002805D12320C2009A48264903F0CD
:1052500037FD2078002806D02320C000421C70486B
:10526000214903F02DFDE04D08350026F74328467F
:10527000394604F033FF0298002827D0E068002860
:1052800002D004F02FF9E66026612046029900F072
:105290002FF800281AD02846394604F01FFF6078FE
:1052A00000280FD0FA48001D224628320146006827
:1052B000002801D09042F9D1002801D00068086090
:1052C0006670A662284604F05FFE07E066610198FA
:1052D000A061E06106F05AFB20623746284604F0E0
:1052E00053FE384603B0F0BDD6F90008E4020020B2
:1052F000F0B581B00D460446002848D0207800283B
:1053000004D0474845498F2203F0DAFCE0680028C2
:1053100004D044A04149902203F0D2FC2069002827
:1053200004D047A03D49912203F0CAFC002003E0CD
:105330002169491C2161001D295C2C2910D00029FC
:105340002ED029184A782C2A11D0002A2AD08A78FF
:105350002C2A12D0002A27D0CA782C2A13D1E7E7AA
:105360002169491C216129184A782C2AEDD122692A
:10537000521C22618A782C2AECD12269521C2261AB
:10538000CA782C2AD4D0002AD5D1C91C0DE02248D5
:1053900022498E2203F094FC20780028B1D1B5E791
:1053A000291802E0491C00E0891C2069491E09787F
:1053B0002C2901D0401C20610421CF43002821D09A
:1053C000800004F0B7FB00281DD021698A00002767
:1053D0000090394604F02EFD2069002816D0009E6A
:1053E00003E07F1C2069874210D22846FBF712F9A0
:1053F00001C62C212846FAF770FF05460028F0D098
:105400006D1CEEE73F1D384601B0F0BD0098E0602E
:105410000027384601B0F0BDACEB00082EFA0008BA
:10542000A8F900086C65642D3E6C696768745F615B
:105430007272203D3D2052545F4E554C4C0000008E
:105440006C65642D3E6172725F6E756D203D3D200E
:105450003000000010B50446002805D1FF22F232CA
:10546000054806A103F02CFCA06841424141606858
:1054700005F0D8F910BDC046ACEB00086167696C57
:10548000655F6C65645F6F666600000010B504467A
:10549000002804D06068A16805F0C4F910BDF320AD
:1054A0004200044804A103F00BFC6068A16805F009
:1054B000B9F910BDACEB00086167696C655F6C659C
:1054C000645F6F6E00000000F0B585B08C4F3D4604
:1054D000083500200190C1432846029104F0FEFDEA
:1054E0007E68002E7AD0009518E030462438006897
:1054F00005F098F906F04AFA0546049800683968FC
:105500008900405806F03EFA401920603868401C77
:105510003860009D7A4F3668002E5FD031460C39D6
:105520000868002824D003913446083C06F02EFA7F
:105530002168401A2D498842EDD230461C3804902B
:105540003546183D3746143F38682968884233D2BB
:105550008100049A12685158002936D1401C3860E5
:1055600006F014FA2168401A20498842ECD3D0E7AB
:105570002846029904F0B2FD304627380178002908
:105580000DD0391D0A460968002901D0B142F9D170
:10559000002901D009681160019901703160284625
:1055A00004F0F2FC3C1D301F0168002902D0283EA7
:1055B000304688472646AEE7019838600399086868
:1055C0000128A6DB401E0860A3E7314620390968A0
:1055D0004A424A41C00788D0114686E7284604F06F
:1055E000D3FC05B0F0BDC046E4020020FFFFFF7F02
:1055F00080B5FFF721FE80BDF0B581B004460028DC
:1056000005D1FF229A321D481DA103F059FB3C4DE4
:1056100008350027FE432846314604F05FFD6078D8
:10562000002825D13946364FE068002820D020696F
:1056300000281DD00E466161A069E06106F0A6F960
:105640002062391D0A68002A08460BD0116800291B
:10565000104607D00A68002A084603D011680029BE
:105660001046EFD121462831016001206070A6620A
:10567000284604F089FC304601B0F0BDACEB0008D0
:105680006167696C655F6C65645F737461727400F7
:10569000E4020020F0B581B00446002805D1FF22C5
:1056A000B632124812A103F00BFB154F3D460835E8
:1056B0000026F143284604F011FD607800280ED042
:1056C000381D2246283201460068002801D0904249
:1056D000F9D1002801D0006808606670A6622846EB
:1056E00004F052FC002001B0F0BDC046ACEB000855
:1056F0006167696C655F6C65645F73746F700000EF
:10570000E402002080B501F00BFC002080BD80B5D4
:1057100002F0C4F8002080BD80B586B0C17E827ED4
:10572000C08904900092C806000F029091001EA24A
:105730005158019180001EA1085803900720284964
:10574000012228A308F0CEF9324800F0F9FD012823
:105750000BD0304800F0F4FD022811D02D4800F0A5
:10576000EFFD042817D006B080BD06201C49012299
:1057700029A308F0B7F9274800F0E2FD0228EDD18F
:105780000620174901222A4B08F0ACF9214800F005
:10579000D7FD0428E7D1062011490122254B08F046
:1057A000A1F906B080BDC046F3EB00080FED00087C
:1057B0007BEC00084AEC00082EEC00085FEC0008C7
:1057C000F4EC0008C2EC0008DAEC0008ABEC0008CE
:1057D00001EC00088FEC00081FED00081AEC00082F
:1057E00032ED000869643A205B2564202D20257382
:1057F0005D20206576656E743A205B2564202D203F
:10580000253330735D20207265706561743A202500
:10581000640A0000E4290020464C45585F42544E7B
:105820005F50524553535F434C49434B0A000000BD
:10583000BAEB0008D7EB000880B5807E002807D0BF
:1058400006A007A13E2203F03BFA0020C0B280BDB3
:105850000D2004F0CBFFC0B280BDC0463000000078
:10586000636F6D6D6F6E5F62746E5F726561640011
:10587000F0B589B01E4608920D4607460E9C04F00E
:10588000DDF8002809D000960194002039462A4608
:10589000089B07F0DFFB09B0F0BD0796069542486C
:1058A00001680029F7D0456B002D77D02246A6204D
:1058B000F840C007059415D1B8003C490818049079
:1058C000101F029033E028461038046807980090B3
:1058D000019230463946069A089BA047059A2D68E2
:1058E000002DD8D0284618380068B842F7D32E4685
:1058F0002C3E281F0468002CE5D0079800900192E8
:1059000030463946069A089BA047059A0028DAD106
:10591000E5E7284610380468079800900192304661
:105920003946069AA047059A2D68002DB3D028461F
:1059300018380068B842F7D32E462C3E281F04685A
:10594000002C0AD007980090019230463946069AFA
:10595000089BA047059A0028E6D028461C38006816
:10596000089B1843D5D104980068144605F02DFA19
:10597000024600282046079C214608D00C48039286
:1059800005F023FA039941180298401A61182A4633
:10599000103A1468009101900023C0E7079804F0C2
:1059A00095F809B0F0BDC0469C280020C0DE000874
:1059B000A2FA000810B5094C6069002803D005F070
:1059C0005DF8002010BD064806A1C82203F078F952
:1059D000606905F053F8002010BDC046D8010020D2
:1059E0005FF0000866696E73685F72785F696E6465
:1059F00000000000F0B581B00546214E7069002816
:105A000014D0284603F0FEF9002819D0044685205A
:105A1000850070694059844206D0FF2144312046F8
:105A200003F0F6F9002811D001B0F0BD154816A119
:105A3000DB2203F045F9284603F0E4F90028E5D11C
:105A400017A0294604F016F801B0F0BD776978591F
:105A5000002807D003F09CF970694059002103F039
:105A6000E9FA7769DF20400038185421FAF71DFC65
:105A70007C510A49204603F0DDFA01B0F0BDC04672
:105A8000D80100205FF0000866696E73685F736577
:105A9000745F64657669636500000000B5590008AD
:105AA00066696E73683A2063616E206E6F7420665B
:105AB000696E64206465766963653A2025730A001F
:105AC00070B582B01E4E1F481F4931607060432080
:105AD000C1000124204603F037F97061002827D067
:105AE0000A20152100910190A30218A01949002451
:105AF000224605F07BFB0546706917A12246234626
:105B000004F092FF7069002805D115481549A722B5
:105B100003F0D6F870692921425C022313434354F1
:105B2000002D02D0284605F005FE204602B070BDCB
:105B30000DA003F09FFF0020C443204602B070BDBB
:105B4000D8010020DCFC00088CFB00087473686539
:105B50006C6C0000815B00087368727800000000C4
:105B60005FF0000873F000086E6F206D656D6F7256
:105B70007920666F72207368656C6C0A0000000003
:105B800088B0AA4C60692922815C012305931943DE
:105B90000392815485218E008059002805D103F09D
:105BA000F1F8002801D0FFF725FF60690399405CF8
:105BB000800703D49E48002101701DE0216900295F
:105BC00004D09B488022FAF77BFB15E002F054FDDD
:105BD000002803D096489749052202E09448964948
:105BE0000722FAF73BFB924C2046FAF780FB3E2156
:105BF00021542018002141708D4803F03BFF002004
:105C00000690C543009627E106983870384603F0A1
:105C100031FFDF204000616908185421FAF745FB85
:105C20001AE10599017007A806990170002F1BD091
:105C3000B859002822D007AA0123294603F098F971
:105C400001287A4F0CD07869294604F067FF7869FB
:105C5000805907AA0123294603F08AF90128F2D1C5
:105C600007A80478754A0EE0B322754875A103F0C1
:105C700027F86E484769B8590028DCD103F032FD97
:105C80006E4A0446694F7F69384628301B2CC8D0BD
:105C900070497B180178022900D09BE00021017037
:105CA000442C00D98FE00491A00001A10858874638
:105CB000C55D0008115F0008115F0008115F000852
:105CC000115F0008115F0008115F0008115F0008F4
:105CD0001F5F0008B15E00085F5E0008115F0008EA
:105CE000115F00085F5E0008115F0008115F000887
:105CF000115F0008115F0008115F0008115F0008C4
:105D0000115F0008115F0008115F0008115F0008B3
:105D1000115F0008115F0008115F0008115F0008A3
:105D2000115F0008115F0008115F0008115F000893
:105D3000115F0008115F0008115F0008115F000883
:105D4000115F0008115F0008115F0008115F000873
:105D5000115F0008115F0008115F0008115F000863
:105D6000115F0008115F0008115F0008115F000853
:105D7000115F0008115F0008115F0008115F000843
:105D8000115F0008115F0008115F0008115F000833
:105D9000115F0008115F0008115F0008115F000823
:105DA000115F0008115F0008115F0008115F000813
:105DB000115F0008955F0008DF5F0008F15F0008D1
:105DC000196000082FE7FF2C00D12CE77F2C00D1B1
:105DD000A5E09DE0012906D15B2C02D102210170D2
:105DE0003AE0069901700D2C00D98DE0A00001A1C8
:105DF00008588746595E0008115F0008115F0008C7
:105E0000115F0008115F0008115F0008115F0008B2
:105E1000115F00081F5F0008B15E00085F5E0008A8
:105E2000115F0008115F00085F5E0008D8010020C4
:105E30008C11002053F0000858F000084BF00008C7
:105E40005FF0000866696E73685F67657463686118
:105E5000720000000E020000FC484769E3E6BC8DBA
:105E60001888002800D107E1052C00D2E3E0029059
:105E7000B72040003818DF214900791850220490DB
:105E80000191FAF73BFA002800D1F5E038462E30B0
:105E900039467E310524A201FAF7E0F95021049831
:105EA000FAF703FA04980199029AFAF7D7F9E2E0AF
:105EB00058880028EF490DD01646069C30460F46FC
:105EC00003F0D8FD3946212000017F69385A641C4F
:105ED0008442F3D3E84803F0CDFDDF2044003F19AE
:105EE00002F0CAFB012802D1384602F08FF9E149DD
:105EF0004869039A805C8007009E049700D543E1BF
:105F00000020DE4F3870C9E17F2C08D0FF2CA3D0D1
:105F10001888502800D2D4E00020188007E1598862
:105F2000002999D0481E58801A88521E1A8080B2C3
:105F300092B2824200D81AE1121ADF235C003B19A8
:105F40001818591803F00CFFEF4F7869F249415ABD
:105F5000401800210155212000017969085A0818CC
:105F60000119F4A003F086FDED4A7869EA4BC15AA5
:105F7000C0184088884200D96EE7441E104603F0DE
:105F800079FDE74AE0484069E349405A641C84428D
:105F9000F4D361E7788D002800D133E1401E788585
:105FA000DF2149007C1880B25022504339182E312D
:105FB00020461F46FAF752F92046FAF798F97880FA
:105FC0003880D84803F056FDCF494869039A805C71
:105FD000800700D519E1CD4F049838708DE1798D97
:105FE000BA8D501E884200DCDFE00293481CE0E0DE
:105FF00058881988884200D32EE73818DF214900D5
:10600000415CC64803F036FD21200001BE494969C4
:106010000A5A521C0A521FE75888002800D11BE771
:10602000104603F027FD21200001B74949690A5AAB
:10603000521E0A5210E70293002C0BD0DF204000C2
:106040003918502210466043C0192238FAF756F921
:10605000002811D050214C433C192E342046FAF729
:1060600024F9DF2040003918029802882046FAF708
:10607000F5F8B88D441CBC857C8502F0FDFA01283A
:10608000A14CA24F0FD160690399415CC90703D0AD
:10609000A64803F0EFFC60699F49415ADF22520095
:1060A000801802F05FF960690399405C800700D4B2
:1060B000AAE52169002970D080223846FAF700F954
:1060C000A4E55988814232D2421A7918FF20C030A3
:1060D0000818DF235F00C91903F042FE21200101E7
:1060E000894B5869425A8018C4551C465B69039A0B
:1060F0009A5CD20707D0591809885818C1198FA07F
:1061000003F0B8FC6369844F8548D95BDA19548879
:106110008C427D4A1CD2174603F0ACFC3A467E4FB7
:106120007F485369D95B641C8C42F4D310E0381863
:10613000DF2149004454744F7B690399595CC907B6
:10614000754F05D07548214603F094FC6E484369AD
:10615000D95B491CD953D8194288521C428089B254
:10616000502900D278E600214180018074E670A0B9
:1061700003F080FC644840696749415A4018DF21B8
:1061800049000022425467E60969002946D080226E
:106190005E4F3846FAF794F880E002F06DFA002876
:1061A00045D0052238465A4944E0002A00D153E63A
:1061B00002937885DF2149007C1880B25022504339
:1061C00039182E312046FAF749F801942046FAF79B
:1061D0008EF8029C60802080524803F04BFC4A49B4
:1061E0004869039A805C800703D4484F049838704C
:1061F00070E0096900292BD08022444F3846FAF715
:106200005FF867E00498788526E60969002928D0B8
:1062100080223E4F3846FAF753F86EE002F02CFA2F
:1062200000282DD00522394F384639492CE0072265
:1062300038463849FAF712F83846FAF758F83E2146
:106240003954381806994170E0E4C046D80100205E
:1062500002F012FA00282D4F2FD0052238462C4983
:106260002EE002F009FA0028284F39D005223846DE
:10627000274938E0D801002084E700088C1100206D
:106280000722224F38462349F9F7E8FF3846FAF744
:106290002EF83E21395438180021417022483946E1
:1062A000049A03F0E7FB184847693819FAF71FF812
:1062B0001949785279184880CEE5072238461549A1
:1062C000F9F7CCFF3846FAF712F83E21395438185E
:1062D00004994170019A1448394603F0CBFBBBE5A1
:1062E000072238460B49F9F7B9FF3846F9F7FFFF9F
:1062F0003E2139543818049941700B4839462246DA
:1063000003F0B8FBA8E5C046D80100208C1100209E
:1063100053F0000858F000080E02000070F000086A
:106320004BF000084DF0000889F0000884E70008F1
:1063300008200800082573202008000025730000AD
:10634000C07EC006000F7047B0B501460024E04390
:10635000002919D0994A1378202B15D815460C35E9
:106360002D68002D11D08D420ED02D68002D0CD03F
:106370008D4209D02D68002D07D08D4204D02D68A4
:10638000002D02D08D42EBD1B0BDD06808600F2047
:106390000882CC60D160581C1070CC7E012525404D
:1063A0002C461634CC769D40516829435160C0B2CA
:1063B000B0BDC046F0B581B0804DEC68002C00D176
:1063C000F1E02F7800266168002908D02046884730
:1063D0007F1EF9B2884006432468002CF3D1686818
:1063E0007040C043A860EC68002C00D1E2E02F7838
:1063F000002603E02468002C00D1D8E0E07E2028AD
:1064000006D3A189491CA18189B26D4A91423AD033
:106410007F1E410902293CD0012916D000296FD1E5
:10642000F9B2AA68CA40D1073ED00021E160E1215B
:106430000840E076A168002902D020468847E07E27
:106440001F2101402031E1765AE0F9B2AA68CA4022
:10645000D1072DD0A189E289002A57D0238A9942F9
:106460004ED9032A00D30322E12108405100014301
:10647000E176A268002A02D020469047E17E002003
:10648000E0601F200DE0218BA1817F1E41090229C0
:10649000C2D1F9B2AA68CA40D1071BD00021A1819C
:1064A0001F21084020302AE0E1210840163026E074
:1064B000A189228B91423ED2E28A91424FD2A28A96
:1064C000914268D21F2108404030E076E089401CAC
:1064D000E08115E0218AA2898A4211D9E189032944
:1064E00000D30321E122104049000143E176A26874
:1064F000002A02D020469047E17E1F200840E07627
:10650000E07E1F2800D875E7761C73E7228B914246
:1065100019D2E28A914230D21E220240082AEFD0DC
:10652000A28A9142ECD3E12108400830E076A168CC
:1065300000292DD1E4E7E12108401230E076A1687E
:10654000002913D115E01E2101401029D8D0E121E6
:1065500008401030E076A168002919D1D0E7E12188
:1065600008400E30E076A168002902D02046884716
:10657000E07E1F210140E176C2E71E2101400C2987
:10658000BED0E12108400C30E076A1680029B7D0E8
:1065900020468847B4E7E12108400A30E076A16848
:1065A0000029E3D1E5E76868C043A8600026F0B29F
:1065B00001B0F0BD0026F0B201B0F0BD180300201C
:1065C000FFFF0000B0B5EFF31082EFF3108072B65A
:1065D000124908684B68C01A3A4B1B685B0106D524
:1065E0000B681B1A102B02DB09684018401CC417EB
:1065F0003A4B596A1D6A28186141DC6A9D6A451B3D
:106600000D46A54104DAD96A986A82F31088B0BDB4
:106610009862D96282F31088B0BDC04614E000E0F1
:1066200080B502A003F026FA002080BD48656C6C9E
:106630006F2052542D546872656164210A00000075
:10664000B0B5EFF31081EFF3108272B6012252065B
:106650001C4B002803D01A6081F310880AE01A4806
:1066600000240460194D45608460072404601A60AA
:1066700081F310881648046816492046FAF72EF868
:10668000154D68607D20C1002046FAF727F8286084
:10669000EFF31084EFF3108072B6FFF793FF0F4D06
:1066A000E961A861FFF78EFFE969A969401A2860CE
:1066B00084F31088002068622862A8602861FEF7D1
:1066C0006DFBB0BD04ED00E010E000E0FFFFFF0057
:1066D0000C00002040420F00040000203003002086
:1066E000F0B581B010A003F0C5F91448056814484E
:1066F0000768AF4214D213A402E00C37AF420FD2A6
:106700003E68022230462146F9F705FE0028F4D003
:106710007A680DA0314603F0ADF908480568ECE74A
:10672000002001B0F0BDC0462D2D46756E63746922
:106730006F6E204C6973743A0A000000DC0100207F
:10674000D80100205F5F0000252D313673202D2DEC
:106750002025730A00000000F0B593B0092003F073
:1067600033FF0446D0A01021D9A203F083F901F031
:1067700085FFD9A003F07EF9271D00240120089091
:106780000D970CE01346143B917B00900191102172
:10679000DC480A4603F06EF9002C00D180E1002CA1
:1067A0003D4600D02546F9F7A5FC002C06D0211F58
:1067B00009787F220A40092A00D06FE12D68BD4286
:1067C00000D16BE12E68BE42129623D03168B942E7
:1067D00023D00A68BA422AD006901368BB422DD053
:1067E0001868B84234D00468BC423ED01194246882
:1067F000BC4248D000271097119F0397049005933F
:10680000079209911196029410980F900E900C9097
:106810000B9046E00024109403E0002411960899A0
:1068200010910F940E940C940B940A943BE0002466
:1068300009911196109408990F91F3E7002407929B
:106840000991119610940F9408980E900C9409E0F9
:106850000024059307920991119610940F940E94B9
:1068600008980C900B940A941CE000240490059363
:1068700007920991119610940F940E940C94089815
:106880000B900A940EE00024119F03970490059347
:1068900007920991119610940F940E940C940B94F6
:1068A00008980A900698F9F729FC2F1FF9F722FC9F
:1068B0003F78F9F723FC7F2006460740092F0D9FFC
:1068C00010D1297A1E298D4802D888008C49085891
:1068D000A97B143D0090019110218A480A462B465D
:1068E00003F0C8F81298B84200D155E71198051F77
:1068F000F9F700FC2D78F9F701FC3540092D12D18C
:106900001198017A1E297D4802D888007C490858D0
:1069100011990B46143B897B009001911021794815
:106920000A4603F0A7F81098002800D034E7099829
:10693000051FF9F7DFFB2D78F9F7E0FB3540092D4E
:1069400012D10998017A1E296C4802D888006C4936
:10695000085809990B46143B897B0090019110213E
:1069600068480A4603F086F80F98002800D013E71D
:106970000798051FF9F7BEFB2D78F9F7BFFB3540E7
:10698000092D12D10798017A1E295C4802D8880087
:106990005B49085807990B46143B897B009001918D
:1069A000102158480A4603F065F80E98002800D0D8
:1069B000F2E60598051FF9F79DFB2D78F9F79EFB88
:1069C0003540092D11D1059A117A1E294B4802D85C
:1069D00088004B4908581346143B917B0090019165
:1069E000102148480A4603F045F80C98002800D0CA
:1069F000D2E60498051FF9F77DFB2D78F9F77EFBA9
:106A00003540092D11D1049A117A1E293B4802D82C
:106A100088003B4908581346143B917B0090019134
:106A2000102138480A4603F025F80B98002800D0BA
:106A3000B2E60398051FF9F75DFB2D78F9F75EFBC9
:106A40003540092D11D1039A117A1E292B4802D8FD
:106A500088002B4908581346143B917B0090019104
:106A6000102128480A4603F005F80A98002800D0AB
:106A700092E60298051FF9F73DFB2D78F9F73EFBEA
:106A80003540092D00D087E6029A117A1E291B484D
:106A900000D977E688001A49085873E6F9F72EFB03
:106AA000002013B0F0BDC046252D2A2E73202020D3
:106AB0002020202020207479706520202020202094
:106AC00020202072656620636F756E740A000000D6
:106AD0006465766963650000202D2D2D2D2D2D2DEB
:106AE0002D2D2D2D2D2D2D2D2D2D2D2D2D202D2DE3
:106AF0002D2D2D2D2D2D2D2D0A000000E3EF00084A
:106B0000E0DE0008EEED0008F0B58FB00420039041
:106B100003F05AFD044658A0102160A202F0AAFF1B
:106B200001F0ACFD5FA002F0A5FF271D00266B4C15
:106B3000049704E0059E002E049F00D198E0002EEB
:106B40003D4600D03546F9F7D5FA002E06D0311F64
:106B500009787F220A40042A00D087E02968B942D8
:106B600000D183E0079109680026B9421FD008913F
:106B70000968B9421DD009910968B9421BD00A9130
:106B80000968B9420596039A06921DD00B910968CF
:106B9000B94212D00C910968B94210D00D91096820
:106BA000B9420ED005910E91082106910CE0012109
:106BB00008E0022106E0032104E0052102E00621AD
:106BC00000E0072106910596F9F798FA06E0454896
:106BD00002F050FF761C06988642ABD0B00007A9A1
:106BE0000F583D1FF9F786FA2D78F9F787FA7F20BD
:106BF00028400428EED13B46143B3869B968083771
:106C0000B94210D000213A461268BA4215D0126833
:106C1000BA420FD01268BA420ED0091D1268BA42A9
:106C2000F2D1491E09E0009010212FA00A4602F07F
:106C300021FFCFE7491C00E0891C00900191102141
:106C400020A00A4602F016FF3D68BD42BFD029468B
:106C50001C39204602F00EFF2868B842B7D0204801
:106C600002F008FF2D68BD42F1D1B0E7F9F746FA0E
:106C700000200FB0F0BDC046252D2A2E7320202005
:106C80002020207365742020202073757370656E3A
:106C900064207468726561640A0000006576656E40
:106CA0007400000020202D2D2D2D2D2D2D2D2D2D6E
:106CB000202D2D2D2D2D2D2D2D2D2D2D2D2D2D0A34
:106CC00000000000252D2A2E2A7320203078253040
:106CD000387820253033643A000000008BF000083B
:106CE0008BFA000884E70008252D2A2E2A7320201D
:106CF00030782530387820300A000000F0B58FB0A9
:106D00000520039003F060FC044664A010216CA2EF
:106D100002F0B0FE01F0B2FC6BA002F0ABFE271D4A
:106D20000026764C049704E0059E002E049F00D1B7
:106D3000B0E0002E3D4600D03546F9F7DBF9002ED5
:106D400006D0311F09787F220A40052A00D09FE033
:106D50002968B94200D19BE0079109680026B94231
:106D60001FD008910968B9421DD009910968B9423C
:106D70001BD00A910968B94219D00B910968B94230
:106D80000596039A069219D00C910968B94210D061
:106D90000D910968B9420ED005910E910821069116
:106DA0000CE0012108E0022106E0032104E00421B7
:106DB00002E0062100E0072106910596F9F79EF909
:106DC00006E0504802F056FE761C06988642ABD08C
:106DD000B00007A90F583D1FF9F78CF92D78F9F786
:106DE0008DF97F2028400528EED13B46143BB88A18
:106DF000F98ABA680837BA4210D000223D462D6899
:106E0000BD421FD02D68BD4219D02D68BD4218D09B
:106E1000121D2D68BD42F2D1521E13E000223D46E4
:106E20002D68BD422BD02D68BD4225D02D68BD42B6
:106E300024D0121D2D68BD42F2D1521E1FE0521CFB
:106E400000E0921C009101900292102125A00A46B8
:106E500002F010FE3D68BD42B3D029461C392046E1
:106E600002F008FE2868B842ABD0254802F002FEC6
:106E70002D68BD42F1D1A4E7521C00E0921C0091A4
:106E800001900292102120A00A4602F0F3FD9BE738
:106E9000F9F734F900200FB0F0BDC046252D2A2E99
:106EA0007320656E7472792073697A6520737573C7
:106EB00070656E64207468726561640A0000000089
:106EC0006D61696C626F7800202D2D2D2D20202D95
:106ED0002D2D2D202D2D2D2D2D2D2D2D2D2D2D2DEF
:106EE0002D2D0A00252D2A2E2A73202530346420CA
:106EF00020253034642025643A0000008BF000081F
:106F00008BFA000884E70008252D2A2E2A732025F5
:106F10003034642020253034642025640A000000C9
:106F200010B5074CA16807A002F0A4FDA1690AA052
:106F300002F0A0FDE1690DA002F09CFD10BDC0466D
:106F4000FC010020746F74616C206D656D6F727947
:106F50003A2025640A00000075736564206D656D34
:106F60006F7279203A2025640A0000006D6178690B
:106F70006D756D20616C6C6F6361746564206D6507
:106F80006D6F72793A2025640A000000F0B58FB069
:106F90000620039003F018FB044662A0102168A2AB
:106FA00002F068FD01F06AFB68A002F063FD271D96
:106FB0000026714C049704E0059E002E049F00D12A
:106FC000ADE0002E3D4600D03546F9F793F8002E8F
:106FD00006D0311F09787F220A40062A00D09CE0A3
:106FE0002968B94200D198E0079109680026B942A2
:106FF0001FD008910968B9421DD009910968B942AA
:107000001BD00A910968B94219D00B910968B9429D
:1070100017D00C910968B9420596039A069215D0CB
:107020000D910968B9420ED005910E910821069183
:107030000CE0012108E0022106E0032104E0042124
:1070400002E0052100E0072106910596F9F756F8C0
:1070500006E04B4802F00EFD761C06988642ABD047
:10706000B00007A90F583D1FF9F744F82D78F9F73C
:1070700045F87F2028400628EED13B46143B388B4C
:10708000B9680837B94210D000213A461268BA42AE
:107090001FD01268BA4219D01268BA4218D0091D1E
:1070A0001268BA42F2D1491E13E000213A46126832
:1070B000BA422AD01268BA4224D01268BA4223D007
:1070C000091D1268BA42F2D1491E1EE0491C00E0B7
:1070D000891C00900191102122A00A4602F0CAFCEE
:1070E0003D68BD42B5D029461C39204602F0C2FC9D
:1070F0002868B842ADD0214802F0BCFC2D68BD42E2
:10710000F1D1A6E7491C00E0891C009001911021F3
:107110001CA00A4602F0AEFC9EE7F8F7EFFF002045
:107120000FB0F0BD252D2A2E7320656E7472792064
:1071300073757370656E64207468726561640A00AB
:107140006D7367717565756500000000202D2D2D2C
:107150002D20202D2D2D2D2D2D2D2D2D2D2D2D2D79
:107160002D0A0000252D2A2E2A7320253034642074
:107170002025643A000000008BF000088BFA00081C
:1071800084E70008252D2A2E2A7320253034642018
:107190002025640A00000000F0B597B0032003F03A
:1071A00013FA0546F0A01021F8A2119102F062FC3A
:1071B00001F064FAF7A002F05DFC2D1D002601200D
:1071C0000A9010950FE06D1C1199009101920290A8
:1071D0000395049B143BF7480A4602F04BFC109DB4
:1071E000002E00D153E2002E2C4600D03446F8F792
:1071F00081FF002E06D0311F09787F220A40032A22
:1072000000D042E22668AE4200D13EE23468AC4291
:1072100015942DD02168A9422DD00A68AA4256D0D3
:107220001368AB4200D193E01F68AF4200D1CFE0BA
:10723000079038463F681497AF4200D109E1129099
:10724000149F3F680020AF4200D112E113903846EE
:10725000149F0597129F0697089309920B91149417
:1072600016900490139912910F910E910D9110E1C7
:107270000021139103E0002114940A9A13921291B1
:107280000F910E910D9116910C91F8F737FF371F62
:10729000F8F730FF3F78F8F731FF7F2004460740CA
:1072A000032F2FD133460833F07C726900251F4627
:1072B0003F689F421AD03F689F4214D03F689F4268
:1072C00013D02D1D3F689F42F2D16D1E0EE00022AB
:1072D0000B91149413920A9912910F920E920D929F
:1072E00016920C92D1E76D1C00E0AD1C1199009133
:1072F000019202900395143EE6480A46334602F096
:10730000B9FB109D1598A842169E00D168E7274644
:107310001498041FF8F7EEFE2478F8F7EFFE3C40CF
:10732000032C31D114990B460833C87C4A690025D7
:107330001C4624689C421BD024689C4215D02468BB
:107340009C4214D02D1D24689C42F2D16D1E0FE08A
:10735000002309920B911494139312930A990F919D
:107360000E930D9316930C938FE76D1C00E0AD1CEC
:1073700011990091019202900395149B143BC5480A
:107380000A4602F077FB109D1398002800D027E7EB
:107390000B98041FF8F7AEFE2478F8F7AFFE3C40D8
:1073A000032C32D10B990B460833C87C4A6900255F
:1073B0001C4624689C421CD024689C4216D0246839
:1073C0009C4215D02D1D24689C42F2D16D1E10E008
:1073D0000027089309920B911494139712970F9713
:1073E0000A990E910D9716970C974EE76D1C00E0C9
:1073F000AD1C119900910192029003950B9B143BD7
:10740000A4480A4602F036FB109D1298002800D0CE
:10741000E6E60998041FF8F76DFE2478F8F76EFE8B
:107420003C40032C47D109990B460833C87C4A6974
:1074300000251C4624689C4231D024689C422BD0F5
:1074400024689C422AD02D1D24689C42F2D16D1ED6
:1074500025E000270690089309920B9114943A4670
:10746000139712970F970E970A990D9116970C97ED
:1074700010E01690149F05971298069008930992B1
:107480000B9114941699139112910F910E910D91E5
:107490000A990C910798F8E66D1C00E0AD1C119953
:1074A0000091019202900395099B143B79480A468A
:1074B00002F0E0FA109D0F98002800D090E608989E
:1074C000041FF8F717FE2478F8F718FE3C40032C49
:1074D00024D108990B460833C87C4A6900251C460C
:1074E00024689C420ED024689C4208D024689C42A8
:1074F00007D02D1D24689C42F2D16D1E02E06D1C48
:1075000000E0AD1C11990091019202900395089B37
:10751000143B60480A4602F0ADFA109D0E98002810
:1075200000D05DE60698041FF8F7E4FD2478F8F72C
:10753000E5FD3C40032C4CD106990B460833C87C32
:107540004A6900251C4624689C4236D024689C4227
:1075500008D024689C422FD02D1D24689C42F2D173
:107560006D1E2AE06D1C28E0252D2A2E7320202078
:107570006F776E65722020686F6C6420737573700E
:10758000656E64207468726561640A006D75746567
:1075900078000000202D2D2D2D2D2D2D2D202D2D71
:1075A0002D2D202D2D2D2D2D2D2D2D2D2D2D2D2D18
:1075B0002D0A0000D7ED0008AD1C11990091019231
:1075C00002900395069B143B32480A4602F052FA99
:1075D000109D0D98002800D002E60598041FF8F7CA
:1075E00089FD2478F8F78AFD3C40032C24D10599C5
:1075F0000B460833C87C4A6900251C4624689C4217
:107600000ED024689C4208D024689C4207D02D1DCF
:1076100024689C42F2D16D1E02E06D1C00E0AD1C9E
:10762000059B11990091019202900395143B194812
:107630000A4602F01FFA109D0C98002800D0CFE5F2
:107640000498041FF8F756FD2478F8F757FD3C40DE
:10765000032C00D0C4E504990B460833C87C4A6962
:1076600000251C4624689C4200D1ADE524689C425C
:1076700000D1A8E524689C4205D02D1D24689C42B9
:10768000F0D16D1EA0E5AD1C9EE5F8F737FD00209A
:1076900017B0F0BDD7ED0008F0B58FB00220039011
:1076A00002F092FF044662A0102168A202F0E2F903
:1076B00000F0E4FF68A002F0DDF9271D0026704C01
:1076C000049704E0059E002E049F00D1ADE0002E3B
:1076D0003D4600D03546F8F70DFD002E06D0311F8F
:1076E00009787F220A40022A00D09CE02968B9422A
:1076F00000D198E0079109680026B9421FD008918F
:107700000968B9420596039A069225D0099109683D
:10771000B94216D00A910968B94214D00B91096890
:10772000B94212D00C910968B94210D00D91096884
:10773000B9420ED005910E91082106910CE001216D
:1077400008E0032106E0042104E0052102E006210F
:1077500000E0072106910596F8F7D0FC06E04A48BC
:1077600002F088F9761C06988642ABD0B00007A9D3
:107770000F583D1FF8F7BEFC2D78F8F7BFFC7F20AF
:1077800028400228EED13B46143B388AB9680837B6
:10779000B94210D000213A461268BA421FD012688E
:1077A000BA4219D01268BA4218D0091D1268BA42FA
:1077B000F2D1491E13E000213A461268BA422AD09B
:1077C0001268BA4224D01268BA4223D0091D126846
:1077D000BA42F2D1491E1EE0491C00E0891C00900B
:1077E0000191102122A00A4602F044F93D68BD42F1
:1077F000B5D029461C39204602F03CF92868B84229
:10780000ADD0204802F036F92D68BD42F1D1A6E78F
:10781000491C00E0891C0090019110211BA00A4620
:1078200002F028F99EE7F8F769FC00200FB0F0BDE0
:10783000252D2A2E73207620202073757370656E97
:1078400064207468726561640A00000073656D618C
:1078500070686F7265000000202D2D2D202D2D2DBC
:107860002D2D2D2D2D2D2D2D2D2D2D0A000000001F
:10787000252D2A2E2A7320253033642025643A00D2
:107880008BF000088BFA000884E70008252D2A2ECB
:107890002A7320253033642025640A00F0B58FB0A8
:1078A0000120039002F090FE05465A4810215AA28A
:1078B00002F0E0F800F0E2FE59A002F0DBF82C1D27
:1078C0000020059404E004980028059C00D19EE067
:1078D000002800D004460546F8F70CFC002D059B57
:1078E00007D02946291F09787F220A40012A00D0A3
:1078F0008BE02168994200D187E007910968002454
:1079000099422246039F26D008910968994216D0D1
:1079100009910968994214D00A910968994212D0D4
:107920000B910968994210D00C91096899420ED0C8
:107930000D910A689A420CD00E9208270BE002279C
:1079400008E0032706E0042704E0052702E00627F5
:1079500000E0072722460492F8F7D0FB069704E0E0
:10796000F8F7CCFB641CBC42ADD0A00007A90E58B0
:10797000351FF8F7BFFB29787F220A40012AEFD193
:1079800035462835F8F7BAFB687800903346143B43
:10799000102133A00A4602F06DF829780F20084024
:1079A000042804D8800031A1085802F063F8F56972
:1079B0002846017823290FD14178232909D18178DC
:1079C000232908D1011DC07823280846F1D0481E7C
:1079D00002E0401C00E0801C281A376AC1196420AC
:1079E00048433946F8F77AFE03463069F16B726A0C
:1079F000009101927919091A21A03A4602F03AF849
:107A0000069F641CBC42B0D15DE7F8F777FB00200D
:107A10000FB0F0BD0EEE000874687265616400007E
:107A2000202D2D2D20202D2D2D2D2D2D2D202D2DBA
:107A30002D2D2D2D2D2D2D2D202D2D2D2D2D2D2D83
:107A40002D2D2D20202D2D2D2D2D2D20202D2D2D9A
:107A50002D2D2D2D2D2D2D202D2D2D0A000000003A
:107A6000252D2A2E2A7320253364200052EE00088B
:107A700064EE000889EE0008DAEF00085BEE00080B
:107A8000203078253038782030782530387820201C
:107A900020202530326425252020203078253038DC
:107AA0007820253033640A00F0B593B00A2002F044
:107AB0008BFD044607A0102110A201F0DBFF00F0AF
:107AC000DDFD10A001F0D6FF271D00260120079044
:107AD0000C972EE0252D2A2E732020706572696F79
:107AE00064696320202074696D656F75742020209F
:107AF00020202020666C61670A00000074696D65B3
:107B000072000000202D2D2D2D2D2D2D2D2D2D2001
:107B10002D2D2D2D2D2D2D2D2D2D202D2D2D2D2DA2
:107B20002D2D2D2D2D2D0A00F8F7E8FA002E00D16D
:107B3000D8E11295002E3C4600D03446F8F7DAFA28
:107B40000346002E06D0311F09787F220A400A2AF8
:107B500000D0C4E12568BD4200D1C0E12C68BC4220
:107B600023D02168B94223D00A68BA422AD011939F
:107B70001368BB422DD01868B84234D00668BE42A4
:107B80003ED00F963668BE4248D0002710970F9F10
:107B9000039704900593069208910E9412961098FC
:107BA0000F900D900B900A9046E00026109603E08F
:107BB00000260E94079810900F960D960B960A9635
:107BC00009963BE0002608910E94109607980F90B6
:107BD000F3E70026069208910E9410960F960798E8
:107BE0000D900B9609E000260593069208910E94DD
:107BF00010960F960D9607980B900A9609961CE022
:107C0000002604900593069208910E9410960F9604
:107C10000D960B9607980A9009960EE000260F9F86
:107C2000039704900593069208910E9410960F9670
:107C30000D960B960A9607980990119B1846F8F72F
:107C40005DFA2F1FF8F756FA39787F22119211400A
:107C50000A2913D1F8F752FAA869E969009001914D
:107C60002B46143B1021A4480A4601F003FFE81EEE
:107C70000078C0070C9F08D1A14807E0F8F73EFA4A
:107C80000C9F129DBC4207D150E79C4801F0F2FEC8
:107C9000129DBC4200D149E712950E9D2C1FF8F7AA
:107CA00029FA2178119A11400A2912D1F8F726FAF7
:107CB000A869E969009001912B46143B10218E4878
:107CC0000A4601F0D7FEE81E0078C00708D18C48AC
:107CD00007E0F8F713FA129D1098002808D025E75E
:107CE000864801F0C7FE129D1098002800D01DE7BD
:107CF000089D2C1FF8F7FEF92178119A11400A29E6
:107D000012D1F8F7FBF9A869E969009001912B46B7
:107D1000143B102178480A4601F0ACFEE81E0078BA
:107D2000C00708D1764807E0F8F7E8F9129D0F98E8
:107D3000002808D0FAE6714801F09CFE129D0F98C9
:107D4000002800D0F2E6069D2C1FF8F7D3F9217821
:107D5000119A11400A2912D1F8F7D0F9A869E969F6
:107D6000009001912B46143B102163480A4601F014
:107D700081FEE81E0078C00708D1614807E0F8F7E7
:107D8000BDF9129D0D98002808D0CFE65B4801F0A0
:107D900071FE129D0D98002800D0C7E6059D2C1F8E
:107DA000F8F7A8F92178119A11400A2912D1F8F7A9
:107DB000A5F9A869E969009001912B46143B1021AF
:107DC0004D480A4601F056FEE81E0078C00708D16B
:107DD0004B4807E0F8F792F9129D0B98002808D05D
:107DE000A4E6464801F046FE129D0B98002800D0FC
:107DF0009CE6049C201F1090F8F77CF910990978F4
:107E0000119A11400A2912D1F8F778F9A069E169AD
:107E1000009001912346143B102137480A4601F097
:107E200029FEE01E0078C00707D1354806E0F8F7C4
:107E300065F90A98002807D078E6304801F01AFE64
:107E40000A98002800D071E6039D2C1FF8F752F91C
:107E50002178119A11400A2912D1F8F74FF9A8692F
:107E6000E969009001912B46143B102122480A46F3
:107E700001F000FEE81E0078C00708D1204807E0A6
:107E8000F8F73CF9129D0998002808D04EE61B48E7
:107E900001F0F0FD129D0998002800D046E62C1F45
:107EA000F8F728F92178119A11400A2900D03BE609
:107EB000F8F724F9A869E969009001912B46143B71
:107EC00010210D480A4601F0D5FDE81E0078C007D4
:107ED00001D10B4800E0094801F0CCFD26E6184628
:107EE000F8F70CF903F052FD014606A001F0C2FDBF
:107EF000002013B0F0BDC0466DEE000803EE000890
:107F000001EE000863757272656E74207469636BAC
:107F10003A3078253038780A00000000002807D071
:107F20000168002904D04168002901D000210160C6
:107F300070470146002000290FD00A68002A0CD0A3
:107F40004A68002A09D08868C968884204D001D9E3
:107F5000421A01E0511A0A18501E704701460020CB
:107F600000290ED00A68002A0BD04A68002A08D0DF
:107F70008B68C968994204D001D9C81A704788181B
:107F8000C01A704701460020002907D00A68002A5D
:107F900004D04B68002B01D0886810187047014648
:107FA000002000290ED00A68002A0BD04A68002A57
:107FB00008D08868C968814201D9081A704781428F
:107FC00001D300207047101A704703460020002B91
:107FD00009D0002907D0002A05D0002006C3186068
:107FE0005860986001207047F0B581B000240028E7
:107FF00036D005460068002832D0002A30D00E4620
:1080000000292DD0696800292AD0AF68EB68BB42EF
:1080100026D0BB4200D85B18BB4221D0C91BDC1B59
:10802000944200D31446A14200D321460091C119C5
:108030003046009AF8F712F90098221A13D0301837
:1080400029681646F8F70AF96868864200D30026C0
:10805000AE602B69002B03D00021284622469847AA
:10806000204601B0F0BDC61968688642EFD2EFE73E
:1080700010B50024002819D00268002A16D0002963
:1080800014D04268002A11D08368C4689C420FD182
:1080900000248C4200D30C4619198A1A0ED2816032
:1080A0000369002B02D0002122469847204610BDCC
:1080B00000D8A418E41A8C42EDD2EDE71146816095
:1080C0000369002BEFD1F1E7F0B583B0044600203F
:1080D000002C3FD00D46216800293BD0002A39D022
:1080E000002D37D06368002B34D0A668E76802976C
:1080F000BE421F4602D028D9029FF71B7E1E29D000
:1081000002981F1A964200D31646B74200D337464C
:10811000081829463A46F8F7A1F80196F61B1BD035
:10812000E91920683246F8F799F86068864200D36A
:108130000026E6602369002B14D001212046019C13
:1081400022469847204603B0F0BD029FDF1BBF19AF
:108150007E1ED5D103B0F0BD02983E1860688642FD
:10816000E6D2E6E7019803B0F0BD000082B0062435
:108170000C4D01260CA320462946324605F0B2FCE0
:10818000114800681149F8F7A9FA009010A3204699
:108190002946324605F0A6FC7D20C00003F038FADF
:1081A000FAE7C046A8E70008746573742043495590
:1081B0003332204C3035312052542D546872656171
:1081C00064210D0A000000000C00002040420F0056
:1081D00053797374656D436F7265436C6F636B2085
:1081E0003D202564204D485A0A000000B0B5054CDA
:1081F000054DA54203D201CD8047A542FBD3FFF731
:10820000B5FFB0BD88FB00084CFB0008F0B585B099
:1082100002900078002870D04E4804684E480568E7
:10822000A54200D393E000204C4E0390049006E05A
:1082300048490C6803900C35A54200D380E02F68B4
:10824000062238463146F8F766F80028F3D1029E38
:108250003046F8F74CF80246BF1D30463946F8F76D
:108260005AF8002801D03D4EE5E703980028049C09
:1082700003D13846F8F73BF83C46039021780029B3
:108280002046364E04942CD000203A5C002A20D0A0
:1082900091421ED121184B78002B1CD03A185478EB
:1082A000002C18D0A34216D18B78002B15D09478CF
:1082B000002C12D0A34210D1CB78002B0FD0D27853
:1082C000002A0CD093420AD10979001D0029049C90
:1082D000DBD1201805E0481C02E0881C00E0C81C27
:1082E000049C01901EA0394601F0C4FB0198001BBC
:1082F000039988429CDB08469AE7D94801F0BAFB0B
:108300001448076814480568BD4214D2134C02E0B3
:108310000C35BD420FD22E68062230462146F7F7B3
:10832000FAFF0028F4D16A68B11DD14801F0A2FB20
:1083300008480768ECE7CF4801F09CFB05B0F0BDAA
:108340000499002903D00298039A02F069FD05B050
:10835000F0BDC046DC010020D801002044F0000838
:1083600025730A00F0B58BB0002938D0002202E056
:10837000521C914233D0845C202CF9D0092CF7D0C8
:10838000831802938D1A691EAB1E0195EE1E0025FF
:10839000E4B2092C2FD0202C2DD0019CAC4221D04E
:1083A0004419A4186778092F20D0202F1ED0A94285
:1083B00018D0A778092F1DD0202F1BD0AB4211D089
:1083C000E778092F00D1C2E0202F00D1BFE0AE42F4
:1083D00008D024792D1DE4B2092CDCD10BE000205B
:1083E0000BB0F0BD019D002D08D1B4E06D1C002D37
:1083F00004D1B0E0AD1C002D00D1ACE0724804689F
:1084000072480668A64200D3A5E0A81D009003E0CC
:108410000C36A64200D39EE03768062238466C49E7
:10842000F7F779FF0028F3D1B81D02992A46F7F72C
:1084300072FF0028ECD10098385C0028E8D1B068C1
:108440000090002800D186E000270A970997089736
:108450000797069705970497039738460299019A5C
:108460009042024605D8019A03E000230B70401C9D
:10847000491C0B78202B01D0092B02D18242F4D168
:108480001046082F00D388E0019A904200D393E071
:10849000222B09D1BB004A1C03ACE250431C019CB7
:1084A000A34224D3002623E0BA0003AB9950019ADB
:1084B0009042034600D8019B1A1AC31A5C1C7F1C09
:1084C0000023CD5C092D0FD0202D0DD09A4275D000
:1084D000CD186E78092E30D0202E2ED0E5186DD014
:1084E0009B1CCD5C092DEFD1C018C91828E00126CE
:1084F000497802E000265178521C222915D0019CAF
:10850000A34212D25C2904D15178222903D0184603
:1085100002E0184603E0801C222900D1521C431CB3
:1085200001998B42E6D20126E5E77F1C002E45D05B
:1085300000211170801C511C05E0C018401C691CF2
:10854000019A90423AD2019A904288D336E0ED1CCB
:10855000002D00D052E70298027820210A43202AF9
:1085600012D042780A43202A09D082780A43202A6E
:1085700007D0C2780A43202A05D0001DECE7401C32
:1085800002E0801C00E0C01C002404701BA00299C3
:1085900001F070FAE0430BB0F0BD0EA001F06AFAF2
:1085A00003AC14A63D4602CC304601F063FA6D1EC2
:1085B000F9D1114801F05EFA002FCCD003A938465A
:1085C000009A90470BB0F0BDDC010020D8010020DC
:1085D00044F00008546F6F206D616E7920617267FE
:1085E000732021205765206F6E6C79205573653A92
:1085F0000A0000002573200084E7000825733A2054
:10860000636F6D6D616E64206E6F7420666F756E42
:10861000642E0A00F0B581B0114801F02BFA114820
:10862000076811480568BD4214D2104C02E00C35B1
:10863000BD420FD22E68062230462146F7F76BFE68
:108640000028F4D16A68B11D094801F013FA054801
:108650000768ECE7074801F00DFA002001B0F0BD13
:108660001DF00008DC010020D801002044F00008C3
:1086700038F0000884E700080120704710B5194C55
:10868000204601F0F7F9204601F0F4F9204601F008
:10869000F1F9204601F0EEF9204601F0EBF9204611
:1086A00001F0E8F9204601F0E5F9204601F0E2F991
:1086B000204601F0DFF9204601F0DCF9204601F008
:1086C000D9F9204601F0D6F9204601F0D3F9204629
:1086D00001F0D0F9204601F0CDF9204601F0CAF9A9
:1086E00010BDC04683EE000870B50446224DE86810
:1086F000A04227D82869A0422CD96088002804D03D
:1087000032A02649A32200F0DBFA6168E86842182B
:10871000A2420FD05388002B0CD12B699A4209D06A
:108720006969914200D16C6151686160231A526895
:1087300082189360A2688318A34202D05E88002E3C
:1087400011D070BD0DA01549A12200F0B9FA286919
:10875000A042D2D812A01149A22200F0B1FA60883A
:108760000028CDD1D1E76E69A64200D16B61596076
:1087700061684018826070BDFC0100202872745F3F
:1087800075696E74385F74202A296D656D203E3DD1
:1087900020686561705F707472000000DBF500088E
:1087A0002872745F75696E74385F74202A296D654C
:1087B0006D203C202872745F75696E74385F742078
:1087C0002A29686561705F656E6400006D656D2DB6
:1087D0003E75736564203D3D20300000F0B58DB0DE
:1087E000079316460F460546149C600605D5F1A072
:1087F00002900123E00605D405E0FCA002900123CD
:10880000E00600D59C43E00701D0302000E02020A6
:108810000890A00700221399069100280597049458
:108820004ED403930092002E00D18AE007980A28C4
:10883000019259D103200790029C0A2730463946FD
:10884000F7F74CFF4743F11B615C09AA079FD21958
:10885000D21E11700A2E79D30A21F7F73FFF605C10
:1088600009A9C919891E0870642E73D36421304682
:10887000F7F734FF0A21F7F731FF605C09A9C9193E
:10888000491E0870F0087D28059F00D28DE07D20EC
:10889000C1003046F7F722FF0A21F7F71FFF605C9F
:1088A00009A9079FC8553046DA49F7F717FF3F1D5A
:1088B0000797D8498E420646BFD2079CE41E4AE07D
:1088C000002E07D4600734D4200700220028A8D542
:1088D00020202FE07642002003902D2000901A46A1
:1088E00007980A280192A5D00324029B0F20314645
:1088F0000140595C09AA1219D21E1170310927D002
:108900000140595C09AA1219921E1170310A25D032
:108910000140595C09AA1219521E1170310B1ED068
:108920000140585C09A90855241D360CDED1E41E0F
:1089300015E02B200090002003901A46002E00D056
:1089400074E709A830210170012409E0BC1E02E08F
:10895000A41E04E07C1E019A059F01E0641E019A9A
:10896000129806998C42214600DC0699401A112380
:10897000049E1E4231D1002805DC00231A40821AD1
:10898000501E05DA29E001231A40821A501E24DB0A
:10899000032313401CD0BD4201D2202028706E1C3E
:1089A000012B05D1901E354612E0019A079CD7E7AE
:1089B000BE4201D220203070AE1C022B02D1D01E4C
:1089C000354605E0BE4201D220203070101FED1C5C
:1089D0000023DB43042A2BD21846039A002A06D030
:1089E000049AD2060CD5069A944258DB78E0BD4230
:1089F00001D2009A2A706D1C401E049AD206F2D44D
:108A0000431E10DB0322024040D0BD4201D2089B2E
:108A10002B706E1C012A2FD1831E35460022D243B3
:108A2000042838D326E11846069A944237DB57E0EB
:108A3000001D03E0001F2D1D0328CDDDBD4209D31D
:108A40006A1CBA420BD3AA1CBA420DD3EA1CBA4222
:108A5000F0D20EE020222A706A1CBA42F3D22026FD
:108A60001670AA1CBA42F1D220261670EA1CBA422D
:108A7000E0D220261670DDE7BE4201D2089B33709B
:108A8000AE1C022A00D0EAE0C31E35460022D243C3
:108A9000042800D3EEE01046069A944220DA0A1B1E
:108AA00003231340E2438A18002B16D0BD4201D2A3
:108AB00030262E706E1C012B04D1491E3546032A28
:108AC0000ED3AEE0BE4202D230273770059FAE1CF7
:108AD000022B00D094E0891E3546032A00D3A0E083
:108AE0000699002925D009A9091F04E0241F2D1D7E
:108AF000221D042A1DD9BD4202D20A19D2782A7039
:108B00006A1C022C14DBBA4202D20B199B78137038
:108B1000AA1C032C0CD3BA4202D20B195B78137037
:108B2000EA1C042C04D3BA42E0D20B5D1370DDE7DB
:108B30001546012826DB032101400BD0BD4201D29E
:108B400020222A706A1C012908D1411E15460428DA
:108B500018D31AE00146042814D316E0BA4201D211
:108B600020231370AA1C022904D1811E1546042853
:108B700008D30AE0BA4201D220211170C11EED1CB7
:108B8000042802D228460DB0F0BD481E05E0001FA3
:108B90002D1D0121C9438842F4D2BD4214D3691C62
:108BA000B94216D3A91CB94218D3E91CB942EED276
:108BB00019E0C04630313233343536373839414226
:108BC000434445460000000020212970691CB94239
:108BD000E8D220220A70A91CB942E6D220220A70EB
:108BE000E91CB942D3D220220A70D0E730313233A7
:108BF00034353637383961626364656600000000D9
:108C0000BE4201D230233370C91EED1C032A08D2A4
:108C100066E7C04610270000091F2D1D8C4200DBAF
:108C20005EE7BD4209D36A1CBA420BD3AA1CBA4202
:108C30000DD3EA1CBA42EFD20EE030222A706A1C31
:108C4000BA42F3D230231370AA1CBA42F1D23023B5
:108C50001370EA1CBA42DFD230231370DCE7BE4245
:108C600001D2089A3270031FED1C0022D24304285F
:108C700000D210E7181D04E0001F2D1D032800DCA2
:108C800009E7BD4209D36B1CBB420BD3AB1CBB42F3
:108C90000DD3EB1CBB42EFD20EE0089B2B706B1C7C
:108CA000BB42F3D2089E1E70AB1CBB42F1D2089EA1
:108CB0001E70EB1CBB42DFD2089E1E70DCE700007A
:108CC00010B582B013460A46014601A8002404707C
:108CD0000E480468002C05D0084611461A46A047E5
:108CE00002B010BD0AA000F0C5FE01A8007800285F
:108CF000F6D101A800780028F2D101A80078002858
:108D0000EED101A800780028EFD0E9E7C8170020CD
:108D10002825732920617373657274696F6E2066EC
:108D200061696C65642061742066756E6374696F37
:108D30006E3A25732C206C696E65206E756D6265C8
:108D4000723A2564200A0000B0B504464C43204620
:108D500000F0F0FE0546002804D0002128462246F7
:108D600001F068F82846B0BDB0B5044C044DA542EA
:108D700003D201CD8047A542FBD3B0BD4CFB000818
:108D80003CFB0008014800687047C046DC03002037
:108D9000B0B50446002817D0204601F049FC092848
:108DA00006D095204000421CD6481549FFF788FFA1
:108DB0002220215C0020002912D022462232491EA6
:108DC000117009060ED0B0BD95204200CB480C4969
:108DD000FFF776FF204601F02BFC0928E1D1E7E7F9
:108DE000C043B0BD616B00250029284605D0204650
:108DF0008847002801D0811DE5D12584B0BDC0463B
:108E0000A0F8000880B5092101F076FB80BD0000C4
:108E1000F0B583B00D46044600281AD0204601F074
:108E200007FC09281FD1E08BC10624D4E16A002980
:108E300028D020468847002823D006460094019079
:108E4000032031490122314B04F04CFE304603B07F
:108E5000F0BD2A482A49E422FFF732FF204601F0FC
:108E6000E7FB0928DFD027482549E522FFF728FF3F
:108E7000E08BC106DAD50146208C0827090708D403
:108E80000FE0E08B10210143E183208C08270907C4
:108E900007D50146394004D00620C643304603B00A
:108EA000F0BD010705D51A492A460A4008409042FC
:108EB00010D0226B002A0AD0204629469047064649
:108EC000002808D0B01D06D0304603B0F0BD1048D1
:108ED0000540258400262220215C491C2154208C39
:108EE00038432084C8B28842EED0FF22183209A04D
:108EF0000349FFF7E5FE304603B0F0BD04F8000873
:108F000006F9000857F8000892F8000813F800085E
:108F10000F0F00006465762D3E7265665F636F75A6
:108F20006E7420213D203000F0B581B003460C481E
:108F30000024192505770B4D0B4E0C4F44628462BB
:108F4000C462046344638763C663056442648164E6
:108F50000322194600F04EF8204601B0F0BDC0468D
:108F6000E0030020694E0008C14F00084D4F000883
:108F7000F0B581B01C4615460E460746002812D0B3
:108F8000384601F055FB092818D12220385C00280A
:108F90001FD02346BC6B002C23D0384631462A46CE
:108FA000A04701B0F0BD2B20C20054481049FFF784
:108FB00087FE384601F03CFB0928E6D02B20C00094
:108FC000421C50480A49FFF77BFE2220385C0028EB
:108FD000DFD10520C043401D01F07EFE002001B01E
:108FE000F0BD0520C04301F077FE002001B0F0BDC8
:108FF00048F80008F0B581B00027FC43002808D0ED
:109000000E46054600920921304601F075FA002807
:1090100002D0204601B0F0BD09212846324601F0B9
:1090200027FB22202F540098E8832F843C462046BB
:1090300001B0F0BDB0B50C460546002807D0284663
:1090400001F0F6FA09280DD16C620020B0BDFF22B4
:10905000C4322A480849FFF733FE284601F0E8FAEF
:109060000928F1D0FF20C430421C26480249FFF7EE
:1090700027FE6C620020B0BDB0F80008F0B581B0EA
:109080001C4615460E460746002812D0384601F009
:10909000CFFA092818D12220385C00281FD0234697
:1090A000FC6B002C23D0384631462A46A04701B03D
:1090B000F0BDFF22843211481149FFF701FE384606
:1090C00001F0B6FA0928E6D0FF208430421C0D4892
:1090D0000B49FFF7F5FD2220385C0028DFD1052081
:1090E000C043401D01F0F8FD002001B0F0BD052097
:1090F000C04301F0F1FD002001B0F0BD04F800080C
:10910000E4F8000857F8000880B5F6F7F3FFF449D3
:109110004A88521C4A80F6F7F1FF80BD70B51546AB
:109120000E460446002804D1084809A10C4AFFF75E
:10913000C7FD04212046324601F09AFA21461C312F
:1091400065740020E1612162606270BD6CF100080D
:1091500072745F6576656E745F696E697400000095
:10916000B3030000F0B589B007920D46074604939B
:109170000893F6F7BFFF06904920040102F098FA21
:10918000002809D18148824E314600F073FC8148A5
:1091900031462246FFF794FDF6F7ACFF064600F095
:1091A0004DFC002805940ED07B482C463D46784F58
:1091B000394600F05FFC774839462F462546059C26
:1091C0002246FFF77DFD3046F6F798FF0698F6F742
:1091D00095FF002F2FD0384601F02AFA042834D109
:1091E0000120C443002D39D0039502F061FA0646F0
:1091F0000020B06369480168002901D038468847DB
:109200003D460E98019006963D360296079EF7075A
:10921000F6F770FF0246002F24D1B0072F4661D425
:109220001546059A2332F5485949FFF749FD2A4664
:10923000039B029D1EE0E21C98485549FFF740FD44
:10924000384601F0F5F90428CAD0221D9648504945
:10925000FFF736FD0120C443002DC5D1641C204614
:1092600009B0F0BD2F46686A0146039B1940994238
:10927000029D3CD0049800284BD005920798E872D4
:10928000069843647C7C02F0ADFA38461C30002C12
:1092900047D0012C4DD101460968814241D021229D
:1092A0008B5C2C789C4214D30968814239D08B5C4A
:1092B0002C789C420DD30968814232D08B5C2C788B
:1092C0009C4206D3096881422BD08A5C2B7893425A
:1092D000E2D24868069B1A461C320260D9611862C5
:1092E0004A6026E0786A039B1842029DC2D0019929
:1092F000002902D018400860786A0799E9720C4684
:1093000001461940069D6964610731D5984378622A
:109310002EE0069884631046F6F7F0FE204609B06A
:10932000F0BD396A069B1A461C320A60D861196280
:109330003A6204980128069D09DB2C46543400212A
:1093400008AA204602F09EFB204602F0B3FC0598D6
:10935000F6F7D4FE01F086FAAC6B002C00D07EE765
:10936000F6F7C8FE02460199002901D0686C086032
:109370001046F6F7C3FE0A480168002901D03846B6
:109380008847AC6B204609B0F0BDC046EEF000083F
:109390002AF40008FFEB0008B1F000086418002070
:1093A00060180020F0B583B00F460446002847D06F
:1093B000204601F03DF904284CD10920C043002F7C
:1093C00052D00090F6F796FE0290606A38436062D1
:1093D00036480168002901D020468847E6692746BB
:1093E0001C37BE424ED000200190304609E0826A10
:1093F000656A2B4613400668934213D0BE4230463E
:1094000035D02C21415CCA07F1D18A0740D5826A48
:10941000656A2A4004D10668BE423046F1D126E092
:1094200082620668490701D5954365621C3802F0DF
:10943000F7F80120BE42D7D10298F6F75FFE1CE094
:1094400016481749174AFFF73BFC204601F0F0F891
:109450000428B2D01348421C13481149FFF730FCCE
:109460000920C043002FACD1093003B0F0BD0298F1
:10947000F6F744FE0198C00701D001F0F3F900208F
:1094800003B0F0BD0298F6F739FE002003B0F0BD3E
:109490000298F6F733FE009803B0F0BD6CF10008B7
:1094A0009FF1000827040000D1F300085C18002099
:1094B00010B5F6F71FFE0A4C6188491E618009B29B
:1094C000002902DDF6F71AFE10BD00216180F6F7D3
:1094D00015FE60680028F7D001F0C4F910BDC04641
:1094E00044020020F0B585B0002876D00446F6F797
:1094F00001FE06468B20850000F0A0FA002809D066
:109500003C483D4F394600F0B5FA3C4839462A46BA
:10951000FFF7D6FB3046F6F7F1FDA00704D0AA1CF2
:1095200037A03549FFF7CCFB414EF068A04202D886
:109530003069A04204D82A1D3E482F49FFF7C0FBDE
:109540007168002901D020468847F068A04244D8BD
:109550003069A04241D90195304620300021039165
:10956000C943049001F0DAFA27460C3FF520410187
:1095700025460A3D2888002802D03888884217D01E
:1095800002912DA000F076FA3B882A8831A0394656
:1095900000F070FA2888002821D038880299884283
:1095A00006D0019A23323A481349FFF789FB029902
:1095B0003980039828807069874200D27761F0680B
:1095C000083C21680818381AB1694018B06138465B
:1095D000FFF78AF8049801F051FA05B0F0BD019A3E
:1095E000223228A00449FFF76BFB38880299884291
:1095F000D7D1DDE7B1F00008D3F50008FFEB000894
:1096000028282872745F75626173655F7429726DB2
:10961000656D292026202852545F414C49474E5FF2
:1096200053495A45202D20312929203D3D20300025
:10963000FC01002034F50008746F20667265652017
:109640006120626164206461746120626C6F636B8D
:109650003A0A00006D656D3A203078253038782C54
:10966000207573656420666C61673A2025642C2040
:109670006D6167696320636F64653A2030782530D7
:1096800034780A006D656D2D3E75736564000000C9
:1096900006F5000880B503F0EDFB02F0C3FF7D2066
:1096A000C1000B480068F7F719F8401E010E08D1F9
:1096B000084948600848FF2202700720086000201F
:1096C0008860FFF751FB0548054901F0EFFB80BDBD
:1096D0000C00002010E000E023ED00E0103100203D
:1096E0000040002010B582B001A8002404700B488F
:1096F000FEF734FC002809D0084801AC01222146BD
:10970000FEF772FC2478204602B010BD04480068C1
:10971000E14301F003FA204602B010BDA802002088
:1097200070020020F0B503AF85B06E46054601F02B
:109730004CFB04460A21F6F7D1FF2018113007210F
:1097400088436946081A8546002C1BD0032122460F
:109750000A403260042C306116D200231946326868
:10976000002A63D01C46EA5C0A2A04D10D23306922
:1097700043543069491C42544A1C3368012B38D188
:10978000114653E0002151E08C43746000231946D8
:10979000B56006E0F3680255611C1B1D72689A42B1
:1097A000DDD0EA5C0A2A02D10D244454491C4254FB
:1097B000EA1854784D1C0A2CF36004D10D2330694B
:1097C000435530698D1C44559478691C0A2C04D18A
:1097D0000D23306943543069A91CB5684454D278CC
:1097E0004C1C0A2AD6D10D233069035530698C1CD4
:1097F000D0E763195C780A2C04D10D203569A85490
:109800008A1C00E03569AC54511C3068022801D133
:1098100030690BE09B780A2B04D10D203469605429
:10982000911C00E034696354491C2046FAF7AEFEEF
:10983000FE1F053EB546F0BD0446C16913A000F009
:1098400019F9A16915A000F015F9616917A000F0D8
:1098500011F9216919A000F00DF9E1681BA000F0D1
:1098600009F9A1681DA000F005F961681FA000F0CA
:1098700001F9216821A000F0FDF82448016824A026
:1098800000F0F8F8FEF70AF8FEE7C0467073723A87
:10989000203078253038780A000000002070633AC4
:1098A000203078253038780A00000000206C723AA9
:1098B000203078253038780A000000007231323AC2
:1098C000203078253038780A000000007230333AB2
:1098D000203078253038780A000000007230323AA3
:1098E000203078253038780A000000007230313A94
:1098F000203078253038780A000000007230303A85
:10990000203078253038780A000000004802002016
:1099100068617264206661756C74206F6E20746873
:10992000726561643A2025730A00000080B507481B
:1099300001682F220A43026000BF00BF00BF04A0DD
:1099400004490022FFF7F0FA80BDC0462C10024007
:1099500070696E00A4DE000870B5121D0724A243D2
:1099600014461C3C002525601646203E31601146F9
:109970002439124E0E60114628390E6011462C39DA
:109980000E60114630390E60114634390E601146B2
:1099900038390E6011463C390E60114640390E6070
:1099A0006560A560E560141F01252D06256014463D
:1099B000083C20600C3A1360084670BDEFBEADDE77
:1099C000B0B5104C211F0D6868437D21C900F6F722
:1099D00085FE2268002101E0814212D213462268EE
:1099E0009A4208D122689A4205D122689A4202D14D
:1099F00022689A42F3D05918891A9A42ECD349192D
:109A0000EAE7B0BD18E000E010B5E1204002002414
:109A10002146FBF7C3F8204610BD000010B5F6F74D
:109A200069FB044612480178491C0170406800280F
:109A300000D080472046F6F761FB10BD10B5F6F761
:109A400059FB0B490C78F6F759FB204610BDC04670
:109A500010B5F6F74FFB044605480178491E017022
:109A60008068002800D080472046F6F747FB10BDED
:109A7000F001002083B070B581B0054605A80EC086
:109A800005AB009310487F2421462A4602F0E4F9F2
:109A90000346274D286800280DD0068C402131430D
:109AA00001847F2B00D323460021074AFFF7E6FA03
:109AB0002868068402E00448FFF734FE01B070BC59
:109AC00001BC03B00047C046D4170020F0B581B0F8
:109AD00000282BD00246164C2068002816D0058C92
:109AE0004021294301840021CB43565C002E12D033
:109AF00056187778002F10D0B778002F0FD0F6784F
:109B00001B1D091D002EF0D1D11809E01046FFF7EA
:109B100009FE01B0F0BD511802E0711C00E0B11C5B
:109B20008B1A0021FFF7AAFA2068058401B0F0BD66
:109B3000DC030020F0B585B00027002834D00446AF
:109B4000F6F7D8FA0546FFF779FF00280AD06848EB
:109B5000684E3146FFF78EFF2320C200664831462B
:109B6000FFF7AEF82846F6F7C9FAE41C0320844351
:109B7000624EB068844217D83046203000210391ED
:109B8000C943049000F0CAFF0C2C00D80C24B06824
:109B9000F1680190051B70690290461AAE4209D324
:109BA000049800F06BFF039F384605B0F0BDAA4251
:109BB0001646F5D28F197A6878880028F7D133468F
:109BC0000C33D01AA042F2D325460C350095F5256A
:109BD0006D01039525461835A8420CD201207880E6
:109BE000901B464DAA691218AA61E8699042009E2E
:109BF000039B1AD31AE01D19039B4B53481942606B
:109C0000002242807D60866001227A804068019A4D
:109C10000C32904201D008188560384DA869009E2A
:109C20003218AA61E869904200D2EA613B802320A1
:109C3000C0000390029887422CD143882A69002BE8
:109C40001ED090421CD0406808184388002B16D0C4
:109C5000904214D0406808184388002B0FD09042DF
:109C60000DD0406808184388002B08D0904206D0D9
:109C7000406808184388002B01D09042E3D1686106
:109C8000002B07D0904205D0039A6A321CA01949D4
:109C9000FFF716F8049800F0F1FEF01929698842E0
:109CA000039E05D932466E321F481249FFF708F865
:109CB00038460C300546800705D032466F321B48C7
:109CC0000C49FEF7FDFFB80705D0703618A009490A
:109CD0003246FEF7F5FF09480268002A2F4600D1F8
:109CE00062E7384621469047384605B0F0BDC04689
:109CF000B1F000082AF50008FFEB0008FC01002085
:109D000028286C66726565203D3D20686561705F3E
:109D1000656E6429207C7C2028216C667265652D27
:109D20003E7573656429290090F50008BDF40008AC
:109D300028282872745F75626173655F74296D6588
:109D40006D292026202852545F414C49474E5F53CD
:109D5000495A45202D20312929203D3D2030000041
:109D6000F0B5814211D28D1885420ED9002A5FD0FC
:109D7000032616408118002E39D04B1E6C1E277802
:109D80001F70012E37D1511E42E0002A50D003230C
:109D9000134009D00C780470012B0AD1431C491CD4
:109DA000541E042A16D243E003461446042A11D254
:109DB0003EE04C784470022B05D1831C891C941E14
:109DC000042A07D234E08B788370C31CC91CD41ECC
:109DD000042A2DD30A781A704A785A708A789A70B1
:109DE000CA78DA701B1D091D241FF3D120E02C4610
:109DF0000B4611460CE08B1EAC1E27781F70022EFE
:109E000001D1911E04E0CB1EEC1E21781970D11EE9
:109E1000042A0DD31A1F231FDC78D4709C78947009
:109E20005C7854701C781470121F1B1F091FF3D12B
:109E3000F0BD000070B50446042A18D30320234661
:109E4000034014D1CDB2344B6B43102A11D31546C5
:109E5000103D2E09761C06400DD023606360A36080
:109E6000E360012E09D1204610302A4616E0204634
:109E700048E020462AE0204610E023616361A361A8
:109E8000E361022E03D1203A2046203006E023620F
:109E90006362A362E362303A20463030302D13D340
:109EA000036243628362C362036343638363C36386
:109EB000036043608360C360036143618361C36186
:109EC0004030403A0F2AEBD8042A1BD3054608C578
:109ED000161F042E0FD343601546083D042D0DD3E5
:109EE000836015460C3D042D0AD3C360103A103030
:109EF000032AEBD806E02846324603E0083000E0AB
:109F00000C302A46002A04D0CBB211461A46F6F786
:109F1000C5F9204670BDC04601010101F0B581B010
:109F200014460E46054607462637002809D0032169
:109F30002846324600F09CFB28461C30E861286227
:109F40000DE00B480BA10F4AFEF7BAFE00200321DB
:109F5000324600F08DFB20201C21016009600020AA
:109F6000A8620121A984FF2139806C7401B0F0BD81
:109F70007DF1000872745F6D757465785F696E6954
:109F8000740000001D020000F0B581B004464F4D82
:109F900000284AD0204600F04BFB032804D06A1F5B
:109FA000D1484B49FEF78CFEF6F7A4F8064601F0BF
:109FB0007FFB002809D1C748454F3946FFF75AFDB6
:109FC000C64839462A46FEF77BFEF6F793F8074661
:109FD000FFF734FD002809D0C1483D4D2946FFF761
:109FE00049FDBE482946394AFEF76AFE3846F6F76B
:109FF00085F83046F6F782F801F05AFB0746F6F787
:10A0000079F8054633480168002901D02046884781
:10A01000A06A874214D00220C043841CBC63284637
:10A02000F6F76CF8204601B0F0BDAA1FAD482849EC
:10A03000FEF746FE204600F0FBFA0328AFD1B3E757
:10A04000264626367078401E7070000606D02846D8
:10A05000F6F754F80024204601B0F0BD3D20385CEE
:10A060003178814204D002213846324601F05EF850
:10A07000E16920461C30814215D008461C38A06298
:10A080002122895C31707178FF2910D0491C7170D0
:10A0900001F0C6FA2846F6F731F800F0E3FB002499
:10A0A000204601B0F0BDA08C0B49884207D128465C
:10A0B000F6F724F80220C443204601B0F0BD002189
:10A0C000A162FF213170401CA084C0E73203000070
:10A0D0001BF200085C180020FFFF0000F0B585B0FF
:10A0E000044603910491F6F705F805465320C6008F
:10A0F00001F0DEFA002809D17648774F3946FFF79C
:10A10000B9FCB94839463246FEF7DAFDF5F7F2FFF9
:10A110000746FFF793FC002808D0B1486E49FFF7C7
:10A12000A9FCB1486C493246FEF7CAFD3846F5F73E
:10A13000E5FF2846F5F7E2FF002C3ED0204600F070
:10A1400077FA032804D0321D67486349FEF7B8FD4B
:10A1500001F0AEFA0746F5F7CDFF06466348016801
:10A16000002901D020468847214626310025BD63BD
:10A17000A06AB84208D0A28C002A29D0A762501E3B
:10A18000A0843D20385C08704878FF2807D130460D
:10A19000F5F7B4FF0220C543284605B0F0BD401CCA
:10A1A00048703046F5F7AAFF514801680029F3D0FE
:10A1B00020468847284605B0F0BDF21C494846496C
:10A1C000FEF77EFD204600F033FA0328BBD1BFE73F
:10A1D0000399002943D0019600953D21425C795CAA
:10A1E0003D463D35914203D202212A4600F09EFFB2
:10A1F000667C384601F0F6FA029420461C30002EA8
:10A2000037D0012E029C019E3CD101460968814253
:10A2100054D021228B5C2C789C4214D30968814253
:10A220004CD08B5C2C789C420DD30968814245D080
:10A230008B5C2C789C4206D3096881423ED08A5CB4
:10A240002B789342E2D248683A461C320260F961A8
:10A2500038624A60029C0398012816DA20E0022046
:10A26000C043451CBD633046F5F748FF284605B09E
:10A27000F0BD029C216A3A461C320A60F8613962DC
:10A280002262019E039801280ADB3C4654340021D7
:10A2900004AA204601F0F6FB2046029C01F00AFDCC
:10A2A0003046F5F72BFF00F0DDFABD6B002D00D036
:10A2B00072E7F5F71FFF0646009D72E7029C216AD0
:10A2C0003A461C320A60F86139622262039801281A
:10A2D000DBDAE5E7EEF00008B9F10008FFEB000873
:10A2E000B1F000087DF1000838F40008641800207F
:10A2F00060180020F0B581B000910546F5F7FAFE30
:10A300000646FFF79BFB00280AD0AC48354F39467C
:10A31000FFF7B0FBDF204200AA483946FEF7D0FC29
:10A320003046F5F7EBFEC14C2078A84230D0207CB7
:10A33000A84201D110342BE02020205CA84201D19A
:10A34000203425E03020205CA84201D130341FE0C9
:10A350004020205CA84201D1403419E05020205C0C
:10A36000A84201D1503413E06020205CA84201D102
:10A3700060340DE07020205CA84201D1703407E009
:10A38000DF204000021DF3481649FEF799FC002427
:10A39000E068FFF7CFFB064600281ED0E2680027E2
:10A3A00030463946FFF746FD777435741022304643
:10A3B000009900F035FDED480168002901D03046D4
:10A3C0008847F5F797FE61687161324614324A603A
:10A3D0006260211DB161F5F791FE304601B0F0BD1C
:10A3E000B1F0000832F60008FFEB000810B5044693
:10A3F00000281CD010202056002822D43D48016897
:10A40000002901D02046884700202074F5F772FE0D
:10A410006169A2694A60A2691160214614316161D3
:10A42000A161F5F76BFE2046FFF75CF810BDF9203F
:10A4300042000A480A49FEF743FC10202056002833
:10A44000DCD5F9204000421C06A00549FEF738FC87
:10A45000284801680029D5D1D6E7C04611F6000882
:10A4600045F6000821286F626A6563742D3E747991
:10A47000706520262052545F4F626A6563745F43A3
:10A480006C6173735F537461746963290000000029
:10A4900010B50446002815D016480168002901D0DF
:10A4A0002046884700202074F5F724FE6169A269E0
:10A4B0004A60A2691160214614316161A161F5F71A
:10A4C0001DFE10BDCF204200044805A1FEF7F8FB99
:10A4D000084801680029E3D1E4E7C04611F6000806
:10A4E00072745F6F626A6563745F646574616368E8
:10A4F0000000000058180020F0B581B00446944FC9
:10A500003878884229D0387C884201D1103724E03D
:10A510002020385C884201D120371EE03020385C92
:10A52000884201D1303718E04020385C884201D1A0
:10A53000403712E05020385C884201D150370CE09F
:10A540006020385C884201D1603706E07020385CBA
:10A55000884201D0002700E070370025002C2AD067
:10A56000002F28D0F5F7C6FD0546FFF767FA00284B
:10A570000AD01248124E3146FFF77CFA9120820031
:10A5800010483146FEF79CFB2846F5F7B7FDFEF76D
:10A59000BBFD3E1D37463F68B74209D03D46143DDE
:10A5A00010222846214600F028FC0028F3D100E0C4
:10A5B0000025FEF77DFF284601B0F0BDB1F0000890
:10A5C00023F60008FFEB00080146614802788A4242
:10A5D00000D17047027C8A4201D11030704720229E
:10A5E000825C8A4201D1203070473022825C8A42EC
:10A5F00001D1303070474022825C8A4201D1403024
:10A6000070475022825C8A4201D1503070476022EC
:10A61000825C8A4201D1603070477022825C8A423B
:10A6200001D00020704770307047C04610000020F5
:10A6300010B50446002803D0217C7F20084010BDBF
:10A64000044805A1094AFEF73BFB217C7F20084016
:10A6500010BDC04611F6000872745F6F626A6563D0
:10A66000745F6765745F747970650000270200008D
:10A67000F0B583B002920D460446354E30788842DC
:10A680002FD0307CA84201D110362AE02020305C47
:10A69000A84201D1203624E03020305CA84201D10C
:10A6A00030361EE04020305CA84201D1403618E030
:10A6B0005020305CA84201D1503612E06020305C5E
:10A6C000A84201D160360CE07020305CA84201D174
:10A6D000703606E09B2042001E481F49FEF7F0FA44
:10A6E00000260195FEF710FD351D7668AE4210D0AC
:10A6F0009B2047000E3702E03668AE4209D0304654
:10A700001438A042F8D115A013493A46FEF7D8FAFA
:10A71000F2E78020019E0643FEF7CAFE267410224F
:10A720002046029900F07CFB10480168002901D006
:10A7300020468847F5F7DEFC29686161224614321D
:10A740004A602A60A561F5F7D9FC03B0F0BDC046A8
:10A7500010000020FAF5000856F600086F626A2023
:10A76000213D206F626A6563740000005418002068
:10A7700010B50446002802D0207CC00910BD8520F9
:10A780008200034803A1FEF79BFA207CC00910BD9C
:10A7900011F6000872745F6F626A6563745F6973B3
:10A7A0005F73797374656D6F626A6563740000002E
:10A7B00070B50C460546084EB06C002805D1074818
:10A7C00007A18A22FEF77CFAB06C0368024829468A
:10A7D0002246984770BDC046E00300205DFA00089D
:10A7E00072745F70696E5F6D6F646500B0B504462A
:10A7F000074DA86C002805D1064807A19622FEF750
:10A800005FFAA86C8268024821469047B0BDC046F6
:10A81000E00300205DFA000872745F70696E5F7279
:10A820006561640070B50D460446084EB06C0028A2
:10A8300005D1074807A19022FEF742FAB06C4368A1
:10A84000EAB202482146984770BDC046E0030020A6
:10A850005DFA000872745F70696E5F777269746583
:10A8600000000000F0B581B0F5F744FC0446544FF9
:10A870007888002804D02046F5F740FC01B0F0BDF0
:10A88000F868FAF78DFA401EC1004C4A555829461F
:10A890001C397E68B142EED079603870BA68002AFF
:10A8A00001D030469047083524360B480078002800
:10A8B00008D030462946F5F724FC2046F5F71EFC63
:10A8C00001B0F0BD30462946F5F71BFC2046F5F7F0
:10A8D00015FC01B0F0BDC046F0010020F0B581B01C
:10A8E000044605463C35002805D1FF2218320F48A2
:10A8F0000FA1FEF7E5F9F5F7FDFB6978C9002F4ACE
:10A9000051184A68226223461C331360226C2C4E75
:10A91000F7681743F7602A78F0261640721C2A70F1
:10A920004B60E161F5F7EAFB01B0F0BD65F60008A8
:10A9300072745F7363686564756C655F696E736577
:10A9400072745F74687265616400000010B504463B
:10A95000002805D1FF224632104811A1FEF7B0F9B8
:10A96000F5F7C8FBE169226A4A60226A1160214654
:10A970001C31E16121623D21615CC9000F4A53181D
:10A980005158994202D0F5F7B9FB10BD216C0C4A21
:10A99000D3688B43D360F5F7B1FB10BD65F60008B3
:10A9A00072745F7363686564756C655F72656D6F03
:10A9B00076655F7468726561640000006C18002041
:10A9C00044020020F0B581B016460D460090F5F720
:10A9D00091FB0446FF270E37FFF730F8002808D018
:10A9E000BB481049FFF746F8B8480E493A46FEF70B
:10A9F00067F92046F5F782FB280C04D07A1C1E4824
:10AA00000849FEF75DF902200099FFF773FC002862
:10AA100005D08584467401461C31C161016201B0D4
:10AA2000F0BDC04639F20008F0B581B01C461646AC
:10AA30000F460546002814D0300C04D00E480D49AE
:10AA4000D322FEF73DF9022128463A46FFF710FED1
:10AA5000AE8428461C30E86128626C74002001B086
:10AA6000F0BD95480349D222FEF72AF9300CE5D112
:10AA7000E9E7C046B8F300088EF10008B0B5044617
:10AA800000281CD02046FFF7D3FD022822D1214800
:10AA90000168002901D020468847F5F72BFB0546C1
:10AAA000E06921461C31884220D01C3800F0B8FDF6
:10AAB0002846F5F723FBFFF7D5FE0020B0BDFF22A7
:10AAC000B8327D481249FEF7FBF82046FFF7B0FD8B
:10AAD0000228DCD0FF20B830421C79480C49FEF730
:10AAE000EFF80C4801680029D5D1D6E7A08C0A49B7
:10AAF000884205D12846F5F701FB0220C043B0BDCE
:10AB0000401CA0842846F5F7F9FA0020B0BDC046E5
:10AB10000CF200085C180020FFFF0000F0B583B0C5
:10AB20000D4604460291FF276E3700281DD02046AF
:10AB3000FFF77EFD022823D162480168002901D079
:10AB400020468847F5F7D6FAA18C002923D0491E64
:10AB5000A184F5F7D3FA5F4801680025002901D0E8
:10AB600020468847284603B0F0BD3A46213A52486D
:10AB70005249FEF7A5F82046FFF75AFD0228DBD020
:10AB80003A46203A4E484D49FEF79AF84D4801683A
:10AB90000029D5D1D6E7002D5FD00190F5F7AAFAAC
:10ABA000009000F085FD002809D14748434E31460A
:10ABB000FEF760FFE44831463A46FEF781F8F5F7C4
:10ABC00099FA0646FEF73AFF002808D0DC483B49D0
:10ABD000FEF750FFDC4839493A46FEF771F8304637
:10ABE000F5F78CFA0098F5F789FA00F061FD074651
:10ABF0000020B863667C384600F0F4FD20461C3027
:10AC0000002E31D0012E36D100953A463D32014614
:10AC10000968814245D02123CE5C1578B54214D312
:10AC2000096881423DD0CD5C1678AE420DD30968EB
:10AC3000814236D0CD5C1678AE4206D30968814297
:10AC40002FD0CB5C15789D42E2D248683A461C3240
:10AC50000260F96138624A602AE0F5F74FFA012094
:10AC6000C543284603B0F0BD216A3A461C320A604B
:10AC7000F86139622262012D09DB3D46543500211D
:10AC800002AA284600F0FEFE284601F013F80198BB
:10AC9000F5F734FAFFF7E6FDBD6B002D00D061E754
:10ACA00059E7216A3A461C320A60F8613962226229
:10ACB000009D012DE1DAEAE73DF10008ADF1000861
:10ACC000C7F1000864180020EEF00008FFEB000850
:10ACD000B1F000086018002010B50446FEF7AEFE83
:10ACE000002802D00448046010BD00F0E1FC0028F8
:10ACF000F8D0846310BDC046D803002080B582B070
:10AD000009A0FEF7B7FE0BA0FEF7B4FE12A000905C
:10AD100014A0032101220523FEF7ACFE19A0FEF7C3
:10AD2000A9FE02B080BDC0460A205C207C202F0A0C
:10AD3000000000002D205254202D202020202054DF
:10AD40006872656164204F7065726174696E672016
:10AD500053797374656D0A00536570203139203260
:10AD600030323400202F207C205C20202020202521
:10AD7000642E25642E2564206275696C6420257319
:10AD80000A0000002032303036202D2032303230A0
:10AD900020436F70797269676874206279207274D9
:10ADA0002D746872656164207465616D0A0000002D
:10ADB00081B080B581B0039303AB009301F04CF8F0
:10ADC00001B080BC02BC01B0084701460A78002AE5
:10ADD0000ED04A78002A0AD08A78002A0AD00A1DA2
:10ADE000C97800291146F1D1511E081A7047491C33
:10ADF000081A7047891C081A704710B5002A0DD030
:10AE00000B780478002C06D09C4204D1521E401CC2
:10AE1000491C002AF4D1E01A40B210BD002010BD38
:10AE2000F0B583B00290002A26D050420190002550
:10AE3000029B4C5D02984455002C20D00198471984
:10AE40007C1C19D24C190298461960787070002841
:10AE500019D0B81C10D0A078B070002818D0F81CF9
:10AE60000AD0E078F070002817D01B1D2D1D019826
:10AE70004019121F0028DCD1029803B0F0BD581C05
:10AE8000511E0ED1F8E7981C521E511E09D1F3E74E
:10AE9000D81C921E511E04D1EEE7301DD21E511E49
:10AEA000EAD0F5F702FA029803B0F0BDF0B581B030
:10AEB0000C4607460320C54300912C40F5F71AF9CC
:10AEC0000646FEF7BBFD002808D01D481D49FEF7C9
:10AED000D1FD1D48D2221B49FDF7F2FE3046F5F7A1
:10AEE0000DF9192C24D3F81C284021461839814229
:10AEF0001ED3211A0A46183A144DAA60F5225201AF
:10AF00000C3900230260416083600C3C6160E860A2
:10AF10002C610F482060A8680C30A06028462030C3
:10AF20000CA10122FFF780FDE868686101B0F0BD67
:10AF30000AA03946009AFEF79DFD01B0F0BDC0465B
:10AF4000B1F00008E6F50008FFEB0008FC01002066
:10AF5000A01E010068656170000000006D656D2035
:10AF6000696E69742C206572726F72206265676900
:10AF70006E206164647265737320307825782C20AC
:10AF8000616E6420656E6420616464726573732011
:10AF9000307825780A000000F0B583B05C490020C5
:10AFA000029048805B4D2C460834284610300090B3
:10AFB0002E461836284620302F462837294630316D
:10AFC0002B4638332A464032019228626862AF62CB
:10AFD000EF6229636963AB63EB632F4648372D60EB
:10AFE0006D60AC60EC60009828616861AE61EE61F4
:10AFF0002B46803380202B502A46883288202A50C6
:10B000002846503029465831019C2C646C64AF644A
:10B01000EF6428656865A965E965284660302946BA
:10B0200068312C4670342E46783628666866A966E4
:10B03000E9662C676C67AE67EE675B605260284616
:10B0400090304060902168502946983101919820B5
:10B0500029502946A0310091A02029502A46A83223
:10B06000A8202A502E46B036B0202E502F46B83792
:10B07000B8202F502846C030C02168502946C8311A
:10B08000C823E9502B46D033D0242B51019C646057
:10B09000009C6460526076607F60406049605B60E5
:10B0A0002846D8304060D82168502846E0304060BB
:10B0B000E02168502846E8304060E8216850284682
:10B0C000F0304060F02168502846F8304060F821A8
:10B0D00068500F4A10461030029B53601F211170B8
:10B0E000D3601061506103B0F0BDC04610B5084C8C
:10B0F000E068F9F755FEC0000649401808380068B6
:10B1000001461C3961600830F5F733F810BDC046C0
:10B11000440200206C180020024801460C31C16036
:10B12000016170475C02002070470000F0B581B0FB
:10B1300015460E460446002820D02046FFF778FA30
:10B14000012825D1002E2BD0012E2FD0022E2AD15E
:10B1500027463C37F4F7CEFF064638780F210140EA
:10B1600001292ED12046FFF7F1FB287878700121C4
:10B17000814021642046FFF7B1FB27E09C48194934
:10B18000194AFDF79DFD2046FFF752FA0128D9D054
:10B190001548421C98481349FDF792FD002ED3D163
:10B1A000204600F0C7FA002001B0F0BD2046FFF7AE
:10B1B000DFFA012810D1204600F0BAF8002001B0D3
:10B1C000F0BD287878700121814021643046F4F781
:10B1D00095FF002001B0F0BD204600F033F80020BC
:10B1E00001B0F0BD14F7000877020000F0B585B09B
:10B1F0001F4604920D4601460120FFF77BF800240C
:10B20000002811D006463846FEF794FC00280ED0E0
:10B2100003460B980A9900970191029030462946FF
:10B22000049AF9F7EDFE3446204605B0F0BD3046ED
:10B23000FFF7DCF8204605B0F0BD80B500F03CFA21
:10B24000002080BD70B50446CF204500002C1DD0E5
:10B250002046FFF7EDF9012804D06A1C2448234951
:10B26000FDF72EFD26463C362046FFF781FA0028E2
:10B2700004D0AA1C1FA01D49FDF722FD31780F2024
:10B28000084011D004280CD1002070BD1648174981
:10B290002A46FDF715FD2046FFF7CAF90128DCD143
:10B2A000E0E72046FFF752FBF4F724FF0546F16C78
:10B2B000002901D0204688472846F4F71FFF204682
:10B2C000543000F055FC25461C35F4F713FF964921
:10B2D0000A685560042333700D60E2612162F4F75F
:10B2E0000DFF002070BDC04665F60008DCF60008C2
:10B2F00077F6000872745F6F626A6563745F6973E2
:10B300005F73797374656D6F626A65637428287200
:10B31000745F6F626A6563745F74297468726561D3
:10B320006429203D3D2052545F46414C5345000066
:10B3300070B50446FF253A35002815D02046FFF7A2
:10B3400077F9012804D06A1C2B482A49FDF7B8FC7C
:10B3500026463C362046FFF70BFA00280FD03178FE
:10B360000F20084014D11AE0214822492A46FDF74F
:10B37000A7FC2046FFF75CF90128E4D1E8E7AA1C06
:10B380001EA01C49FDF79CFC31780F20084006D018
:10B39000042801D1002070BD2046FFF7D7FAF4F74A
:10B3A000A9FE0546F16C002901D0204688472846B1
:10B3B000F4F7A4FE2046543000F0DAFB042030708D
:10B3C0002046FFF7D5F9012804D12046FFF760F8A1
:10B3D000002070BD25461C35F4F78CFE52490A68E2
:10B3E00055600D60E2612162F4F788FE002070BDB7
:10B3F00065F60008EDF6000877F6000872745F6FD6
:10B40000626A6563745F69735F73797374656D6F86
:10B41000626A656374282872745F6F626A65637418
:10B420005F7429746872656164290000F0B581B0A9
:10B43000EB480568F4F75EFE04462F463C37F4F708
:10B4400059FE0646F96C002901D028468847304647
:10B45000F4F754FE2846FFF779FA0420387028469E
:10B46000543000F085FB2846FFF782F9012803D10C
:10B470002846FFF70DF807E02B4801682A461C32E2
:10B480004A600260E9612862FFF7ECF92046F4F7B0
:10B4900035FE01B0F0BDC0461F4E234D02E03846D8
:10B4A000F4F72CFE3068002800D080477068002830
:10B4B00000D08047B068002800D08047F06800289E
:10B4C00000D08047F4F716FE0446FEF7B7FA0028CE
:10B4D00009D01248124F3946FEF7CCFA9322114890
:10B4E0003946FDF7EDFB2046F4F708FEF4F702FEBF
:10B4F00007462C68AC42D2D003CC4160083C61685E
:10B500000860246064606069FDF7ECFF1C3C204625
:10B51000FEF76CFF3846E7E734170020B1F000086B
:10B52000D8F00008FFEB00085402002010B584B0EA
:10B53000202003901F200290084800900120000264
:10B540000190074C07A1094A0023204600F010F89B
:10B55000204600F0EFF804B010BDC046701900207E
:10B56000A41600207469646C6500000099B400089A
:10B57000F0B587B0069305920A4606460C9C002853
:10B5800006D11B481B491546E922FDF799FB2A46BF
:10B590000F9804900E9F0D9D002C10D00121304675
:10B5A000FFF766F8009501970498029030460599D8
:10B5B000069A2346F9F724FD002007B0F0BD0EA03F
:10B5C0000C491446EA22FDF77BFB01213046224656
:10B5D000FFF74EF80095019704980290002330463B
:10B5E0000599069AF9F70CFD002007B0F0BDC0469A
:10B5F00065F6000848F70008737461636B5F737445
:10B6000061727420213D2052545F4E554C4C000015
:10B6100080B500F0B7F900F04FF8002080BD0000C1
:10B6200070B50446002831D02046FFF701F8012804
:10B6300005D01D48421CBB481A49FDF741FB3C2080
:10B64000205C0F210140002502291DD1F4F752FD95
:10B650000646E069216A4160216A086020461C3084
:10B66000E06120622046543000F0B0FB3046F4F731
:10B6700045FD2046FFF732F90C480168002901D04A
:10B6800020468847284670BDE84370BD9448054968
:10B69000054AFDF715FB2046FEF7CAFF0128C8D171
:10B6A000CDE7C046CBF60008F70200006C19002079
:10B6B000B24800687047C046F0B581B00090F4F71A
:10B6C00019FD0546AD480468002C25D02046FEF73C
:10B6D000AFFF012806D0FF20FC30421C91481449DE
:10B6E000FDF7EEFA204600F07DF827465437002695
:10B6F0006A463846314600F0C5F9384600F0DAFAB5
:10B700002846F4F7FBFCFFF7ADF8A06B801C00D1D6
:10B71000A663002001B0F0BDFF22FC32704804494E
:10B72000FDF7CEFA2046FEF783FF0128D3D1D9E7F3
:10B7300026F7000870B50446FF250E3506463C3650
:10B74000002823D03078000704D06A1C16A01549C1
:10B75000FDF7B6FA2046FEF76BFF012804D0AA1CBD
:10B7600070481049FDF7ACFA02203070B078707064
:10B770000121814021642046FFF752FF7F48006885
:10B78000002801D0FFF76EF8002070BD044805497D
:10B790002A46FDF795FA30780007D6D1DAE7C04699
:10B7A00065F6000836F70008287468726561642D34
:10B7B0003E7374617420262052545F5448524541B0
:10B7C000445F535441545F4D41534B29203D3D202C
:10B7D00052545F5448524541445F494E4954000019
:10B7E00048020020F0B581B00446002832D020463F
:10B7F000FEF71EFF012805D01D48421C49481B4981
:10B80000FDF75EFA3C20205C0F2101400025012954
:10B810001CD127463C37F4F76DFC06462046FFF75F
:10B8200095F83878F0210140881C38702046543053
:10B8300000F0CCFA3046F4F761FC0E4801680029AC
:10B8400001D020468847284601B0F0BDED43284688
:10B8500001B0F0BD22480549054AFDF731FA2046FE
:10B86000FEF7E6FE0128C7D1CCE7C046B9F60008CE
:10B87000CD020000701A0020B0B50446174D002814
:10B8800004D1174817492A46FDF71AFA3C20205CD4
:10B890000F210140022904D06A1C13A01149FDF7B1
:10B8A0000FFA2046FEF7C4FE012804D0AA1C1D484A
:10B8B0000C49FDF705FAE069216A4160216A0860D8
:10B8C0000120C043A06320461C30E0612062204676
:10B8D000FFF704F8FEF7C6FFB0BDC0462303000023
:10B8E00065F6000857F70008287468726561642DD2
:10B8F0003E7374617420262052545F54485245416F
:10B90000445F535441545F4D41534B29203D3D20EA
:10B9100052545F5448524541445F53555350454E2D
:10B920004400000077F60008B0B5F4F7E3FB1349D4
:10B9300009683C228A5C0F231340012B1AD1CA6983
:10B940000B6A9A4216D00C463C340D461C355360A7
:10B950000B6A0D621A606278D200094B9A1853681C
:10B960001D60CA610B625560F4F7C8FBFEF77AFFF1
:10B970000020B0BDF4F7C2FB0020B0BD480200209B
:10B980006C180020C1170843704700000C4800687D
:10B990007047C04680B50A480168491C0160FFF73E
:10B9A00087FE016D491E016502D000F00BF880BDD5
:10B9B000C16C0165FFF7B8FF00F004F880BDC04618
:10B9C000781A0020F0B585B003A803900490FFF723
:10B9D000DDFF0646F4F78EFB0190FB48C5680C308E
:10B9E000029002E0F848C5680298854243D0686931
:10B9F000301A234988423ED82C461C3CF248016844
:10BA0000002901D02046884703CD4160083D696880
:10BA100008602D602F460B3F3878810702D4FE2145
:10BA20000840387003984560286003A86860039553
:10BA3000A968E8688847FFF7A9FF0646E248416819
:10BA4000002901D02046884703A803998142C9D024
:10BA500003CD4160083D696808602D606D603878ED
:10BA6000032101400329BDD1FE2108403870204642
:10BA700000F020F9B6E70198F4F740FB05B0F0BDFF
:10BA8000FEFFFF7F70B515460E46044600280CD019
:10BA90002046FEF7CDFD0A2812D1F4F72BFB042E29
:10BAA00019D9F4F72BFB002070BDFF22DA32E648EB
:10BAB0002249FDF705F92046FEF7BAFD0A28ECD029
:10BAC000FF20DA30421CE2481C49FDF7F9F8F4F790
:10BAD00011FB042EE5D8C0467E4436797600B74483
:10BAE0000211171F08002968E162F4F707FB002024
:10BAF00070BD617CC9071BD100212960F4F7FEFAF3
:10BB0000002070BDE16A2960F4F7F8FA002070BDEA
:10BB1000617CFD220A406274F4F7F0FA002070BDE7
:10BB2000617C02220A436274F4F7E8FA002070BDD7
:10BB300001212960F4F7E2FA002070BD9AF70008AD
:10BB400070B51C4615460E4601460A20FEF7D2FB8C
:10BB500000280CD004990022FE230B4043740146B8
:10BB60001C31C161016246628562C462026370BDBC
:10BB700010B5044600281FD02046FEF759FD0A28BC
:10BB800024D12046FEF7F4FD002829D0F4F7B2FABC
:10BB9000E169226A4A60226A1160617CFE220A40E1
:10BBA000627421461C31E1612162F4F7A7FA204654
:10BBB000FEF76EFC002010BD0C480D49DD22FDF79C
:10BBC0007FF82046FEF734FD0A28DAD009480849F4
:10BBD000DE22FDF775F82046FEF7CAFD0028D5D114
:10BBE00005A00349DF22FDF76BF8CFE769F70008EE
:10BBF0008AF70008B9F7000872745F6F626A6563BC
:10BC0000745F69735F73797374656D6F626A65637E
:10BC100074282674696D65722D3E706172656E744C
:10BC200029000000F0B583B0029315460E46074682
:10BC3000FE20099C044008980190002F12D00A2190
:10BC400038463246FEF714FD00207C7439461C311C
:10BC5000F96139627D620299B9620199F9623863CA
:10BC600003B0F0BD0E480FA1C922FDF729F8002747
:10BC70000A2138463246FEF7FBFC242005601120DD
:10BC80000470282002990160302007602C2001995F
:10BC9000016020201C210160096003B0F0BDC04696
:10BCA00069F7000872745F74696D65725F696E6927
:10BCB00074000000F0B581B00446FF26423600282B
:10BCC00047D02046FEF7B4FC0A2804D0721C324844
:10BCD0003049FCF7F5FFF4F70DFA0090E069216AAE
:10BCE0004160216A0860607CFE2101406174274642
:10BCF0001C37E761276229480168002901D02046E6
:10BD00008847E06A264DA84205D3103625A0214970
:10BD10003246FCF7D5FFFFF739FEE16A09182163C7
:10BD2000294806460C36026996420FD03368586996
:10BD3000401A01D0A84217D3934207D01E687069F9
:10BD4000401AF1D0A8423046EED20FE010681346F8
:10BD50000CE00F480F493246FCF7B2FF2046FEF7D1
:10BD600067FC0A28B2D1B6E718463346E06147605F
:10BD70001F60236214498868401C8860607C012130
:10BD8000014361740098F4F7B9F9002001B0F0BDE7
:10BD900069F70008F5F70008B9F7000860180020F7
:10BDA000FFFFFF7F74696D65722D3E696E69745F78
:10BDB0007469636B203C2052545F5449434B5F4D80
:10BDC0004158202F203200005C020020B0B504460C
:10BDD00000280AD02046FEF72BFC0A2810D10025A7
:10BDE000607CC00717D1E843B0BDDB204200164895
:10BDF0001649FCF765FF2046FEF71AFC0A28EED02C
:10BE0000DB204000421C12481049FCF759FF002576
:10BE1000607CC007E7D00F480168002901D02046A8
:10BE20008847F4F767F9E169226A4A60226A11607B
:10BE3000617CFE220A40627421461C31E16121626C
:10BE4000F4F75CF92846B0BD69F70008ABF70008C5
:10BE5000B9F700085C180020F0B58FB01F461646F1
:10BE6000044600220992D54306910029089501D481
:10BE700006996518E143049105940C9501E0641C52
:10BE8000761C3178252906D0002900D17CE3AC420C
:10BE9000F5D22170F3E70B94761C099C33781A468F
:10BEA000203A102A17D810217A4412795200974468
:10BEB0000C12120E12121212121212101209121277
:10BEC000080001210C43761CE8E70821FAE720214D
:10BED000F8E70421F6E718463038092817D800217A
:10BEE0000A225143C9183039737818463038092866
:10BEF00019D84A43D1183039B21CB37818463038B3
:10BF00000A281646ECD316462E2B0FD009E02A2B12
:10BF100027D102CF761C002900D5B1E033782E2B33
:10BF200004D0089A2EE0761C2E2BFAD1737818468E
:10BF3000303809281AD8751C00220A267243D218F4
:10BF4000303A6B7818463038092815D85643F2181D
:10BF5000303AAE1CAB78184630380A283546ECD358
:10BF60000EE0089933782E2BE0D0DAE72A2B05D1A2
:10BF7000B37804CFB61C03E06E1C01E0761C089A6F
:10BF8000D0178243042018436C280D9707D1777887
:10BF9000761C0E933D46253D532D08D982E00020A6
:10BFA0000E901F463D46253D532D00D97AE00A23C9
:10BFB0006D00C0467D44AD886D00AF4469007300DC
:10BFC00073007300730073007300730073007300D9
:10BFD00073007300730073007300730073007300C9
:10BFE00073007300730073007300730073007300B9
:10BFF00073007300730073007300730073007300A9
:10C000007300730073007300730073007300730098
:10C010007300730073007300730073007300730088
:10C020007300850073007300730073007300730066
:10C0300073007300730073009E005300730073005D
:10C040007300730053007300730073007300730078
:10C05000BD00C30073007300DB0073008800730031
:10C0600073008700022004430E9868280A9332D197
:10C070000D980388A00700D51BB20C9D0D9F2EE0E4
:10C0800010200443494233782E2B00D14EE748E775
:10C090000C9D0B9CAC4201D225202070641C0D9F8E
:10C0A000761CEEE60C9D0B9CAC4202D22520207043
:10C0B0003778611C002F00D18CE0A94200D20F70AC
:10C0C000A41C0D9F761CDCE64020044310230E9830
:10C0D00068280A93CCD06C280D9F3B680C9DE0B279
:10C0E0000091019202900B9829461A460A9BFCF790
:10C0F00075FB04463F1D761CC3E6E00600D514E13F
:10C100004C1E022900DA0FE1032525408B1E002D6D
:10C1100000D166E10C980B9C844201D22020207053
:10C12000621C012D0D9F00D069E11C460C9D002171
:10C13000032B00D2BEE1C2E108230E9868280A93BF
:10C14000C9D195E70D9880C80D9001924A1C00D185
:10C1500008210C9D0091504250410443E0B20290EE
:10C1600010230B9829463A46FCF738FB04460D9FEE
:10C17000761C86E60D9808C8002B00D1F9A30E9313
:10C1800000290D902BD0089B4B43C81E0A90002716
:10C190000E980793C05D002822D0DD19681C17D2C5
:10C1A0000E98C3195878002800D126E1A81C0FD09A
:10C1B0009878002800D130E10A98B84208D0D878A1
:10C1C000002800D169E13F1D079BD8190E98E1D1E5
:10C1D0000F4605E0761E0C460D9F761C51E60027A3
:10C1E0009742134622DC3B46002A21DDE0060A93F3
:10C1F00022D44D1E994200DCCCE0C81A0327074028
:10C20000D8430C18002F00D1F1E00C9B0B9A9A42F6
:10C2100001D220201070521C012F00D0FFE08D1E93
:10C220000D9F0A9B032C00D277E182E1002ADDDC1E
:10C230003B46E0060A93DCD50B9A0D9F0E98012B26
:10C2400000DA6FE10324042B18D20C9D1C404FD060
:10C25000AA4201D203781370531C012C09D0AB42BF
:10C2600003D2079444781C70079C931C022C00D0C6
:10C27000AEE01A460A9B99423DDC57E10794A3437E
:10C280000B93002403E0241D0B9BA34228D0151917
:10C290000C9FBD4210D2035D2B706B1CBB420ED3B2
:10C2A000AB1CBB4213D20E980019807818700E9800
:10C2B000EB1CBB42E7D20DE06B1CBB42F0D20E98E8
:10C2C0000019407818700E98AB1CBB42EBD3EB1CE6
:10C2D000BB42D8D20E980019C07818700E98D2E7D9
:10C2E000121900190C9D0D9F0A9B079C1C40AFD191
:10C2F000994200DC1AE1C81A03240440D843081804
:10C30000002C4FD02B46AA4203D2054620201070A5
:10C310002846551C012C49D1491E2C461D460A9B16
:10C32000032800D39BE0E6E621460BAFB0CFAC423A
:10C3300001D2386820703F1D022928DB221D06E04B
:10C34000411C121D0223DB43401E98423DD2D01EE9
:10C35000A84201D220230370941E032900D2CAE60A
:10C36000AC4201D220202070091F541E0320C34379
:10C37000994200D9BFE6AC4201D220202070481E6D
:10C3800098421FD8AA42DBD220211170D8E7641C42
:10C39000761C76E50B9A29460D9F0E98012B00DB43
:10C3A00050E7BFE01446032859D2A4E60E909D4200
:10C3B00001D220202870901C022C3ED1891E0446F8
:10C3C0001D4642E01446761C5BE5D41E761C58E5FB
:10C3D000AB4201D280781870D21C0A9B99428ADC49
:10C3E000A4E00BAFA4CF0021032B63D367E00B9A2B
:10C3F0000D9F032C00D290E09BE07F1CF0E60C9890
:10C40000824201D220201070A21C022D47D1CC1EE6
:10C410000C9D0021032B4DD351E0BF1CE0E69A4256
:10C4200001D2202010700B98821C022F0D9F6AD120
:10C43000CD1E0A9B032C70D37BE01D46984202D28E
:10C44000044620202070C91ED41C0A9B0E98032885
:10C4500005D250E6091F241D8B4200DB4BE6AC429F
:10C460000DD220202070621CAA420BD3A21CAA422B
:10C470000DD220201070E21CAA42EBD20AE0621C0E
:10C48000AA42F3D220201070A21CAA42F1D3E21CCF
:10C49000AA42DFD220201070DCE7FF1CA0E60C9D32
:10C4A000AA4201D2202010700C1F0B98C21C002140
:10C4B000032B04D21446AC4200D23AE73BE7201DDE
:10C4C00003E0001F121D0428F4DDAA420DD2202330
:10C4D0001370531CAB420BD3931CAB420DD22024E0
:10C4E0001C70D31CAB42ECD20AE0531CAB42F3D21B
:10C4F00020241C70931CAB42F1D3D31CAB42E0D27E
:10C5000020241C70DDE79A4201D2202010700D1FFC
:10C510000B98C21C0A9B032C0BD2591E0E98012BA0
:10C5200000DB8FE60C9D994200DDE4E61446761CA4
:10C53000A7E4681C04E0001F121D0A9B8342ECDA8A
:10C540000C9CA24212D220211170511CA14210D386
:10C55000911CA14212D220230B70D11CA142EAD21D
:10C560000FE0C046284E554C4C290000511CA142FA
:10C57000EED220230B70911CA142ECD3D11CA1421E
:10C58000D9D220230B70D6E706980028049900D44E
:10C5900001460029059905D0AC42204600D3681E0B
:10C5A000099A0270601A0FB0F0BD00207047002099
:10C5B00070470020704700207047000010B582B01F
:10C5C000F3F798FDFDF766F8FEF798FBFEF7A4FD7C
:10C5D000FEF7E2FC14200A21009101900120830261
:10C5E0000C480D490022FEF701FE0446002804D144
:10C5F0000A480B49C522FCF763FB2046FFF79AF86F
:10C60000FEF792FDFEF792FFFEF770FD002002B0EC
:10C6100010BDC046A8E70008ED8100088EF00008B4
:10C620009DF000080448016804220A430260016882
:10C6300001220A430260704710E000E0B0B50268D2
:10C6400014215143154A8C580A4B23404468C5684D
:10C65000254304692C434569254384692C431C43C5
:10C660008C508B581F242404A34380680004184373
:10C670008850B0BD0FE7FFFF10B5016814224A4390
:10C6800006495318C4685C6044689C608068D86040
:10C69000505801230343535010BDC04608000240C8
:10C6A000F0B581B000910546714800680124270467
:10C6B000704E3168C90308D430686F493160C006D4
:10C6C000400F204620D001B0F0BD7D21C900F4F715
:10C6D00005F8052141430220411A04200229F2D025
:10C6E00032683A42E8D00129EDD032683A42E3D0CC
:10C6F0000029E8D032683A42DED0091D0329E2D091
:10C7000030683842E9D1D7E7706806239843284358
:10C710007060022D09D17F2000027168814300986A
:10C72000000208437060052400E03224706808218C
:10C73000014371604E480068316839420BD131685D
:10C740004D4830601C200840411E88417168994363
:10C75000716001B0F0BD7D21C9001D46F3F7BEFF39
:10C760002B4644430220011B04200229EED03268EC
:10C770003A42E4D00129E9D032683A42DFD00029B8
:10C78000E4D032683A42DAD0091D0329DED030689D
:10C790003842E9D1D3E7C046F0B581B00B46054633
:10C7A0003348006801242704324E3168C90308D495
:10C7B000306831493160C006400F204624D001B0B6
:10C7C000F0BD7D21C90000942C461D46F3F786FF7D
:10C7D0002B462546009C0221091A04200229EED08E
:10C7E00032683A42E4D00129E9D032683A42DFD0D7
:10C7F0000029E4D032683A42DAD0091D0329DED09C
:10C8000030683842E9D1D3E7706801242043706072
:10C810002B6017480068316839420BD131681648DF
:10C8200030601C200840411E88417168A14371603E
:10C8300001B0F0BD7D21C900F3F750FF0221091AB4
:10C8400004200229F1D032683A42E7D00129ECD025
:10C8500032683A42E2D00029E7D032683A42DDD06D
:10C86000091D0329E1D030683842E9D1D6E7C04636
:10C870000C000020102002401C000001F0B584B024
:10C88000039001910E68002E3AD0002300960EE02E
:10C890006D436D432C460F226243974366433E43EC
:10C8A00003984650009E5B1C3146D94028D0012594
:10C8B0009D403540F7D02C466C43019E7068029035
:10C8C000214641430327674303980268BA430A435A
:10C8D0000260B1686143C268BA430A43C260029809
:10C8E0000228009EDFD12D0A01D0242100E0202162
:10C8F000019A166903984758002DC9D16443CAE7C5
:10C90000019A5168491E012906D8D16871430398DC
:10C910004268B2430A43426004B0F0BD70B50E46AF
:10C92000044600680125A84320602803216881434C
:10C93000F068084320600320410222688A4371693D
:10C9400011432160010362688A43316911436160C8
:10C95000E16A0F22914332680A43E2620002A16851
:10C960008143B0690843A060B168204600F030F808
:10C9700000280FD120680C21884371680143216091
:10C98000216822680120024322600A0704D400259E
:10C9900049070FD4284670BD4205E3691342F6D11A
:10C9A000E3691342F3D1E3691342F0D1E36913421F
:10C9B000F3D0ECE78005E1690142EBD1E169014286
:10C9C000E8D1E1690142E5D1E1690142F3D0E1E753
:10C9D00070B50D4604460026214884420ED02148F9
:10C9E000844230461ED1204800680005810F1F4850
:10C9F0007944097949008F440D1015131A480068CD
:10CA00008005810F1948C0467944097949008F444F
:10CA10000104090700F03EF804E000F0BFF801E06F
:10CA20000120C003E16A0907C90E11A2515AF3F7A8
:10CA300055FE010E00026A08801871412A463346ED
:10CA4000F3F7C4FB10494118104A914206D8E16837
:10CA50000F4A0A400243E260002070BD012070BD11
:10CA600000840040008000403C1002400024F4009C
:10CA7000010002000400060008000A000C0010007B
:10CA8000200040008000000100FDFFFFFFFC0F00C0
:10CA90000000F0FFB0B55A4D2C1F20688006400FF3
:10CAA000411E032921D857487944097949008F4408
:10CAB000220116192968C90700D1534829680906B7
:10CAC000C90E00D12021484329684905490F00D1EA
:10CAD0000821F3F703FE29684903890F0AE07D2046
:10CAE000000208E00120C00305E00C3D2868C004F6
:10CAF000810F4548C840216807221203236813406C
:10CB00001A0B032A01D3D21E00E000224905490F67
:10CB1000C840D040B0BDC046B0B5394D2C1F2068CC
:10CB20008006400F411E032921D8364879440979EF
:10CB300049008F44220116192968C90700D13248DB
:10CB400029680906C90E00D12021484329684905F2
:10CB5000490F00D10821F3F7C1FD29684903890F66
:10CB60000AE07D20000208E00120C00305E00C3D42
:10CB70002868C004810F2448C84021680722120495
:10CB8000236813401A0C032A01D3D21E00E00022AE
:10CB90004905490FC840D040B0BDC04610B5184C3B
:10CBA000201F00688006400F411E032921D8154828
:10CBB0007944097949008F44220116192168C9076F
:10CBC00000D1114821680906C90E00D1202148432F
:10CBD00021684905490F00D10821F3F77FFD21683D
:10CBE0004903890F0AE07D20000210BD0120C00327
:10CBF00010BD0C3C2068C004810F0348C84010BD24
:10CC00000C10024000127A000024F400F0B581B04C
:10CC100004466B4ECA20B0615320B061694F3D6835
:10CC20003068400623D43068802101433160306889
:10CC300040061CD47D20C1002846F3F74FFD481B59
:10CC4000811C0420022929D0326852060FD4012900
:10CC500024D0326852060AD400291FD03268520606
:10CC600005D4091D032919D030684006E9D5A078FC
:10CC7000217849030818617809020143E07800042B
:10CC800008433146083908603C6830688021884391
:10CC9000306030680025400604D428460021B16188
:10CCA00001B0F0BD7D20C1002046F3F717FD081B41
:10CCB000811C04200229F1D0326852060FD50129C7
:10CCC000ECD0326852060AD50029E7D03268520605
:10CCD00005D5091D0329E1D030684006E9D428466E
:10CCE0000021B16101B0F0BDF0B581B00446344E11
:10CCF000CA20B0615320B061324F3D6830684006B1
:10CD000023D43068802101433160306840061CD450
:10CD10007D20C1002846F3F7E1FC481B811C04205C
:10CD2000022926D0326852060FD4012921D0326858
:10CD300052060AD400291CD03268520605D4091DB7
:10CD4000032916D030684006E9D5207800046178C0
:10CD500009020818A178401831460C3908603C686F
:10CD6000306880218843306030680025400604D454
:10CD700028460021B16101B0F0BD7D20C1002046F0
:10CD8000F3F7ACFC081B811C04200229F1D03268A7
:10CD900052060FD50129ECD0326852060AD5002977
:10CDA000E7D03268520605D5091D0329E1D0306865
:10CDB0004006E9D428460021B16101B0F0BDC0466B
:10CDC0000C2800400C00002070B50546012420030B
:10CDD0002A688243C86810432860032002036B68F6
:10CDE00093430A691A436A60E2032B6893434A68D3
:10CDF0001A432A602A680C239A430B6813432B605A
:10CE000042022B6893434A691A432A600002AA68C7
:10CE1000824388691043A8608E68114885420BD010
:10CE20001048854205D01048854202D00F488542FF
:10CE300014D1FFF72FFE01E0FFF76EFE2968090409
:10CE4000C90F8840710840183146F3F747FC014686
:10CE50001039074A914201D8E8600024204670BD8D
:10CE60000038014000440040004C004000480040B1
:10CE7000EFFF0000B0B53048026802210A430123E9
:10CE80009A430260032002052C48046894431A0563
:10CE9000A21802601A040468144304609C04056824
:10CEA000254208D10568254205D10568254202D1F1
:10CEB00005682542F3D0C468214D2540FF24223463
:10CEC0002C19C4601C060568254305605B060468D0
:10CED0001C4208D104681C4205D104681C4202D1DE
:10CEE00004681C42F3D0C3681343C36082680A43DA
:10CEF00005218A438260826838210A40102A0BD0BB
:10CF000082680A40102A07D082680A40102A03D09B
:10CF100082680A40102AEED107210A0283689343EF
:10CF200083600A03836893438360090482688A43A9
:10CF30008260F7F72BFAB0BD0020024000100240DB
:10CF400006F8F9FFF0B581B016460D4604462C4FA1
:10CF5000002832D0002D37D02E4F386800283CD022
:10CF6000E069002842D0A169002901D02046884705
:10CF7000072026616061102220462946FDF750FFF8
:10CF80003437F3F7B7F83A68002A39460BD01368FC
:10CF9000002B114607D01A68002A194603D01768DB
:10CFA000002F1146EFD122462C320A600025E5629F
:10CFB000F3F7A4F8284601B0F0BD124812493A46EA
:10CFC000FBF77EFE002DC7D17A1C10A00E49FBF79F
:10CFD00077FE104F38680028C2D10948821C0E48DD
:10CFE0000949FBF76DFEE0690028BCD10448C21C6A
:10CFF0000AA00549FBF764FEA1690029B6D1B7E78D
:10D0000013050000A9FA0008E5FA00086E616D65D5
:10D01000000000009C280020B5FA00086261636BE4
:10D02000656E642D3E6F75747075740080B500F088
:10D030003FFD04480449C16104A10122FFF782FFBA
:10D04000002080BD5C11002055D00008636F6E7316
:10D050006F6C650070B5049CFBF794FE00280CD043
:10D060000546059B068C4020304328840021284635
:10D070002246FCF703F82E8470BD2046FCF752FBD5
:10D0800070BD0000F0B58DB006930E460746012036
:10D0900007900502002F0A9234D0082E3AD2129C33
:10D0A000002A40D008960594002C45D0F04C00266C
:10D0B0002660F048FDF789FE6060A621089AD140FD
:10D0C0000798014003912468099700D083E09500F8
:10D0D0003846E94F002804D1E848E9499222FBF795
:10D0E000EFFD7819E7497F2C0B46099F31D83A1993
:10D0F0001B2313707F2C25D00223E24DEB187F2CCD
:10D1000025D126E0E0A0E2492A46FBF7D9FD0A9A9C
:10D11000082EC4D36A1CDF48DD49FBF7D1FD0A9A0B
:10D12000129C002ABED1AA1CDB48D949FBF7C8FDD6
:10D1300008960594002CB9D1EA1CD848D449FBF7CD
:10D14000BFFDB3E70123CF4DEB187F2C01D05B244B
:10D150005470591AFB4B1A688D181D600468002F13
:10D1600004D1FA48FA499222FBF7AAFD7F2D204606
:10D170002CD82278002A204628D00C957919002036
:10D180000A5422185578002D1AD00C9B1B187E2BA0
:10D1900016D80F187D709578002D13D07D2B11D8DF
:10D1A000BD70D578002D0FD07C2B0DD8FD70127975
:10D1B000001D002A099F01D07C2BE1D3201805E037
:10D1C000501C03E0901C00E0D01C099F001BDD4AAE
:10D1D000116844181460139804905B20019038552E
:10D1E00038190C90401C0290FEF7D0FB07460A2429
:10D1F00038462146F3F772FA0C998D190B94444383
:10D20000391B3024214369700A2F10D30A21F3F708
:10D2100065FA2143A97064213846F3F75FFAB61C1A
:10D22000642F0746E3D20094741E324602E0009455
:10D23000721C3446029800218154002C26D00C9890
:10D24000821E23460C9846187578C7187878707037
:10D250007D70581E4D1C854218D2B078D518AF7815
:10D26000B770A870981E8F1C87420FD2F0786F7825
:10D27000F7706870D81ECD1C854207D23079D55C16
:10D280003571D0541B1F091D9942DBD3AD4821468F
:10D29000044600680918099FC91900220C92CA7037
:10D2A0005D228A703818FDF790FD21680818A94999
:10D2B0007F280A4603D820223A54A64A521C511A03
:10D2C0000E18A0480660089A9000A3A10C582620CA
:10D2D000D040C00704D0A8489D499322FBF7F0FC3A
:10D2E0007F2E22D82278002A1FD0B91900200A5494
:10D2F00022185778002F28D033187E2B25D80D18E8
:10D300006F709778002F22D07D2B20D8AF70D77800
:10D31000002F1ED07C2B1CD8EF701279001D002A24
:10D3200001D07C2BE3D3201814E0864804683E1912
:10D330000A9B002B1AD1904885499322FBF7C0FC29
:10D340000A9B7F2C184614D946E0501C02E0901C22
:10D3500000E0D01C099F0A9B001B7A4A1168441800
:10D3600014603E19002F28D0002BE4D07F2C1846E3
:10D3700032D81978002918462ED00C983154191833
:10D380004D78002D22D022187E2A1FD833185D70C8
:10D390008D78002D1CD07D2A1AD89D70CD78002D57
:10D3A00018D07C2A16D8DD700979001D00290A9B47
:10D3B00001D07C2AE2D318180EE064486449922216
:10D3C000FBF77EFC0A9B002BD0D1B4E7481C03E09E
:10D3D000881C00E0C81C0A9BC01A5A4A11684418ED
:10D3E0001460002F04D065487F2C014609D913E052
:10D3F000564857499222FBF763FC60487F2C014650
:10D400000AD839193A220A705C4A7E2C03D82023A4
:10D410004B70911C00E0511C081A4A4D29684118B4
:10D42000296078188024611A059A049BFEF714FD80
:10D4300029680E18812E00D32646002800DA2646D9
:10D4400040480660406881197C398122D24391426C
:10D4500003D87B210E1A3B480660069800283A4CF8
:10D4600039D0002F1CD07F2E214621D92EE0C04676
:10D470002803002078E90008C0DE00081AFB000835
:10D480002BFB0008A2FA00086C6F675F62756600EC
:10D49000D7FA00088DFA0008B1FA000813FB00085B
:10D4A0002A482B499222FBF70BFC7F2E21460DD8F0
:10D4B000B8190D2101707F2E01D002210791224958
:10D4C000079A89187F2E01D00B9A4270081B1D4ABB
:10D4D000116846181660039800282DD1002F04D03B
:10D4E00027487F2E014609D921E018481849922281
:10D4F000FBF7E6FB22487F2E014618D8BA191B21FC
:10D5000011707F21891B032900D303214C1C1C4B64
:10D510001919012C0BD0019C54709C1CA14206D0FF
:10D52000009C9470DB1C994201D06D23D370081AC3
:10D53000044A1168461816600C98B85530460DB06C
:10D54000F0BDC0462803002078E900081AFB000857
:10D550002BFB000881EE00087EFA000800000000A6
:10D560000000000084FA00088AFA000800000000A9
:10D5700087FA000881FA0008A5FA000874FA000882
:10D58000C2FA0008F0B58FB01E4609920F46044655
:10D59000FDF71BFC0390E348006800280AD0FCF765
:10D5A0004DFA00280FD0DF480546C03540680028F6
:10D5B0000FD118E0DC48DDA1E04AFBF781FBFCF766
:10D5C0003DFA0028EFD1D748054638354068002895
:10D5D00009D0FCF733FA002800D124E2F2F78AFDE3
:10D5E000BC21D04A50500694002E00D12AE2A81E39
:10D5F0000190039808300390002005900446089697
:10D600000A970B950FE0CE49601A441900210B9D33
:10D6100029550094072001222B46F8F729F907988D
:10D62000B04200D30EE20C90002809D003982C469B
:10D6300005994518202120462A46FCF7FBFBE1E02E
:10D640005B202855049428190790401C059000265B
:10D65000FEF79CF905460A2728463946F3F73EF8B7
:10D6600007998C194743E91B3027394361700A2D0C
:10D670000FD30A21F3F732F83943A1706421284609
:10D68000F3F72CF8B61C642D0546E4D2711E304623
:10D6900001E0701C31460022059B1A54002926D057
:10D6A000019B049C1B19079EB5186C787618777837
:10D6B0006F7074704C1E561CA64218D2AE785C185F
:10D6C000A778AF70A6708E1E971CB7420FD2EE7867
:10D6D0006778EF706670CC1ED61CA64207D22C79F4
:10D6E0005E5C2E715C54091F121D8A42DBD3049CC0
:10D6F00020180B9940182021029181705D21417002
:10D700000027C7700798FDF760FB059004197F2C70
:10D71000DA4D089E24D844200B9908557F20001B21
:10D72000052800D30520D54A11184D1C002817D014
:10D730000B9800192F214170911C8D4210D0482167
:10D740008170D11C8D420BD04521C170111D8D42BD
:10D7500006D058210171511D8D4201D002994171AD
:10D760000698002804D19322C548C649FBF7A8FAB9
:10D77000C248281A00197F2826D8069C2278002A39
:10D7800021460B9BC04D2AD01918CA55E21955786D
:10D79000002D1CD0C3197E2B19D8CC196570957833
:10D7A000002D16D07D2B14D8A570D578002D12D061
:10D7B0007C2B10D8E57012793F1D002A069C01D001
:10D7C0007C2BE2D3E11908E0069C214605E0511CC0
:10D7D00003E0911C00E0D11C069C0B9BAA4D091B89
:10D7E00008187F2829460A9F09D83A2119547E280B
:10D7F00004D81918029A4A70A91C00E0691C401B41
:10D800001C4645180C9BD8190790401E00906019C3
:10D81000802421469DA2FDF7CBFA802800D8441928
:10D82000002F64D0002503E0611A0C18BD425ED0C1
:10D830000C982818B0420AD209990B5C0DA808214F
:10D8400096A2FDF7B5FA0DA87F2C08D93FE00DA8E8
:10D85000082291A1FDF7E4FA0DA87F2C37D80378B0
:10D86000002B34D00B98011900200B540DAA12186C
:10D870005678002E1FD022187E2A1CD80B185E70F6
:10D880000DAE3618B678002E19D07D2A17D89E70A6
:10D890000DAE3618F678002E15D07C2A13D8DE701F
:10D8A0000DAB1B181B79001D002B01D07C2ADCD38B
:10D8B0000DA908180AE00DA90818401C06E00DA9DA
:10D8C0000818801C02E00DA90818C01C089E0DA9AC
:10D8D000401A04196D1C6807A8D17F2C71490846AD
:10D8E000A2D820200B9908556E49481C9CE77F2C34
:10D8F0006D4B19460FD820200B9A10557F2C04D160
:10D900001946491C7F2C04D105E0591C491C7F2C69
:10D9100001D012195070E01A4518002F63D000276B
:10D920001AE0C0469C280020B5FA0008756C6F67A5
:10D930005F68657864756D7000000000E6020000A5
:10D9400078E900080DA90818441C0DA8281A051923
:10D950007F1C0A98874246D00C983818B042F7D2FC
:10D9600009990B5C184620385F2800D32E230DAC94
:10D97000082120464DA2FDF71BFA7F2DE5D823781C
:10D98000002BE2D00B98411900200B540DAA12185D
:10D990005478002CD6D02A187E2AD3D80B185C7065
:10D9A0000DAC2418A478002C15D07D2A13D89C70B7
:10D9B0000DAC2418E478002C11D07C2A0FD8DC7030
:10D9C0000DAB1B181B79001D002B01D07C2ADCD36A
:10D9D0000DA90C18B9E70DA90818841CB5E70DA905
:10D9E0000818C41CB1E7904C2046FDF7EEF9401929
:10D9F000812804D32046FDF7E8F980210D1A7F2DF8
:10DA00000A9F00D9FFE50D200B99485586487F2DC8
:10DA100000D0401C441C7F2D00D1F4E50B9949191E
:10DA20000A224A70EFE5FDF743FE002800D1D5E554
:10DA3000114808300021C943FCF750FB0694002E22
:10DA400000D0D4E50C484068002808D0FBF7F6FF6A
:10DA5000002806D0BC2008490858F2F74FFB0FB049
:10DA6000F0BDFDF725FE0028F4D003480830FCF790
:10DA70008BFA0FB0F0BDC0469C28002077FA000852
:10DA8000A5FA00082BFB000874FA0008253034586A
:10DA90002D253034583A20002020200025303258DF
:10DAA0002000000081EE00086AEE000825630000F7
:10DAB000B0B5094D2868002801D00020B0BD284627
:10DAC000083006A101242246FCF728FA00206863EA
:10DAD0002C606C600020B0BD9C280020756C6F67C6
:10DAE0000000000010B582B004AC0194009400F076
:10DAF00003F802B010BD0000F0B585B01E46174611
:10DB00000D4604908D20840000290AD0002E0FD0ED
:10DB10000498082814D2424C2068002819D105B076
:10DB2000F0BD3B483B492246FBF7CAF8002EEFD137
:10DB3000621C39483749FBF7C3F804980828EAD330
:10DB4000E21C36483349FBF7BBF8354C2068002807
:10DB5000E5D0FBF773FF002803972F46254604D036
:10DB6000C0356068002804D116E0383560680028A8
:10DB700012D0FBF763FF002804D0F2F7BBFABC21F8
:10DB8000605009E0FDF794FD0028F6D020460830EB
:10DB90000021C943FCF7A2FA0A99224A1078012809
:10DBA00009D13046FBF766FF0398012819D11E48BA
:10DBB000FBF760FF15E001201070009601912846E8
:10DBC0000295049D29463A46039BFFF75BFA0090B5
:10DBD0000026284639463246029BF7F749FE11488F
:10DBE0000670606800289AD0FBF728FF002805D04F
:10DBF000BC202058F2F782FA05B0F0BDFDF758FDC1
:10DC00000028F5D008342046FCF7BEF905B0F0BD79
:10DC1000B1FA00081EFB000813FB00088DFA00088B
:10DC20009C280020E029002078E9000880B5FDF755
:10DC300065F8002080BD000007200649012206A3E8
:10DC4000FFF750FF094C0A4D25607D20C000FDF70D
:10DC5000DFFCF9E7C0ED00087764675F7468726500
:10DC600061645F656E7472790000000000300040EE
:10DC7000AAAA00002021020C01D010211046020A9D
:10DC800001D010460839020901D01046091F820848
:10DC900001D01046891E420801D0881E7047081A1C
:10DCA00070470000004870470000002001480068ED
:10DCB000704700000000002002E008C8121F08C1E1
:10DCC000002AFAD170477047002001E001C1121FFD
:10DCD000002AFBD17047000001490860704700002E
:10DCE0000000002030380A2801D2012070470020AF
:10DCF000704730B583B00446FFF7D8FF05460020D3
:10DD0000009002460190012321466846F2F7EEFD9D
:10DD10002846FFF7E1FF0199009803B030BD0040AD
:10DD200040404040404040404141414141404040EE
:10DD3000404040404040404040404040404040051E
:10DD40000202020202020202020202020202022095
:10DD50002020202020202020200202020202020295
:10DD600090909090909010101010101010101010B3
:10DD700010101010101010101010020202020202F7
:10DD80008888888888880808080808080808080813
:10DD900008080808080808080808020202024000EB
:10DDA0001FDD000800000100020001000300010067
:10DDB0000200010004000100020001000300010054
:10DDC0000200010005000100020001000300010043
:10DDD0000200010004000100020001000300010034
:10DDE0000200010006000100020001000300010022
:10DDF0000200010004000100020001000300010014
:10DE00000200010005000100020001000300010002
:10DE100002000100040001000200010003000100F3
:10DE200002000100070001000200010003000100E0
:10DE300002000100040001000200010003000100D3
:10DE400002000100050001000200010003000100C2
:10DE500002000100040001000200010003000100B3
:10DE600002000100060001000200010003000100A1
:10DE70000200010004000100020001000300010093
:10DE80000200010005000100020001000300010082
:10DE90000200010004000100020001000300010073
:10DEA00002000100B14E00088D4F0008254F000808
:10DEB0000000000000000000000000000000000062
:10DEC000D3FA00080000000000000000C7FA0008B4
:10DED000CFFA000800000000CBFA000800000000A4
:10DEE0007BEF000837EF000892EE0008BAEE00085A
:10DEF000DBEE000885EE00080CEF0008FDEE0008E0
:10DF0000EBEF000819EF000810F00008F3EF00082D
:10DF1000FFEF0008C5EE000807F000085DEF0008FD
:10DF2000D5EF000844EF00086EEF0008A5EF0008E9
:10DF30008CEF00082AEF0008BAEF0008C5EF0008D0
:10DF4000E6EE000852EF0008AFEE0008A4EE00086D
:10DF5000F2EE0008D0EE00089AEF00080100000081
:10DF60000200000004000000080000001000000093
:10DF700020000000400000008000000000010001BF
:10DF80008000800080008000010003030202020282
:10DF9000017B78767472707E00F6000800F000084D
:10DFA00000EC000800E8000800E4000800E00008B9
:10DFB00000FC00085F5F636D645F53797374656D87
:10DFC0005F5265736574002253797374656D5F5297
:10DFD0006573657422005F5F636D645F4253505FD9
:10DFE0005274635F4461746554696D655F4366672D
:10DFF000002220424344E6A0BCE5BC8FE8BE93E586
:10E0000085A520525443E697A5E69C9FE697B6E97E
:10E0100097B4E9858DE7BDAE3A792C6D2C642C68F8
:10E020002C6D2C732C772022005F5F636D645F542E
:10E030004553545F466C6173685F57726974655FDE
:10E040005265636F72640022544553545F466C619D
:10E0500073685F57726974655F5265636F7264229B
:10E06000005F5F636D645F544553545F466C61733A
:10E07000685F526561645F5265636F726400225429
:10E080004553545F466C6173685F526561645F52CB
:10E0900065636F7264220068656C6C6F00736179F0
:10E0A0002068656C6C6F20776F726C6400766572A7
:10E0B00073696F6E0073686F772052542D546872C5
:10E0C0006561642076657273696F6E20696E666F34
:10E0D000726D6174696F6E005F5F636D645F76651A
:10E0E0007273696F6E0073686F772052542D546895
:10E0F000726561642076657273696F6E20696E6601
:10E100006F726D6174696F6E006C6973745F7468AF
:10E1100072656164006C697374207468726561640F
:10E12000005F5F636D645F6C6973745F74687265D0
:10E130006164006C69737420746872656164006C5A
:10E140006973745F73656D006C6973742073656DBA
:10E150006170686F726520696E2073797374656D84
:10E16000005F5F636D645F6C6973745F73656D00FE
:10E170006C6973742073656D6170686F7265206976
:10E180006E2073797374656D006C6973745F657666
:10E19000656E74006C697374206576656E742069B1
:10E1A0006E2073797374656D005F5F636D645F6C7F
:10E1B0006973745F6576656E74006C69737420654D
:10E1C00076656E7420696E2073797374656D006C6A
:10E1D0006973745F6D75746578006C697374206D14
:10E1E0007574657820696E2073797374656D005F4E
:10E1F0005F636D645F6C6973745F6D7574657800DF
:10E200006C697374206D7574657820696E207379FC
:10E210007374656D006C6973745F6D61696C626FB6
:10E2200078006C697374206D61696C20626F78206E
:10E23000696E2073797374656D005F5F636D645FF1
:10E240006C6973745F6D61696C626F78006C69737F
:10E2500074206D61696C20626F7820696E2073791B
:10E260007374656D006C6973745F6D736771756548
:10E270007565006C697374206D65737361676520E3
:10E28000717565756520696E2073797374656D00AD
:10E290005F5F636D645F6C6973745F6D73677175E5
:10E2A000657565006C697374206D6573736167656E
:10E2B00020717565756520696E2073797374656D5D
:10E2C000006C6973745F74696D6572006C69737456
:10E2D0002074696D657220696E2073797374656D41
:10E2E000005F5F636D645F6C6973745F74696D6513
:10E2F00072006C6973742074696D657220696E2098
:10E3000073797374656D006C6973745F64657669A5
:10E310006365006C69737420646576696365206960
:10E320006E2073797374656D005F5F636D645F6CFD
:10E330006973745F646576696365006C69737420E2
:10E3400064657669636520696E2073797374656DA1
:10E35000006C697374006C69737420616C6C207359
:10E36000796D626F6C20696E2073797374656D00CE
:10E370005F5F636D645F68656C700052542D546814
:10E3800072656164207368656C6C2068656C702EC2
:10E39000005F5F636D645F7073004C697374207419
:10E3A00068726561647320696E2074686520737992
:10E3B0007374656D2E005F5F636D645F6672656583
:10E3C0000053686F7720746865206D656D6F727992
:10E3D00020757361676520696E20746865207379A4
:10E3E0007374656D2E006C6973745F6D656D006C80
:10E3F000697374206D656D6F7279207573616765DF
:10E4000020696E666F726D6174696F6E0000000046
:10E4100000000000000000500100000001000000AA
:10E420000000005002000000020000000000005048
:10E43000040000000300000000000050080000007D
:10E440000400000000000050100000000500000063
:10E4500000000050200000000600000000000050F6
:10E460004000000007000000000000508000000095
:10E47000080000000000005000010000090000003A
:10E4800000000050000200000A00000000000050E0
:10E49000000400000B000000000000500008000015
:10E4A0000C00000000000050001000000D000000F3
:10E4B00000000050002000000E000000000000508E
:10E4C000004000000F00000000000050008000002D
:10E4D00010000000000400500100000011000000C6
:10E4E0000004005002000000120000000004005070
:10E4F00004000000130000000004005008000000A9
:10E50000140000000004005010000000150000007E
:10E51000000400502000000016000000000400501D
:10E5200040000000170000000004005080000000C0
:10E530001800000000040050000100001900000055
:10E5400000040050000200001A0000000004005007
:10E55000000400001B000000000400500008000040
:10E560001C00000000040050001000001D0000000E
:10E5700000040050002000001E00000000040050B5
:10E58000004000001F000000000400500080000058
:10E5900020000000000800500100000021000000E1
:10E5A0000008005002000000220000000008005097
:10E5B00004000000230000000008005008000000D4
:10E5C000240000000008005010000000250000009A
:10E5D0000008005020000000260000000008005045
:10E5E00040000000270000000008005080000000EC
:10E5F0002800000000080050000100002900000071
:10E6000000080050000200002A000000000800502E
:10E61000000400002B00000000080050000800006B
:10E620002C00000000080050001000002D00000029
:10E6300000080050002000002E00000000080050DC
:10E64000004000002F000000000800500080000083
:10E6500030000000000C00500100000031000000FC
:10E66000000C00500200000032000000000C0050BE
:10E670000400000033000000000C005008000000FF
:10E6800034000000000C00501000000035000000B5
:10E69000000C00502000000036000000000C00506C
:10E6A0004000000037000000000C00508000000017
:10E6B00038000000000C005000010000390000008C
:10E6C000000C0050000200003A000000000C005056
:10E6D000000400003B000000000C00500008000097
:10E6E0003C000000000C0050001000003D00000045
:10E6F000000C0050002000003E000000000C005004
:10E70000004000003F000000000C005000800000AE
:10E71000416C61726D206576656E74206973206E40
:10E720006F7420696E697469616C697A6564210A25
:10E7300000E887AAE6A380E6A8A1E5BC8F0A00E46A
:10E74000BCA0E6849FE599A8E5A4B1E69588E6A873
:10E75000A1E5BC8F0A00E69585E99A9CE681A2E5D1
:10E76000A48DE6A8A1E5BC8F0A00E69585E99A9CF0
:10E77000E6A8A1E5BC8F0A00E68E89E794B5E6A875
:10E78000A1E5BC8F0A00313030302C313030300000
:10E790003530302C31303030003530302C353030A1
:10E7A0000069203D202564006D61696E00616C6127
:10E7B000726D5F6576656E7400456E74657220419A
:10E7C0006E616C6F675761746368646F6720496E30
:10E7D000746572727570740067657420737061631C
:10E7E00065206661696C0D0A0048525F4765744494
:10E7F0006174614672616D65204661696C210048F3
:10E80000525F476574446174614672616D6520535F
:10E8100075636365737321006B416C61726D526542
:10E82000636F726428256429006B4661756C7452AD
:10E8300065636F726428256429006B416C61726D99
:10E840005263795265636F72642825642900687287
:10E850005F72785F73656D006273705F6872006BE2
:10E860004E756D4F665265636F72647300726561B9
:10E8700064203A68725F73746172745F6164647279
:10E88000203D202523782C20696E6465785F6164C3
:10E8900064723A202523782C2068725F6E756D3A79
:10E8A0002025642C2068725F706167653A25642CAE
:10E8B00020726561645F64617461203A20202523C1
:10E8C000580D0A00466C6173685F4765744D617846
:10E8D0004E756D28282564295F5265636F726473D5
:10E8E000282564292053756D5F436865636B28256F
:10E8F00023582920213D20636865636B5F73756D24
:10E9000028252358292C696E6465785F61646472D8
:10E91000203A2523580D0A00466C6173685F4572E2
:10E9200061736550616765206661696C65640D0A95
:10E9300000466163746F727954696D652063686520
:10E94000636B5F73756D206572726F720D0A00469E
:10E950006163746F727954696D65206973206E6F9D
:10E9600074207365740D0A006572726F725F706156
:10E970006765203D202523780D0A00466C61736889
:10E980005F476574496E6465785F506F73204572A8
:10E99000726F72210072656164203A68725F7374ED
:10E9A0006172745F61646472203D202523782C209D
:10E9B000696E6465785F616464723A202523782CFF
:10E9C0002068725F6E756D3A2025642C2068725F36
:10E9D000706167653A25642C20726561645F6461CB
:10E9E0007461203A20202523580077726974653AB3
:10E9F00068725F73746172745F61646472203D2039
:10EA00002523782C20696E6465785F616464723AAE
:10EA1000202523782C2068725F6E756D3A2025645E
:10EA20002C2068725F706167653A25642C207772CC
:10EA30006974655F64617461203A2025235800463B
:10EA40006C6173685F57726974655F282564295229
:10EA500065636F72643A253034642D253032642D3D
:10EA60002530326420253032643A253032642C203F
:10EA7000636865636B5F73756D203A2025235800CA
:10EA8000496E6465785F4672616D652E68725F6974
:10EA90006E6465785F61646472203D2068725F73A4
:10EAA000746172745F616464725B7265636F7264D7
:10EAB0005D202B2069202A20464C4153485F50415D
:10EAC00047455F425954455F53495A45202D2048D8
:10EAD000525F5245434F52445F4652414D455F4C51
:10EAE000454E203D20252358004572617365205016
:10EAF00061676520256400457261736550616765D3
:10EB000020256400696E646578206E756D20282567
:10EB10006429203E2041637475616C2073746F72A8
:10EB2000616765206E756D20256400466C617368B1
:10EB30005F526561645F282564295265636F726462
:10EB4000282564293A253034642D253032642D255A
:10EB50003032642C253032643A2530326400466C01
:10EB60006173685F526561645F466163746F727957
:10EB700054696D653A253034642D253032642D2575
:10EB80003032642C253032643A25303264004253EE
:10EB9000505F466C6173685F50726F6772616D5F42
:10EBA000496E666F50616765206661696C656400D7
:10EBB0006273705F666C61736800464C45585F42D3
:10EBC000544E5F50524553535F444F55424C455F3E
:10EBD000434C49434B0A00464C45585F42544E5FF4
:10EBE00050524553535F53484F52545F5354415210
:10EBF000540A00555345525F425554544F4E5F30AE
:10EC000000464C45585F42544E5F50524553535F47
:10EC10004C4F4E475F484F4C4400464C45585F426E
:10EC2000544E5F50524553535F4E4F4E4500464C35
:10EC300045585F42544E5F50524553535F444F55C1
:10EC4000424C455F434C49434B00464C45585F425C
:10EC5000544E5F50524553535F434C49434B00461B
:10EC60004C45585F42544E5F50524553535F524596
:10EC7000504541545F434C49434B00464C45585F17
:10EC800042544E5F50524553535F444F574E0046D7
:10EC90004C45585F42544E5F50524553535F4C4F62
:10ECA0004E475F484F4C445F555000464C45585FB7
:10ECB00042544E5F50524553535F4C4F4E475F5541
:10ECC0005000464C45585F42544E5F505245535396
:10ECD0005F53484F52545F555000464C45585F4271
:10ECE000544E5F50524553535F4C4F4E475F535401
:10ECF00041525400464C45585F42544E5F50524575
:10ED000053535F53484F52545F535441525400552C
:10ED10005345525F425554544F4E5F4D4158004643
:10ED20004C45585F42544E5F50524553535F4D41DE
:10ED300058006273705F627574746F6E00353030A6
:10ED40002C3135303000786F725F76616C75653AC2
:10ED50002523582C20636865636B5F76616C75654D
:10ED60003A2523580D0A00636865636B206572724B
:10ED70006F720D0A00457874726163745F53656E3B
:10ED8000736F7244617461206661696C65642E2ED4
:10ED90002E002530325800412B253673202536733E
:10EDA000202538732025367320422B2536732025E5
:10EDB000327320253273006273705F756172740064
:10EDC0006273705F77646700495744475F466565C3
:10EDD000645F496E697400252D2A2E2A7320252D23
:10EDE000382E2A7320253034642025640A00252D0E
:10EDF0002A2E2A7320252D32307320252D38640ABF
:10EE00000064656163746976617465640A00252D28
:10EE10002A2E7320707269202073746174757320B8
:10EE20002020202020737020202020207374616314
:10EE30006B2073697A65206D617820757365642035
:10EE40006C656674207469636B20206572726F72E2
:10EE50000A0020696E69742020200020636C6F73A3
:10EE600065202000207265616479202000252D2A0C
:10EE70002E2A7320307825303878203078253038A5
:10EE80007820002D00525443002073757370656E16
:10EE900064004E6574776F726B20496E746572669C
:10EEA00061636500444143204465766963650041C0
:10EEB000444320446576696365004D5444204465AD
:10EEC000766963650053504920446576696365003F
:10EED00050574D204465766963650043414E204498
:10EEE000657669636500574C414E204465766963D9
:10EEF0006500574454204465766963650047726134
:10EF0000706869632044657669636500536F756E48
:10EF100064204465766963650055534220536C61F3
:10EF200076652044657669636500546F7563682073
:10EF300044657669636500426C6F636B2044657657
:10EF400069636500506F7274616C20446576696313
:10EF5000650050696E2044657669636500504D20F8
:10EF600050736575646F2044657669636500546904
:10EF70006D657220446576696365004368617261FE
:10EF800063746572204465766963650053656E73CA
:10EF90006F7220446576696365004275732044652D
:10EFA00076696365004D697363656C6C616E656F4E
:10EFB00075732044657669636500506879204465FF
:10EFC0007669636500536563757269747920446579
:10EFD000766963650050697065002072756E6E69B0
:10EFE0006E6700556E6B6E6F776E0049324320423C
:10EFF000757300555342204F544720427573005398
:10F00000504920427573005344494F2042757300A4
:10F0100055534220486F7374204275730052542D2B
:10F02000546872656164207368656C6C20636F6DF1
:10F030006D616E64733A0A00252D313673202D20E0
:10F0400025730A005F5F636D645F0008001B5B321D
:10F050004B0D006D7368200066696E736820007345
:10F0600068656C6C20213D2052545F4E554C4C001D
:10F0700025630066696E73685F7365745F70726F95
:10F080006D70745F6D6F646500257325730074691E
:10F090006420213D2052545F4E554C4C0072745FE9
:10F0A0006170706C69636174696F6E5F696E6974B9
:10F0B0000046756E6374696F6E5B25735D207368BF
:10F0C000616C6C206E6F74206265207573656420BE
:10F0D000696E204953520A0072745F7468726561E8
:10F0E000645F69646C655F65786375746500467517
:10F0F0006E6374696F6E5B25735D207368616C6C01
:10F10000206E6F7420626520757365642062656689
:10F110006F7265207363686564756C6572207374C3
:10F120006172740A0073697A6520213D2030006D98
:10F130006220213D2052545F4E554C4C0073656D4A
:10F1400020213D2052545F4E554C4C006D712021C2
:10F150003D2052545F4E554C4C0062756666657298
:10F1600020213D2052545F4E554C4C006576656E13
:10F170007420213D2052545F4E554C4C006D7574E7
:10F18000657820213D2052545F4E554C4C007661ED
:10F190006C7565203C20307831303030305500724D
:10F1A000745F6576656E745F73656E640072745F1C
:10F1B00073656D5F74616B650072745F6D75746506
:10F1C000785F74616B650072745F6F626A65637407
:10F1D0005F6765745F74797065282673656D2D3E71
:10F1E000706172656E742E706172656E7429203D57
:10F1F0003D2052545F4F626A6563745F436C617374
:10F20000735F53656D6170686F72650072745F73D0
:10F21000656D5F72656C656173650072745F6D75B5
:10F220007465785F72656C656173650072745F6D9B
:10F23000625F6372656174650072745F73656D5FB0
:10F240006372656174650072745F6D715F6372658E
:10F250006174650072745F6576656E745F63726574
:10F260006174650072745F6D757465785F63726553
:10F270006174650072745F6D625F64656C6574656E
:10F280000072745F73656D5F64656C6574650072B0
:10F29000745F6D715F64656C6574650072745F6541
:10F2A00076656E745F64656C6574650072745F6D1D
:10F2B000757465785F64656C6574650072745F6F02
:10F2C000626A6563745F6765745F74797065282628
:10F2D0006D712D3E706172656E742E706172656E17
:10F2E0007429203D3D2052545F4F626A6563745F0C
:10F2F000436C6173735F4D657373616765517565C9
:10F3000075650072745F6D625F6465746163680047
:10F3100072745F73656D5F646574616368007274B5
:10F320005F6D715F6465746163680072745F6576B8
:10F33000656E745F6465746163680072745F6D7597
:10F340007465785F6465746163680072745F6D6290
:10F350005F636F6E74726F6C0072745F73656D5F64
:10F36000636F6E74726F6C0072745F6D715F636F48
:10F370006E74726F6C0072745F6576656E745F6335
:10F380006F6E74726F6C0072745F6D757465785F08
:10F39000636F6E74726F6C0072745F6D625F736521
:10F3A0006E645F776169740072745F6D715F73651D
:10F3B0006E645F776169740072745F73656D5F6915
:10F3C0006E69740072745F6D715F757267656E74DB
:10F3D0000072745F6F626A6563745F6765745F74FF
:10F3E00079706528266576656E742D3E706172654C
:10F3F0006E742E706172656E7429203D3D205254EA
:10F400005F4F626A6563745F436C6173735F4576D7
:10F41000656E740072745F6D625F72656376007210
:10F42000745F6D715F726563760072745F65766597
:10F430006E745F726563760072745F6F626A656393
:10F44000745F6765745F7479706528266D7574657F
:10F45000782D3E706172656E742E706172656E7487
:10F4600029203D3D2052545F4F626A6563745F43BB
:10F470006C6173735F4D757465780072745F6F6251
:10F480006A6563745F6765745F7479706528266D5B
:10F49000622D3E706172656E742E706172656E745D
:10F4A00029203D3D2052545F4F626A6563745F437B
:10F4B0006C6173735F4D61696C426F780028727480
:10F4C0005F75626173655F7429282872745F75695E
:10F4D0006E74385F74202A296D656D202B20534986
:10F4E0005A454F465F5354525543545F4D454D293D
:10F4F00020252052545F414C49474E5F53495A459D
:10F50000203D3D2030006D656D2D3E6D6167696366
:10F51000203D3D20484541505F4D414749430072E1
:10F52000745F7265616C6C6F630072745F6D616CA7
:10F530006C6F63002872745F75696E74385F742035
:10F540002A29726D656D203E3D202872745F7569B1
:10F550006E74385F74202A29686561705F707472F8
:10F56000202626202872745F75696E74385F7420B7
:10F570002A29726D656D203C202872745F75696E52
:10F5800074385F74202A29686561705F656E640055
:10F590002872745F75626173655F74296D656D2093
:10F5A0002B2053495A454F465F5354525543545F9D
:10F5B0004D454D202B2073697A65203C3D202872F3
:10F5C000745F75626173655F7429686561705F65FA
:10F5D0006E640072745F6672656500706C75675F5B
:10F5E000686F6C65730072745F73797374656D5FB7
:10F5F000686561705F696E697400696E666F726DCF
:10F600006174696F6E20213D2052545F4E554C4C01
:10F61000006F626A65637420213D2052545F4E552D
:10F620004C4C0072745F6F626A6563745F66696EEA
:10F63000640072745F6F626A6563745F616C6C6FA3
:10F64000636174650072745F6F626A6563745F649E
:10F65000656C6574650072745F6F626A6563745F80
:10F66000696E69740074687265616420213D20527E
:10F67000545F4E554C4C0072745F6F626A656374E0
:10F680005F6765745F74797065282872745F6F6254
:10F690006A6563745F742974687265616429203DCA
:10F6A0003D2052545F4F626A6563745F436C6173BF
:10F6B000735F5468726561640072745F7468726528
:10F6C00061645F73757370656E640072745F7468F3
:10F6D000726561645F726573756D650072745F74E5
:10F6E00068726561645F64656C6574650072745FFF
:10F6F0007468726561645F646574616368007274E4
:10F700005F7468726561645F64656C61795F756E72
:10F7100074696C0072745F7468726561645F636FB2
:10F720006E74726F6C0072745F7468726561645F8E
:10F73000736C6565700072745F7468726561645F94
:10F74000737461727475700072745F74687265614D
:10F75000645F696E69740072745F74687265616475
:10F760005F74696D656F75740074696D65722021D1
:10F770003D2052545F4E554C4C0072745F74696D5D
:10F7800065725F64656C6574650072745F74696D41
:10F7900065725F6465746163680072745F74696D3B
:10F7A00065725F636F6E74726F6C0072745F746900
:10F7B0006D65725F73746F700072745F6F626A65FB
:10F7C00063745F6765745F74797065282674696D0A
:10F7D00065722D3E706172656E7429203D3D205228
:10F7E000545F4F626A6563745F436C6173735F5407
:10F7F000696D65720072745F74696D65725F7374B0
:10F800006172740064657620213D2052545F4E552C
:10F810004C4C00546F20696E697469616C697A653B
:10F82000206465766963653A2573206661696C6555
:10F83000642E20546865206572726F7220636F6455
:10F84000652069732025640072745F64657669635E
:10F85000655F726561640072745F6F626A6563748C
:10F860005F6765745F7479706528266465762D3EE0
:10F87000706172656E7429203D3D2052545F4F6265
:10F880006A6563745F436C6173735F446576696333
:10F8900065006B65726E656C2E64657669636500E4
:10F8A00072745F6465766963655F636C6F7365002E
:10F8B00072745F6465766963655F7365745F72789F
:10F8C0005F696E6469636174650072745F64657614
:10F8D0006963655F7365745F74785F636F6D706C87
:10F8E0006574650072745F6465766963655F7772DD
:10F8F0006974650072745F6465766963655F636FE0
:10F900006E74726F6C0072745F6465766963655FB4
:10F910006F70656E0072745F6465766963655F75AC
:10F920006E72656769737465720072745F64657680
:10F930006963655F64657374726F79007374617273
:10F940007475702075617274315F646D615F727877
:10F950005F7468726561642072657475726E203DB3
:10F960002025640075617274315F72785F7468720B
:10F97000656164006472765F7561727400706572AF
:10F980006600506C656173652063616C6C20616713
:10F99000696C655F6C65645F656E765F696E6974DE
:10F9A0002066697273742E006C65642D3E747970E4
:10F9B00065203D3D204147494C455F4C45445F54DF
:10F9C0005950455F44594E414D4943006167696C48
:10F9D000655F6C6564006167696C655F6C65645F39
:10F9E00064796E616D69635F6368616E67655F6CA2
:10F9F000696768745F6D6F6465006167696C655FF6
:10FA00006C65645F7374617469635F6368616E677A
:10FA1000655F6C696768745F6D6F646500616769D5
:10FA20006C655F6C65645F64656C657465006167D7
:10FA3000696C655F6C65645F6765745F6C69676856
:10FA4000745F617272006C65645F6D7478007069D8
:10FA50006E20213D2052545F4E554C4C005F68771C
:10FA60005F70696E2E6F707320213D2052545F4E7F
:10FA7000554C4C003A2000442F4845582000412F57
:10FA800000442F00452F00492F00572F006C65764A
:10FA9000656C203C3D204C4F475F4C564C5F4442C8
:10FAA00047001B5B00737263006261636B656E6489
:10FAB0000074616700756C6F672E696E69745F6FA3
:10FAC0006B001B5B306D0033316D0033326D0033E2
:10FAD000336D0033356D00756C6F675F666F726DE7
:10FAE0006174657200756C6F675F6261636B656EF0
:10FAF000645F726567697374657200756C6F675FC8
:10FB00006261636B656E645F756E7265676973745D
:10FB1000657200666F726D61740064737400756C59
:10FB20006F675F766F757470757400756C6F675F63
:10FB30007374726370790000B7C50008AFC5000820
:10FB40002D990008099A0008B1DA0008ABC5000831
:10FB5000F11F00085940000831220008194A000826
:10FB6000C95000082DD0000835370008A51F00082F
:10FB7000DD1D0008D9130008011F0008ED3F000833
:10FB8000C15A0008F14D0008B3C50008B4DF0008F1
:10FB9000C7DF000831440008D6DF0008F1DF0008A5
:10FBA0004521000829E0000847E00008CD4400088E
:10FBB00061E000087EE000085144000897E000087A
:10FBC0009DE0000821660008ADE00008B5E00008EF
:10FBD0002DDC0008D8E00008E6E000082DDC000875
:10FBE00009E1000815E100089D78000821E10008FE
:10FBF00033E100089D7800083FE1000848E1000873
:10FC00009976000861E1000870E100089976000823
:10FC100089E1000894E10008096B0008A9E10008E7
:10FC2000BAE10008096B0008CFE10008DAE100083A
:10FC300099710008EFE1000800E2000899710008DE
:10FC400015E2000822E20008FD6C00083AE2000814
:10FC50004DE20008FD6C000865E2000873E2000850
:10FC60008D6F000890E20008A4E200088D6F000884
:10FC7000C1E20008CCE20008A97A0008E1E200082D
:10FC8000F2E20008A97A000807E3000813E300087D
:10FC90005967000829E300083BE30008596700089A
:10FCA00051E3000856E30008E166000870E300082D
:10FCB0007BE300081586000891E300089AE300083A
:10FCC0000F570008B6E30008C1E300080557000815
:10FCD000E6E30008EFE30008216F000800FD0008DC
:10FCE0000000002090000000B8DC000890FD000833
:10FCF0009000002080300000C8DC00082950FFFF81
:10FD00000000000001000000010000000024F400D9
:10FD100001000000140000201400002090000000EA
:10FD20000200000024000020240000202800000021
:10FD30000300000034000020340000202C000000EC
:10FD400004000000440000204400002028000000BF
:10FD5000050000005400002054000020380000007E
:10FD60000600000064000020640000204400000041
:10FD7000090000007400002074000020480000000A
:10FD80000A000000840000208400002034000000ED
:04000005080000C12E
:00000001FF
